:100000004BC0000042C2000040C200003EC20000DF
:100010003CC200000C94466238C2000036C20000A8
:1000200034C2000032C200000C943C620C94326274
:100030002CC200002AC2000028C2000026C2000014
:1000400024C2000022C2000020C200001EC2000024
:100050001CC200000C94126318C2000016C20000FB
:1000600014C2000012C2000010C200000EC2000044
:100070000CC200000AC2000008C2000006C2000054
:1000800004C2000002C2000000C20000FEC1000065
:10009000FCC10000FAC1000011241FBECFEFD0E266
:1000A000DEBFCDBF0E9400F0D7C10000076342361B
:1000B000B79BD8A71A39685618AEBAAB558C1D3CF9
:1000C000B7CC5763BD6DEDFD753EF6177231BF00BD
:1000D0000000803F05A84CCDB2D44EB93836A902F5
:1000E0000C50B9918688083CA6AAAA2ABE00000036
:1000F000803F08000000BE922449123EABAAAA2A03
:10010000BECDCCCC4C3E00000080BEABAAAAAA3E1D
:1001100000000000BF000000803F00000000000859
:100120004178D3BB4387D1133D190E3CC3BD4282F6
:10013000AD2B3E68EC8276BED98FE1A93E4C80EFB4
:10014000FFBE01C4FF7F3F0000000000FF004C8A9B
:1001500097509545406BA6D8E4B2282EAE90BF26A6
:10016000B14EE86FD0FBE0709A51862C379845323B
:10017000539D06840D971A8CE61E2E0DB41D401655
:100180009AC591F9F786A142660620AFAE19EE270F
:10019000C2BB0EBAB90AAA95CA45040444C1796A19
:1001A00091EE7D3E2E4C960BA96E5A6A9FF56D0519
:1001B000BB8F808DB4F54FC14AE99E674536394FF4
:1001C00075ADF44CB227A939D78036F7C49C7E6A46
:1001D000605F677992B4DD0E4786CD1A6DC6258AB9
:1001E000F464D953D154DB67F78B22BD5CFEA44D78
:1001F000F9A7590EC57E3BF9BA7D430AD39F6C3BE4
:100200000BDEB2875E3710ECC8A6856546290CF177
:10021000D6BCA38C755E4934200DFAE9D7C7B6A7C2
:10022000988A7C6E6155493D32271D1209FFF6EE12
:10023000E5DDD5CEC6BFB9B2ACA6A09A958F8A85AA
:10024000817C78736F6B6864605D5A56FF59E97DF5
:1002500015B150F39942EE9D4F04BC7632F1B2765F
:100260003B03CC98653405D8AC8259320CE7C4A264
:100270008161432509EDD3B9A089725C46321E0B1A
:10028000F8E6D5C4B4A596887A6D6053473C30260D
:100290001B1108FEF5EDE4DCD4CDC6BFB8B1ABA5AB
:1002A0009F99948F8A85807C77736F6B6763605D9D
:1002B000595653504D4A484543403E3C3A383634EF
:1002C00032302E2D2B2A282725242321201F1E1DC6
:1002D0001C1B1A19181716161514131312111110C6
:1002E0000F0F0E0E0D0D0C0C0B0B0B0A0A09090952
:1002F0000808080807070706060606060505050597
:1003000005040404040404030303030303030302B6
:1003100002020202020202020202010101010101C3
:1003200001010101010101010101010101000000C0
:1003300000000000000000000000000000000000BD
:10034000000000000000000000000000FF0C0B0B8C
:100350000B0A0A090909080808080707070606061C
:100360000606050505050504040404040403030347
:100370000303030303020202020202020202020258
:10038000010101010101010101010101010101015D
:10039000010101000000000000000000000000005A
:1003A000000000000000000000000000000000004D
:1003B000000000000000000000000000000000003D
:1003C000000000000000000000000000000000002D
:1003D000000000000000000000000000000000001D
:1003E000000000000000000000000000000000000D
:1003F00000000000000000000000000000000000FD
:1004000000000000000000000000000000000000EC
:1004100000000000000000000000000000000000DC
:1004200000000000000000000000000000000000CC
:1004300000000000000000000000000000000000BC
:1004400000000000000000000000000011241FBE9A
:10045000CFEFD0E2DEBFCDBF18E1AEE5B9E001C01D
:100460001D92AF3FB107E1F719E0A0E0B1E0E0E392
:10047000FEED00E00BBF02C007900D92AE35B10754
:10048000D9F70E944B630C94166FBACD2F923F920E
:100490004F925F926F927F928F929F92AF92BF9294
:1004A000CF92DF92EF92FF920F931F93CF93DF9340
:1004B00000D000D000D0CDB7DEB78EEA9EE00E941B
:1004C00054224090DF0E5090E00E20916B0F20FFE1
:1004D00015C025FD02C00C94130E420124FD0FC06F
:1004E0008091C40E9091C50E95958795480E591E22
:1004F00021FD07C0C12CD12C76010BC0420121FF88
:10050000F9CFC090C40ED090C50EEE24D7FCE09475
:10051000FE2C00918C0F10918D0F20E030E01058D0
:10052000210931098091670F882311F40C940F0E73
:1005300080919E0F90919F0FA0E0B0E09058A1098C
:10054000B109B7FF02C00C946910B595A7959795AE
:1005500087959E838D832FB72983F89486EB9CE043
:100560000E941D212090DA0C3090DB0CAA2497FC0D
:10057000A094BA2C662457FC6094762C8091F00EDF
:100580009091F10EB301A201480F591F611D711D19
:10059000DB01CA01009751E0A507B10524F08FEFF8
:1005A0009FEFA0E0B0E0B7FF02C00C941D0E0E94C8
:1005B000E01246EC41BB469A31E035B925E428B952
:1005C00050EF5BB992EA9EB987E881BB00C000C0DA
:1005D00041BB469A35B928B960ED6BB99EB981BB6C
:1005E00000C000C041BB469A35B928B95BB99EB975
:1005F00081BB6D817E819101AA27629FB12D73031A
:10060000C001369FB00D811D9A1F72039A0BB00D69
:10061000811D9A1F1124AA2797FDA095BA2F880D36
:10062000991DAA1DBB1D2091E40E3091E50E820F8D
:10063000931FA11DB11D009731E0A307B10524F060
:100640008FEF9FEFA0E0B0E0B7FF02C00C94270E41
:100650000E94E01246EC41BB469A31E035B921E4F4
:1006600028B950EF5BB990EA9EB987E881BB00C01A
:1006700000C041BB469A35B928B960ED6BB99EB947
:1006800081BB00C000C041BB469A35B928B95BB9EF
:100690009EB981BBA101AA27049FB12D1503C001FA
:1006A000509FB00D811D9A1F14039A0BB00D811D30
:1006B0009A1F1124AA2797FDA095BA2F8C0D9D1D76
:1006C000AE1DBF1D2091FC0E3091FD0E820F931FB9
:1006D000A11DB11D009751E0A507B10524F08FEFD2
:1006E0009FEFA0E0B0E0B7FF02C00C94220E0E9482
:1006F000E01226EC21BB469A2224239425B891E4EB
:1007000098B930EF3BB982EA8EB947E8342E31BA56
:1007100000C000C021BB469A25B898B940EE4BB93D
:100720008EB931BA00C000C021BB469A25B898B92D
:100730003BB98EB931BA82EB9DE02B833C830E949A
:100740001D218091D60D9091D70D0E94E0122B8132
:1007500021BB469A25B895E498B93C813BB980EA1B
:100760008EB931BA00C000C021BB469A25B898B9ED
:1007700040EB4BB98EB931BA00C000C021BB469ADC
:1007800025B898B93BB98EB931BA69816FBF3FB608
:10079000F89480EE9CE00E941D212091040D309180
:1007A000050D3A8329838091F20E9091F30EB301E7
:1007B000A201480F591F611D711DDB01CA0100977D
:1007C00051E0A507B10524F08FEF9FEFA0E0B0E066
:1007D000B7FF02C00C94360E0E94E01246EC41BBFB
:1007E000469A31E035B927E428B950EF5BB992EA6F
:1007F0009EB987E881BB00C000C041BB469A35B9AD
:1008000028B960ED6BB99EB981BB00C000C041BB87
:10081000469A35B928B95BB99EB981BB6D817E8195
:1008200029813A81AA27629FB12D7303C001369FA7
:10083000B00D811D9A1F72039A0BB00D811D9A1F76
:100840001124AA2797FDA095BA2F880D991DAA1DDE
:10085000BB1D2091E60E3091E70E820F931FA11D64
:10086000B11D009731E0A307B10524F08FEF9FEF92
:10087000A0E0B0E0B7FF02C00C94310E0E94E0127D
:1008800046EC41BB469A31E035B923E428B950EF34
:100890005BB990EA9EB987E881BB00C000C041BB4C
:1008A000469A35B928B960ED6BB99EB981BB00C0D5
:1008B00000C041BB469A35B928B95BB99EB981BB26
:1008C00049815A81AA27049FB12D1503C001509F69
:1008D000B00D811D9A1F14039A0BB00D811D9A1F34
:1008E0001124AA2797FDA095BA2F8C0D9D1DAE1D32
:1008F000BF1D2091FE0E3091FF0E820F931FA11D90
:10090000B11D009751E0A507B10524F08FEF9FEFCF
:10091000A0E0B0E0B7FF02C00C942C0E0E94E012E1
:1009200046EC41BB469A31E035B923E428B950EF93
:100930005BB992EA9EB987E881BB00C000C041BBA9
:10094000469A35B928B960EE6BB99EB981BB00C033
:1009500000C041BB469A35B928B95BB99EB981BB85
:100960008091E00D9091E10DA091E20DB091E30D29
:100970008B2F9927AA27BB27892B8A2B8B2B21F01A
:100980008CED9DE00E9414258091050E823009F4C3
:10099000ACC708F0A4C7813011F40C94E80C80E0D7
:1009A00090E06091FE0D7091FF0D0E94D33E20916A
:1009B000FC0D3091FD0D280F391F3093010E20934F
:1009C000000E8091DC0D9091DD0DA091DE0DB091B7
:1009D000DF0D4091E00D5091E10D6091E20D7091BD
:1009E000E30D840F951FA61FB71F8093E00D909312
:1009F000E10DA093E20DB093E30DC9010E94E01256
:100A000046EC41BB469A31E035B927E428B950EFAE
:100A10005BB990EA9EB987E881BB00C000C041BBCA
:100A2000469A35B928B960EB6BB99EB981BB00C055
:100A300000C041BB469A35B928B95BB99EB981BBA4
:100A40003FBE3FB73983F89480910E0D90910F0D02
:100A5000A091100DB091110D8B2F9927AA27BB27BC
:100A6000892B8A2B8B2B09F074C78091330D823030
:100A700009F422C708F01AC7813009F4E0C780E002
:100A800090E060912C0D70912D0D0E94D33E20902E
:100A90002A0D30902B0D280E391E30922F0D2092EA
:100AA0002E0D80910A0D90910B0DA0910C0DB0911F
:100AB0000D0D40910E0D50910F0D6091100D709124
:100AC000110D840F951FA61FB71F80930E0D9093D5
:100AD0000F0DA093100DB093110D8091F40E909115
:100AE000F50EB301A201480F591F611D711D41157B
:100AF000510581E06807710524F04FEF5FEF60E07A
:100B000070E0DB01CA0177FF02C00C94990D0E94CE
:100B1000E01266EC61BB469A51E055B941E448B930
:100B200070EF7BB990EA9EB987E881BB00C000C036
:100B300061BB469A55B948B9E0EEEBB99EB981BBA5
:100B400000C000C061BB469A55B948B97BB99EB98F
:100B500081BB2D813E81B101AA27269FB12D37038C
:100B6000A001729FB00D411D5A1F36035A0BB00DE4
:100B7000411D5A1F1124662757FD6095762F480D99
:100B8000591D6A1D7B1D8091E80E9091E90E480F5A
:100B9000591F611D711D4115510581E068077105DF
:100BA00024F04FEF5FEF60E070E0DB01CA0177FFF8
:100BB00001C0C8C70E94E01266EC61BB469A51E0D2
:100BC00055B945E448B970EF7BB990EA9EB987E81A
:100BD00081BB00C000C061BB469A55B948B9E0ED81
:100BE000EBB99EB981BB00C000C061BB469A55B944
:100BF00048B97BB99EB981BB9101AA27029FB12D4B
:100C00001303A001309FB00D411D5A1F12035A0B50
:100C1000B00D411D5A1F1124662757FD6095762F90
:100C20004C0D5D1D6E1D7F1D8091000F9091010F79
:100C3000480F591F611D711D4115510531E06307B2
:100C4000710524F04FEF5FEF60E070E0DB01CA0157
:100C500077FD74C70E94E01246EC41BB469A31E032
:100C600035B925E428B950EF5BB992EA9EB987E817
:100C700081BB00C000C041BB469A35B928B960EEBF
:100C80006BB99EB981BB00C000C041BB469A35B963
:100C900028B95BB99EB981BB80910A0E90910B0E69
:100CA000A0910C0EB0910D0E8B2F9927AA27BB2770
:100CB000892B8A2B8B2B09F065C680912F0E8230F1
:100CC00009F4C8C508F0C0C5813009F46AC680E0DF
:100CD00090E06091280E7091290E0E94D33E2091E1
:100CE000260E3091270E280F391F30932B0E20939C
:100CF0002A0E8091060E9091070EA091080EB091D9
:100D0000090E40910A0E50910B0E60910C0E7091DD
:100D10000D0E840F951FA61FB71F80930A0E909388
:100D20000B0EA0930C0EB0930D0EC9010E94E012A1
:100D300046EC41BB469A31E035B921E428B950EF81
:100D40005BB992EA9EB987E881BB00C000C041BB95
:100D5000469A35B928B960EB6BB99EB981BB00C022
:100D600000C041BB469A35B928B95BB99EB981BB71
:100D700039813FBF2FB72983F8948091380D909126
:100D8000390DA0913A0DB0913B0D8B2F9927AA27D1
:100D9000BB27892B8A2B8B2B09F0EAC580915D0D2F
:100DA000823009F470C508F068C5813009F456C670
:100DB00080E090E06091560D7091570D0E94D33EF7
:100DC0002090540D3090550D280E391E3092590D3B
:100DD0002092580D8091340D9091350DA091360DD3
:100DE000B091370D4091380D5091390D60913A0D09
:100DF00070913B0D840F951FA61FB71F8093380D70
:100E00009093390DA0933A0DB0933B0D8091F60E5F
:100E10009091F70EB301A201480F591F611D711D7A
:100E20004115510531E06307710524F04FEF5FEF85
:100E300060E070E0DB01CA0177FD73C60E94E0123A
:100E400066EC61BB469A51E055B943E448B970EF8E
:100E50007BB990EA9EB987E881BB00C000C061BB46
:100E6000469A55B948B9E0EEEBB99EB981BB00C0CE
:100E700000C061BB469A55B948B97BB99EB981BBE0
:100E80006D817E819101AA27629FB12D7303A0011C
:100E9000369FB00D411D5A1F72035A0BB00D411DF4
:100EA0005A1F1124662757FD6095762F480D591D4E
:100EB0006A1D7B1D8091EA0E9091EB0E480F591F21
:100EC000611D711D4115510531E06307710524F065
:100ED0004FEF5FEF60E070E0DB01CA0177FD1DC6F8
:100EE0000E94E01266EC61BB469A51E055B947E4B6
:100EF00048B970EF7BB990EA9EB987E881BB00C022
:100F000000C061BB469A55B948B9E0EDEBB99EB94E
:100F100081BB00C000C061BB469A55B948B97BB9D6
:100F20009EB981BBB101AA27069FB12D1703A0016D
:100F3000709FB00D411D5A1F16035A0BB00D411D75
:100F40005A1F1124662757FD6095762F4C0D5D1DA5
:100F50006E1D7F1D8091020F9091030F480F591F46
:100F6000611D711D4115510581E06807710524F06F
:100F70004FEF5FEF60E070E0DB01CA0177FDE6C58F
:100F80000E94E01246EC41BB469A31E035B927E4B5
:100F900028B950EF5BB992EA9EB987E881BB00C0DF
:100FA00000C041BB469A35B928B960EE6BB99EB90D
:100FB00081BB00C000C041BB469A35B928B95BB9B6
:100FC0009EB981BB8091340E9091350EA091360E62
:100FD000B091370E8B2F9927AA27BB27892B8A2BF5
:100FE0008B2B09F0C0C48091590E823009F494C44F
:100FF00008F08CC4813009F4FDC480E090E0609179
:10100000520E7091530E0E94D33E2091500E30919B
:10101000510E280F391F3093550E2093540E809196
:10102000300E9091310EA091320EB091330E40915E
:10103000340E5091350E6091360E7091370E840F3C
:10104000951FA61FB71F8093340E9093350EA09363
:10105000360EB093370EC9010E94E01246EC41BB38
:10106000469A31E035B923E428B950EF5BB992EAEA
:101070009EB987E881BB00C000C041BB469A35B924
:1010800028B960EB6BB99EB981BB00C000C041BB01
:10109000469A35B928B95BB99EB981BB29812FBF62
:1010A0003FB73983F8948091620D9091630DA091C0
:1010B000640DB091650D8B2F9927AA27BB27892B2B
:1010C0008A2B8B2B09F04AC48091870D823009F45A
:1010D000A8C308F0A0C3813009F4D1C480E090E037
:1010E0006091800D7091810D0E94D33E20907E0D05
:1010F00030907F0D280E391E3092830D2092820D84
:1011000080915E0D90915F0DA091600DB091610D89
:101110004091620D5091630D6091640D7091650D69
:10112000840F951FA61FB71F8093620D9093630DC8
:10113000A093640DB093650D8091F80E9091F90E17
:10114000B301A201480F591F611D711D41155105C1
:1011500081E06807710524F04FEF5FEF60E070E019
:10116000DB01CA0177FDE1C40E94E01266EC61BBBD
:10117000469A51E055B945E448B970EF7BB990EA19
:101180009EB987E881BB00C000C061BB469A55B9D3
:1011900048B9E0EEEBB99EB981BB00C000C061BBAD
:1011A000469A55B948B97BB99EB981BB2D813E811C
:1011B000B101AA27269FB12D3703A001729FB00D60
:1011C000411D5A1F36035A0BB00D411D5A1F1124E1
:1011D000662757FD6095762F480D591D6A1D7B1DAA
:1011E0008091EC0E9091ED0E480F591F611D711DFD
:1011F0004115510581E06807710524F04FEF5FEF5D
:1012000060E070E0DB01CA0177FDB4C40E94E01227
:1012100066EC61BB469A51E055B941E448B970EFBC
:101220007BB992EA9EB987E881BB00C000C061BB70
:10123000469A55B948B9E0EDEBB99EB981BB00C0FB
:1012400000C061BB469A55B948B97BB99EB981BB0C
:101250009101AA27029FB12D1303A001309FB00D69
:10126000411D5A1F12035A0BB00D411D5A1F112464
:10127000662757FD6095762F4C0D5D1D6E1D7F1DF9
:101280008091040F9091050F480F591F611D711D2A
:101290004115510531E06307710524F04FEF5FEF11
:1012A00060E070E0DB01CA0177FD60C40E94E012DB
:1012B00046EC41BB469A31E035B921E428B950EFFC
:1012C0005BB990EA9EB987E881BB00C000C041BB12
:1012D000469A35B928B960EB6BB99EB981BB00C09D
:1012E00000C041BB469A35B928B95BB99EB981BBEC
:1012F00080915E0E90915F0EA091600EB091610E94
:101300008B2F9927AA27BB27892B8A2B8B2B09F098
:1013100016C38091830E823009F46AC208F062C25B
:10132000813009F4E4C380E090E060917C0E70911C
:101330007D0E0E94D33E20917A0E30917B0E280FB5
:10134000391F30937F0E20937E0E80915A0E90911C
:101350005B0EA0915C0EB0915D0E40915E0E5091BF
:101360005F0E6091600E7091610E840F951FA61F35
:10137000B71F80935E0E90935F0EA093600EB093A4
:10138000610EC9010E94E01246EC41BB469A31E071
:1013900035B925E428B950EF5BB992EA9EB987E8E0
:1013A00081BB00C000C041BB469A35B928B960EB8B
:1013B0006BB99EB981BB00C000C041BB469A35B92C
:1013C00028B95BB99EB981BB29812FBF3FB739834B
:1013D000F89480918C0D90918D0DA0918E0DB0910F
:1013E0008F0D8B2F9927AA27BB27892B8A2B8B2B15
:1013F00009F0C3C28091B10D823009F4E0C108F058
:10140000D8C1813009F44CC380E090E06091AA0D0E
:101410007091AB0D0E94D33E2090A80D3090A90D85
:10142000280E391E3092AD0D2092AC0D8091880DA2
:101430009091890DA0918A0DB0918B0D40918C0DEA
:1014400050918D0D60918E0D70918F0D840F951FB1
:10145000A61FB71F80938C0D90938D0DA0938E0DBA
:10146000B0938F0D8091FA0E9091FB0E480E591E8D
:10147000611C711C4114510441E0640671042CF09C
:1014800044244A94542C612C712CD301C20177FC62
:1014900069C30E94E01266EC61BB469A51E055B9FF
:1014A00047E448B970EF7BB990EA9EB987E881BB01
:1014B00000C000C061BB469A55B948B9E0EEEBB92F
:1014C0009EB981BB00C000C061BB469A55B948B9FE
:1014D0007BB99EB981BB6D817E819101AA27629FF4
:1014E000B12D7303A001369FB00D411D5A1F720329
:1014F0005A0BB00D411D5A1F1124662757FD6095E8
:10150000762F480D591D6A1D7B1D8091EE0E90911E
:10151000EF0E480F591F611D711D4115510531E036
:101520006307710524F04FEF5FEF60E070E0DB01CF
:10153000CA0177FD13C30E94E01266EC61BB469AB4
:1015400051E055B943E448B970EF7BB992EA9EB9CE
:1015500087E881BB00C000C061BB469A55B948B955
:10156000E0EDEBB99EB981BB00C000C061BB469AFB
:1015700055B948B97BB99EB981BBB101AA27069F6D
:10158000B12D1703A001709FB00D411D5A1F160306
:101590005A0BB00D411D5A1F1124662757FD609547
:1015A000762F4C0D5D1D6E1D7F1D8091060F909155
:1015B000070F480F591F611D711D4115510581E02D
:1015C0006807710524F04FEF5FEF60E070E0DB012A
:1015D000CA0177FDBFC2F4D746EC41BB469A31E061
:1015E00035B923E428B950EF5BB990EA9EB987E892
:1015F00081BB00C000C041BB469A35B928B960EB39
:101600006BB99EB981BB00C000C041BB469A35B9D9
:1016100028B95BB99EB981BB8091880E9091890EE3
:10162000A0918A0EB0918B0E8B2F9927AA27BB27EA
:10163000892B8A2B8B2B09F087C18091AD0E8230CC
:1016400009F4A4C008F09CC0813009F43FC280E0D6
:1016500090E06091A60E7091A70E0E94D33EE0919B
:10166000A40EF091A50EE80FF91FF093A90EE093D8
:10167000A80E4091840E5091850E6091860E709157
:10168000870E0091880E1091890E20918A0E30915C
:101690008B0E400F511F621F731F4093880E509393
:1016A000890E60938A0E70938B0ECF0189D746EC1A
:1016B00041BB469A31E035B927E428B950EF5BB910
:1016C00092EA9EB987E881BB00C000C041BB469A40
:1016D00035B928B960EB6BB99EB981BB00C000C0B9
:1016E00041BB469A35B928B95BB99EB981BB2981FE
:1016F0002FBF20916209922F9C7111E009F010E038
:10170000922F9370923009F4B6C2933009F4D8C482
:10171000913009F4BBC21111E1C40E94484C809180
:101720005E0990915F09A0916009B09161090196ED
:10173000A11DB11D80935E0990935F09A09360097C
:10174000B0936109209162092F5F20936209269668
:101750000FB6F894DEBF0FBECDBFDF91CF911F91C2
:101760000F91FF90EF90DF90CF90BF90AF909F9040
:101770008F907F906F905F904F903F902F90089543
:10178000833009F4C5C1843009F061CF6091880EBF
:101790007091890E80918A0E90918B0E2091AA0EE5
:1017A00021111FC2BB27A92F982F872F80959095B5
:1017B00050CF833009F485C1843009F025CE609183
:1017C0008C0D70918D0D80918E0D90918F0D2091CB
:1017D000AE0D2111F2C1BB27A92F982F872F80951D
:1017E000909514CE833009F4D2C0843009F09BCD9B
:1017F00060915E0E70915F0E8091600E9091610E0F
:101800002091800E2111F7C1BB27A92F982F872F78
:10181000809590958ACD833009F4BEC0843009F05C
:101820005DCC6091620D7091630D8091640D90911B
:10183000650D2091840D2111ABC1BB27A92F982FD5
:10184000872F809590954CCC833009F4F3C0843079
:1018500009F03DCA60910A0E70910B0E80910C0E3A
:1018600090910D0E20912C0E2111CAC1BB27A92FDA
:10187000982F872F809590952CCA833009F4D5C076
:10188000843009F095CA6091380D7091390D8091BE
:101890003A0D90913B0D20915A0D211189C1BB2722
:1018A000A92F982F872F8095909584CA833009F4AB
:1018B000B7C0843009F0E3C860910E0D70910F0D30
:1018C0008091100D9091110D2091300D21119DC12D
:1018D000BB27A92F982F872F80959095D2C883304A
:1018E00009F470C0843009F05AC86091E00D70911D
:1018F000E10D8091E20D9091E30D2091020E44E8FC
:1019000051E00E942722809590954BC8833009F4BE
:1019100082C0843009F071CB6091340E7091350E25
:101920008091360E9091370E2091560E211126C1CE
:10193000BB27A92F982F872F8095909560CB8AE59C
:101940009EE00E941425E5CC84E89EE00E941425C8
:1019500074CE8AE09DE00E94142587C88EE59DE044
:101960000E941425B1CB80E39EE00E9414253BCB5E
:1019700084E39DE00E94142511CA88E89DE00E943E
:10198000142538CD86E09EE00E94142596C98091EA
:101990006E0E90916F0EC9CC8091720D9091730D67
:1019A0009FCB60910A0E70910B0E80910C0E90915E
:1019B0000D0E20912C0E21112DC1BB27A92F982F80
:1019C000872F87C98091F00D9091F10D0C94D1046F
:1019D0006091E00D7091E10D8091E20D9091E30D29
:1019E0002091020E2111D9C0BB27A92F982F872F34
:1019F0000C94D1046091340E7091350E8091360EA6
:101A00009091370E2091560E2111BDC0BB27A92FF2
:101A1000982F872FF4CA8091440E9091450EEFCAFB
:101A200080911E0D90911F0D2CC88091480D9091B2
:101A3000490DC0C980911A0E90911B0E4AC9609140
:101A40000E0D70910F0D8091100D9091110D209140
:101A5000300D44E853E00E94272213C86091380DEE
:101A60007091390D80913A0D90913B0D20915A0D56
:101A7000211199C0BB27A92F982F872F9BC960914F
:101A8000620D7091630D8091640D9091650D2091B0
:101A9000840D2111ABC0BB27A92F982F872F20CBF6
:101AA00060918C0D70918D0D80918E0D90918F0DA8
:101AB0002091AE0D21118BC0BB27A92F982F872F06
:101AC000A5CC80919C0D90919D0DA0CC6091880E2D
:101AD0007091890E80918A0E90918B0E2091AA0EA2
:101AE000211170C0BB27A92F982F872FB2CD6091ED
:101AF0005E0E70915F0E8091600E9091610E20914C
:101B0000800E211169C0BB27A92F982F872F0DCCDC
:101B10008091980E9091990E9CCD80E090E0DC0130
:101B2000DFC980E090E0DC0189C980E090E0DC0161
:101B30001BCB80E090E0DC010C94870580E090E016
:101B4000DC0188C880E090E0DC0134C880E090E0EF
:101B5000DC0116CA80E090E0DC013DCD80E090E041
:101B6000DC01E9CC80E090E0DC0193CC80E090E007
:101B7000DC019CCB80E090E0DC0148CB44E851E004
:101B80000E94E43ED9CE44E853E00E94E43E37CAC6
:101B900044E851E00E94E43E54CE44E853E00E9401
:101BA000E43E0C94D10444E853E00E94E43E02C9B0
:101BB00044E851E00E94E43E76CE44E851E00E94C1
:101BC000E43E0DCE44E853E00E94E43E42CD44E8BA
:101BD00053E00E94E43E1ACC44E853E00E94E43E05
:101BE000A4CB44E851E00E94E43EE0CD44E853E059
:101BF0000E94E43E75CA44E851E00E94E43E08CEEB
:101C000044E851E00E94E43E35CE44E851E00E94B1
:101C1000E43E62CE44E853E00E94E43E5AC81E828D
:101C20001D820C94AB028090C40E9090C50E9594CA
:101C30008794840C951C0C946E0280E090E0DC018B
:101C40000C94D70280E090E0DC010C94770380E0F4
:101C500090E0DC010C94280380E090E0DC010C941F
:101C60008E0480E090E0DC010C943E0480E090E083
:101C7000DC010C94EC0389EC9EE00E9454228091DC
:101C80006B0F88706ED3209162095ECD0E948F5CCD
:101C90008091B50C882371F08091F110882309F4AC
:101CA0003BC380915F0F882329F0815080935F0FA1
:101CB0000E94CE578091580F882309F4FEC180916D
:101CC000560F9091570F4091080F5091090F209196
:101CD000E40E3091E50E2417350708F4EDC24217E3
:101CE000530770F4B901641B750BAB018617970796
:101CF00008F4AC01241B350B3093E50E2093E40E61
:101D00004091140F5091150F2091F00E3091F10E6B
:101D10002417350708F4C4C24217530770F4F901B9
:101D2000E41BF50BAF018E179F0708F4AC01241BD1
:101D3000350B3093F10E2093F00E4091200F50910F
:101D4000210F2091FC0E3091FD0E2417350708F469
:101D50009BC24217530770F4B901641B750BAB01AA
:101D60008617970708F4AC01241B350B3093FD0E42
:101D70002093FC0E40910A0F50910B0F2091E60E1C
:101D80003091E70E2417350708F472C24217530743
:101D900070F4F901E41BF50BAF018E179F0708F4EF
:101DA000AC01241B350B3093E70E2093E60E4091D7
:101DB000160F5091170F2091F20E3091F30E241749
:101DC000350708F448C24217530770F4B901641B81
:101DD000750BAB018617970708F4AC01241B350B74
:101DE0003093F30E2093F20E4091220F5091230F67
:101DF0002091FE0E3091FF0E2417350708F41EC205
:101E00004217530770F4F901E41BF50BAF018E176D
:101E10009F0708F4AC01241B350B3093FF0E209371
:101E2000FE0E40910C0F50910D0F2091E80E309155
:101E3000E90E2417350708F4F4C14217530770F46C
:101E4000B901641B750BAB018617970708F4AC0149
:101E5000241B350B3093E90E2093E80E4091180FA8
:101E60005091190F2091F40E3091F50E241735077B
:101E700008F4CAC14217530770F4F901E41BF50BCB
:101E8000AF018E179F0708F4AC01241B350B30936C
:101E9000F50E2093F40E4091240F5091250F2091C0
:101EA000000F3091010F2417350708F4A0C1421725
:101EB000530770F4B901641B750BAB0186179707C4
:101EC00008F4AC01241B350B3093010F2093000F55
:101ED00040910E0F50910F0F2091EA0E3091EB0EB2
:101EE0002417350708F476C14217530770F4F90137
:101EF000E41BF50BAF018E179F0708F4AC01241B00
:101F0000350B3093EB0E2093EA0E40911A0F50914F
:101F10001B0F2091F60E3091F70E2417350708F4A9
:101F20004CC14217530770F4B901641B750BAB0128
:101F30008617970708F4AC01241B350B3093F70E76
:101F40002093F60E4091260F5091270F2091020FFB
:101F50003091030F2417350708F422C142175307A5
:101F600070F4F901E41BF50BAF018E179F0708F41D
:101F7000AC01241B350B3093030F2093020F4091CB
:101F8000100F5091110F2091EC0E3091ED0E24178F
:101F9000350708F4F8C04217530770F4B901641B01
:101FA000750BAB018617970708F4AC01241B350BA2
:101FB0003093ED0E2093EC0E40911C0F50911D0FAD
:101FC0002091F80E3091F90E2417350708F4CEC091
:101FD0004217530770F4F901E41BF50BAF018E179C
:101FE0009F0708F4AC01241B350B3093F90E2093A6
:101FF000F80E4091280F5091290F2091040F309135
:10200000050F2417350708F4A4C04217530770F4CE
:10201000B901641B750BAB018617970708F4AC0177
:10202000241B350B3093050F2093040F4091120FA2
:102030005091130F2091EE0E3091EF0E24173507BB
:1020400008F074C0421B530B8417950708F462C153
:10205000420F531F5093EF0E4093EE0E40911E0F10
:1020600050911F0F2091FA0E3091FB0E2417350767
:1020700008F049C0421B530B8417950708F448C168
:10208000420F531F5093FB0E4093FA0E40912A0FBC
:1020900050912B0F2091060F3091070F2417350711
:1020A00000F5421B530B8417950708F42FC1420F0C
:1020B000531F5093070F4093060F2091620944CBA2
:1020C00022FD42CB812F0E945438812F0E94FD486F
:1020D000F4CF0196A11DB11D0C94A5020E94852587
:1020E0001CCB4217530748F7F901E41BF50BAF016E
:1020F0008E179F0708F4AC01241B350B3093070F94
:102100002093060FDACF4217530708F0BFCFB9016B
:10211000641B750BAB018617970708F4AC01241BF1
:10212000350B3093FB0E2093FA0EB0CF42175307B6
:1021300008F094CFF901E41BF50BAF018E179F0750
:1021400008F4AC01241B350B3093EF0E2093EE0EF8
:1021500085CF421B530B8417950708F4D5C0420F57
:10216000531F5093050F4093040F60CF421B530B36
:102170008417950708F4C6C0420F531F5093F90EF9
:102180004093F80E36CF421B530B8417950708F483
:10219000B7C0420F531F5093ED0E4093EC0E0CCF7F
:1021A000421B530B8417950708F4A8C0420F531F16
:1021B0005093030F4093020FE2CE421B530B841740
:1021C000950708F499C0420F531F5093F70E4093A0
:1021D000F60EB8CE421B530B8417950708F48AC03D
:1021E000420F531F5093EB0E4093EA0E8ECE421BCC
:1021F000530B8417950708F47BC0420F531F50936D
:10220000010F4093000F64CE421B530B84179507B8
:1022100008F46CC0420F531F5093F50E4093F40E18
:102220003ACE421B530B8417950708F45DC0420F4A
:10223000531F5093E90E4093E80E10CE421B530BF0
:102240008417950708F44EC0420F531F5093FF0E9A
:102250004093FE0EE6CD421B530B8417950708F4FE
:102260003FC0420F531F5093F30E4093F20EBCCD6C
:10227000421B530B8417950788F1420F531F50934D
:10228000E70E4093E60E93CD421B530B8417950740
:1022900018F1420F531F5093FD0E4093FC0E6ACD70
:1022A000421B530B84179507A8F0420F531F5093FE
:1022B000F10E4093F00E41CD421B530B841795074E
:1022C00038F0420F531F5093E50E4093E40E18CDA3
:1022D000AC01F7CFAC01E9CFAC01DBCFAC01CDCF86
:1022E000AC01BFCFAC01B0CFAC01A1CFAC0192CF5C
:1022F000AC0183CFAC0174CFAC0165CFAC0156CF3C
:10230000AC0147CFAC0138CFAC0129CFAC01CFCE67
:10231000AC01B6CEAC019CCE80915F0F882309F44E
:10232000C7CCC3CCE82FF0E0EE0FFF1FE753F04F10
:1023300080819181089596EC91BB469A982F96954D
:10234000969596958295880F807E95B990E498B978
:102350001BB88EB987E881BB85E08A95F1F700004C
:1023600008950F931F93382F2091620FE091650F0E
:10237000222309F407C140917E0F50917F0F60E046
:1023800070E0EE2309F4F9C08091840F9091850FDD
:10239000A0E0B0E03323A1F0222381F020916B0F65
:1023A00025FD0CC00091C40E1091C50E222717FD0B
:1023B0002095322F400F511F621F731FE111E7C09C
:1023C0002FB7F8944115510531E06307710524F0EA
:1023D0004FEF5FEF60E070E077FDEEC0BA01672F6E
:1023E000772766956695062FE6ECE1BB469A162F91
:1023F000110FF12FF670F068607177276260312F4E
:10240000330F3072362B107C312B602F6695627043
:10241000606215B8F8B93BB96EB967E861BB56950B
:10242000479556954795742FE1BB469A142F110F87
:10243000F42FF695771F7727771F312F3670732B80
:102440007068407155274260312F330F3072342B42
:10245000107C312BF27015B878B93BB9FEB961BB6D
:10246000E1BB469A51E055B941E448B970EF7BB9F8
:1024700032EA3EB961BB00C000C0E1BB469A55B923
:1024800048B9F0E7FBB93EB961BB00C000C0E1BB91
:10249000469A55B948B97BB93EB961BB009731E05E
:1024A000A307B10524F08FEF9FEFA0E0B0E0B7FDE8
:1024B0007FC0AC01452F552746954695F42F66EC15
:1024C00061BB469AE42FEE0F7E2F767070684071E4
:1024D000552742603E2F330F3072342BE07C3E2B69
:1024E0004F2F46954270406215B878B93BB94EB946
:1024F00037E831BB9695879596958795482F61BBB0
:10250000469A782F770F582F5695441F4427441F1B
:10251000E72FE6704E2B4068807199278260972FD5
:10252000990F9072982B707C972B527015B848B900
:102530009BB95EB931BB61BB469A41E045B997E4AE
:1025400098B950EF5BB982EA8EB931BB00C000C0C8
:1025500061BB469A45B998B970E77BB98EB931BB72
:1025600000C000C061BB469A45B998B95BB98EB945
:1025700031BB2FBF1F910F9108958FEF9FEFA0E008
:10258000B0E008CF4FEF5FEF60E070E0FACE20914F
:102590006B0F24FD15CF0091C40E1091C50E22279C
:1025A00017FD2095322F800F911FA21FB31F08CF58
:1025B00080E090E0DC017DCF40E050E0BA010ECF3A
:1025C0009C01232F332726952695722F66EC61BB3D
:1025D000469A522F550F452F467040682071332779
:1025E0002260352F330F3072322B507C352B272F42
:1025F00026952270206215B848B93BB92EB957E824
:1026000051BB9695879596958795282F61BB469ADD
:10261000482F440F382F3695221F2227221F642F60
:102620006670262B2068807199278260942F990FFD
:102630009072982B407C942B327015B828B99BB9B6
:102640003EB951BB08956095E9EFF0E19081982B78
:102650006923608386EC81BB469A362F330F962F11
:102660009695262F221F2227221F832F8670282B24
:1026700020646071832F880F8072862B307C832BBF
:102680009270906C31E035B928B98BB99EB987E862
:1026900081BB85E08A95F1F70000E8EFF0E18081E9
:1026A0008F5F8083089580959091F910892380939E
:1026B000F91096EC91BB469A482F440F282F269587
:1026C000382F331F3327331F942F9670392B3064E4
:1026D0008071942F990F9072982B407C942B2270CC
:1026E000206C81E085B938B99BB92EB987E881BBE8
:1026F00085E08A95F1F700008091F8108F5F809354
:10270000F81008958091F91080618093F91096EC8B
:1027100091BB469A382F330F982F9695282F221F5A
:102720002227221F832F8670282B2064832F880F57
:1027300080728061307C832B9270906C31E035B96F
:1027400028B98BB99EB987E881BB85E08A95F1F7F6
:1027500000008091F8108F5F8093F81008958091A9
:10276000F91081608F7E8093F91096EC91BB469AA8
:10277000382F330F982F9695881F8827881F232F6F
:102780002670822B8064232F220F2072307C232B13
:102790009270906C31E035B988B92BB99EB987E851
:1027A00081BB85E08A95F1F700008091F8108F5F7A
:1027B0008093F81008953091F910832F88608E7FF0
:1027C0008093F91096EC91BB469A282F220F982FF0
:1027D0009695881F8827881F422F4670842B806417
:1027E000207C30713062232B9270906C31E035B9CF
:1027F00088B92BB99EB987E881BB85E08A95F1F746
:1028000000008091F8108F5F8093F8100895409138
:10281000F910242F22602093F91086EC81BB469A90
:10282000322F330F922F9695221F2227221F832F9C
:102830008670282B2064832F880F80724071842B30
:10284000307C832B9270906C31E035B928B98BB90C
:102850009EB987E881BB85E08A95F1F700008091F9
:10286000F8108F5F8093F8100895EF92FF920F9306
:102870001F93CF93DF937C01EB01142F40FF09C01E
:102880002091F4103091F510282739272C7F232B25
:1028900071F511FF0AC08091F6109091F7108C2706
:1028A0009D2788279E7F892B39F4DF91CF911F9137
:1028B0000F91FF90EF9008950D2F06954091EF1026
:1028C0004F70406BE0911218F091131821E063E013
:1028D00070E082E198E10995D093F710C093F6106B
:1028E000DF91CF911F910F91FF90EF900895905835
:1028F0009C013595279535952795092F06952F77B6
:1029000033274091EF104F70406EE0911218F09114
:10291000131863E070E082E198E10995F092F510F8
:10292000E092F410B6CF0F93262F4F772F778F704A
:102930008068E0911218F0911318042F482F63E07B
:1029400070E082E198E109950F910895EF92FF926E
:102950000F931F93CF93DF93EC01162FF42EE22EEB
:1029600080913718843071F1C230D10509F453C019
:10297000C330D10571F1C130D105F9F1C430D105B1
:10298000C8F5E0912E18F0912F18309739F00E2DE0
:102990002F2D412FBE0182E198E10995E091301879
:1029A000F0913118309739F00E2D2F2D412FBE01A7
:1029B00082E198E10995DF91CF911F910F91FF90EE
:1029C000EF900895E0912C18F0912D183097F9F6BA
:1029D000D8CF862F807F803A09F48DC008F041C09F
:1029E000803809F456C0803961F6E0911618F091EC
:1029F000171842C0C0E0D0E0C4CF683F50F1E0916A
:102A00002818F0912918309709F4BBCF612F82E183
:102A100098E10995C3CF862F807F803D09F455C08A
:102A2000803F09F440C0803C09F0ABCFE091201812
:102A3000F0912118309709F4A4CF133F09F43FC057
:102A4000113FE9F1612F6F704F2D82E198E10995F7
:102A5000A5CF663F09F095CFE0912A18F0912B1889
:102A6000D2CF803ED9F0803FA9F1803B09F089CFD9
:102A7000E0911418F0911518309709F482CF123FA5
:102A800099F1612F6F702E2D4F2D82E198E10995FC
:102A900085CFE0911818F0911918EECFE0911C182D
:102AA000F0911D18E9CF633F59F1613F09F069CFFB
:102AB000E0912618F0912718309709F462CF4F2D36
:102AC000612F82E198E1099569CFE0912218F09198
:102AD0002318B0CF623F09F054CFE0911E18F09157
:102AE0001F18309709F44DCF2E2D4F2D62EF82E144
:102AF00098E1099553CFE0911A18F0911B18BCCFBB
:102B0000E0912418F09125183097C9F63ACFCF9369
:102B1000DF930E945F3CC82FD0E00E945F3C382FBB
:102B200020E0C22BD32B81E006DC81E004DC86ECC4
:102B300081BB469A15B882E488B91BB880E48EB987
:102B400087E881BB85E08A95F1F7000082E0F3DB3E
:102B5000C095D095CE01DF91CF910895FF920F934C
:102B60001F93CF93DF93F82EABEA8A9FA12D1124F8
:102B7000A695A695A6951A2F1F5F462F50E0A83060
:102B800008F063C08A2F90E0880F991FFC01EE0FB8
:102B9000FF1FEE0FFF1FEE0FFF1FE80FF91FE40FDF
:102BA000F51FEE0FFF1FE753F04FC081D1811830A2
:102BB00008F46FC0FA01EE0FFF1FEB53FF4E0190B8
:102BC000F081E02DDA01AA0FBB1FAF55BF4E8D91EA
:102BD0009C919F01281B390BA12FB0E017970E94F1
:102BE000356A6E0F7F1F811D911D6115710521E0F2
:102BF0008207910508F063C08B010C1B1D0B9BEA3B
:102C0000F99E912D1124969596959695892F880F6A
:102C1000890F880F880F6F2D681B862F90E0A0E02A
:102C2000B0E0772766272CE030E040E050E00E94DB
:102C3000F46ED8010E94BD6EC80FD91FCE01DF917E
:102C4000CF911F910F91FF900895FA01EE0FFF1F92
:102C5000EB53FF4E0190F081E02DEA01CC0FDD1F18
:102C6000CF55DF4E888199819F01281B390BB0E039
:102C700017970E94356A6E0F7F1F811D911D611588
:102C8000710521E082079105F8F4EB01183008F096
:102C900091CF812F90E0880F991FFC01EE0FFF1F4D
:102CA000EE0FFF1FEE0FFF1FE80FF91FE40FF51FD8
:102CB000EE0FFF1FE753F04F608171819DCF6FEFE3
:102CC0007FEF80E090E098CF6FEF7FEF80E090E0C3
:102CD000EB01DCCFAF92BF92CF92DF92EF92FF92E7
:102CE0000F931F93CF93DF93E0E3FFE011921192D4
:102CF0008FE0E435F807D1F71092550F1092540F7A
:102D00008091740F823009F421C1833009F40AC123
:102D1000813059F0DF91CF911F910F91FF90EF908B
:102D2000DF90CF90BF90AF900895C0912E0FD091BB
:102D30002F0F1091730F110F60E0812F0FDF7C01B7
:102D400080E0F0DA9701281B390BDE010E94356A1A
:102D5000CC24CA94DC2CE12CF12CA70196010E9412
:102D6000CD6E3093310F2093300F61E0812FF6DE6E
:102D70005C0181E0D7DA9501281B390BDE010E9446
:102D8000356AA70196010E94CD6E3093330F2093D0
:102D9000320F62E0812FE2DE5C0182E0C3DA95014E
:102DA000281B390BDE010E94356AA70196010E949B
:102DB000CD6E3093350F2093340F63E0812FCEDE3C
:102DC0005C0183E0AFDA9501281B390BDE010E941C
:102DD000356AA70196010E94CD6E3093370F20937C
:102DE000360F64E0812FBADE5C0184E09BDA950146
:102DF000281B390BDE010E94356AA70196010E944B
:102E0000CD6E3093390F2093380F65E0812FA6DE09
:102E10005C0185E087DA9501281B390BDE010E94F1
:102E2000356AA70196010E94CD6E30933B0F209327
:102E30003A0F66E0812F92DE5C0186E073DA95013D
:102E4000281B390BDE010E94356AA70196010E94FA
:102E5000CD6E30933D0F20933C0F67E0812F7EDED7
:102E60005C0187E05FDA9501281B390BDE010E94C7
:102E7000356AA70196010E94CD6E30933F0F2093D3
:102E80003E0F68E0812F6ADE5C0188E04BDA950135
:102E9000281B390BDE010E94356AA70196010E94AA
:102EA000CD6E3093410F2093400F69E0812F56DEA5
:102EB0005C0189E037DA9501281B390BDE010E949D
:102EC000356AA70196010E94CD6E3093430F20937F
:102ED000420F6AE0812F42DE5C018AE023DA95012D
:102EE000281B390BDE010E94356AA70196010E945A
:102EF000CD6E3093450F2093440F6BE0812F2EDE73
:102F00008C018BE00FDA9801281B390BDE010E943F
:102F1000356AA70196010E94CD6E3093470F20932A
:102F2000460FF8CE2091730FA0912E0FB0912F0F66
:102F300030E00E94356A2CE030E040E050E00E9432
:102F4000CD6E3093550F2093540FE4CE2091730F24
:102F5000A0912E0FB0912F0F30E00E94356A2CE027
:102F600030E040E050E00E94CD6E3093490F209356
:102F7000480F30934B0F20934A0F30934D0F2093FF
:102F80004C0F30934F0F20934E0F3093510F2093DF
:102F9000500F3093530F2093520FBCCE21E030E0FE
:102FA00002C0220F331F8A95E2F7F901E095F095F0
:102FB0008091E3099091E4098E239F239093E40983
:102FC0008093E3094091E5095091E6094E235F2380
:102FD0005093E6094093E509662331F0282B392BFD
:102FE0003093E4092093E3090895E3EEF9E080814A
:102FF0009181A5EEB9E02D913C9111973E7F2D93E3
:103000003C939160918380830895FC01623009F4C0
:103010003BC018F1633069F1643011F511A210A2C0
:10302000268D378D46895789AA27249FB12D359F34
:10303000C001529FB00D811D9A1F349FB00D811D9C
:103040009A1F112482A393A34089518962897389AD
:1030500040835183628373830895613009F443C0D0
:1030600011A210A213A212A2108211821282138244
:10307000089511A210A28689978993A382A3108232
:1030800011821282138208952689378944895589CD
:10309000AA27429FB12D539FC001349FB00D811DBF
:1030A0009A1F529FB00D811D9A1F112480A391A3D6
:1030B00040955095AA27429FB12D539FC001349F40
:1030C000B00D811D9A1F529FB00D811D9A1F1124B2
:1030D00082A393A344855585668577854083518374
:1030E00062837383089526893789468D578DAA2771
:1030F000429FB12D539FC001349FB00D811D9A1F77
:10310000529FB00D811D9A1F112480A391A3409559
:103110005095AA27429FB12D539FC001349FB00DF7
:10312000811D9A1F529FB00D811D9A1F112482A3E9
:1031300093A3408551856285738540835183628363
:10314000738308951F93CF93DF93EC01898D0E94C1
:10315000664218A5012E04C09695879577956795C8
:103160000A94D2F724E0660F771F881F991F2A95CB
:10317000D1F7688779878A879B878B8D0E94664203
:10318000012E04C096958795779567950A94D2F796
:1031900034E0660F771F881F991F3A95D1F76C8727
:1031A0007D878E879F878D8D0E94664204C096958D
:1031B0008795779567951A95D2F744E0660F771F44
:1031C000881F991F4A95D1F7688B798B8A8B9B8BC7
:1031D00069A5CE01DF91CF911F9117CFFC01268900
:1031E00037892617370719F0778B668BABCF089591
:1031F0000F931F93FC01808D918D8617970721F007
:10320000718F608F61E001C060E0828D938D8417C3
:10321000950719F0538F428F61E084899589821751
:10322000930719F0358B248B61E0848D958D801781
:10323000910719F0158F048F02C0662321F0CF018A
:103240001F910F917FCF1F910F910895FC0160A7EF
:1032500079CFDF92EF92FF920F931F93CF93DF937B
:10326000ECEEFBE0D0E048E050E0C6ECB7E811E05F
:1032700000EF819191917D2F786F2D2F26952695C6
:1032800026957A0102C0EE0CFF1C2A95E2F76E2DFE
:1032900060956723FFB6F8949C01232F332726956A
:1032A0002695D22EC1BB469AE22EEE0CAE2DA6700C
:1032B000A0682071332722603E2D330F3072322BED
:1032C0002E2D207C322B2D2D26952270206215B8B4
:1032D000A8B93BB92EB9B1BB9695879596958795B8
:1032E000282FC1BB469AA82FAA0F382F3695221F28
:1032F0002227221F0F2EF6E0EF2EF02DEA222E2994
:1033000020688071992782609A2F990F9072982B6C
:10331000A07C9A2B327015B828B99BB93EB9B1BBC5
:10332000C1BB469A372F330F36703164972F96956D
:103330009270906A15B938B90BB99EB9B1BB85E0E6
:103340008A95F1F70000C1BB469A262F220F762FEF
:103350007695A62FAA1FAA27AA1F822F8670A82BB0
:10336000A0646071822F880F8072862B207C822B54
:103370007270706A15B9A8B98BB97EB9B1BB8AE011
:103380008A95F1F700C0C1BB469A15B938B90BB997
:103390009EB9B1BB8AE08A95F1F700C0FFBEDF5F3E
:1033A000D03209F066CF4FB7F89480912C0C96EC90
:1033B00091BB469A382F330F982F9695232F26705E
:1033C0002064582F551F5527551F252B582F5071F6
:1033D000832F880F8072852B307C832B92709066B0
:1033E00031E035B928B98BB99EB987E881BB4FBFA9
:1033F000DF91CF911F910F91FF90EF90DF90089593
:103400006091FE12663028F46F5C81E60E94FB3A00
:103410000BC06C3028F4655D82E60E94FB3A04C064
:103420006B5D86E60E94FB3A81E00E94FD4811CF69
:103430009F92AF92BF92CF92DF92EF92FF920F9343
:103440001F93CF93DF93D82FCEE1DADFC150E9F796
:103450001092F9101092F8106AE081E1F4D857DB6D
:10346000C12CD12C7601DD2309F4DCC016ECC0EEB2
:1034700087E0982EAA24A39490E4B92E00E2C7D93D
:103480009AD980E492E4AFE0B0E067E457EE47EF0A
:1034900032EE05C00097A105B10509F4D4C011BBF7
:1034A000469AC7B99AB8CDB9A5B8B8B81BB80EB97D
:1034B00061BB22E02A95F1F700C026B179B17CB159
:1034C00011BB479A57B94AB93DB90197A109B1094A
:1034D00022FDE0CF892B8A2B8B2B09F4B4C03FD976
:1034E00040E452E46FE070E0E7E437EE27EF92EE5D
:1034F00006C0411551056105710509F4A7C011BB4E
:10350000469AC7B99AB8CDB9A5B8B8B81BB80EB91C
:10351000E1BB82E08A95F1F700C086B1F9B1FCB158
:1035200011BB479A37B92AB99DB941505109610970
:10353000710982FFDECF452B462B472B09F486C04D
:10354000E1D840E452E46FE070E0E7E437EE27EFC3
:1035500092EE06C0411551056105710509F479C067
:1035600011BB469AC7B99AB8CDB9A5B8B8B81BB8B7
:103570000EB9E1BB82E08A95F1F700C086B189B14E
:103580008CB111BB479A37B92AB99DB9415051093D
:103590006109710981FDDECF452B462B472B09F4CC
:1035A00058C080E180D8AED840E452E46FE070E0CB
:1035B000E7E437EE27EF92EE06C0411551056105AD
:1035C000710509F43DC011BB469AC7B99AB8CDB987
:1035D000A5B8B8B81BB80EB9E1BB82E08A95F1F77F
:1035E00000C086B189B18CB111BB479A37B92AB9ED
:1035F0009DB9415051096109710981FFDECF452B09
:10360000462B472BE9F08AE04ED8D15080DAC80E1D
:10361000D91EE11CF11CF4DE8091FD128530E0F42E
:10362000D1112DCFB601C701DF91CF911F910F911D
:10363000FF90EF90DF90CF90BF90AF909F90089554
:103640000E94EE41E0CF0E94EE4149CF0E94EE4140
:1036500077CF0E94EE41A5CFCC24CA94DC2C760112
:10366000E1CF90912C0C9B7F8111946090932C0C56
:103670004FB7F89480912C0C96EC91BB469A382F5A
:10368000330F982F9695232F26702064582F551F9F
:103690005527551F252B582F5071832F880F807267
:1036A000852B307C832B9270906631E035B928B938
:1036B0008BB99EB987E881BB4FBF089590912C0CC0
:1036C000977F8111986090932C0C4FB7F89480915C
:1036D0002C0C96EC91BB469A382F330F982F969569
:1036E000232F26702064582F551F5527551F252B33
:1036F000582F5071832F880F8072852B307C832B3D
:103700009270906631E035B928B98BB99EB987E8D7
:1037100081BB4FBF08950F931F93CF93DF938B010E
:103720004091AA0F5091AB0FAA27049FB12D159F6E
:10373000B001509FB00D611D7A1F149FB00D611D27
:103740007A1F112440955095640F751F9AE28902E3
:10375000E0011124CE018A54934F40DD4091A80F1F
:103760005091A90FAA27049FB12D159FB001509F1A
:10377000B00D611D7A1F149FB00D611D7A1F1124B9
:1037800040955095640F751FCE018E54924FDF9176
:10379000CF911F910F9122CD2F923F924F925F9226
:1037A0006F927F928F929F92AF92BF92CF92DF9251
:1037B000EF92FF920F931F93CF93DF93CDB7DEB7B6
:1037C0002C970FB6F894DEBF0FBECDBFE090980FD8
:1037D000F090990F2090900F3090910F80916F0F83
:1037E0008093D80D80916D0F8093DC0C8091790FC0
:1037F000882309F4D2C463E082EB9DE027DD809149
:103800006E0F882309F4C7C463E086EB9CE01EDDDD
:103810008091F210882309F4BAC480E091E0A0E01E
:10382000B0E020919C0F30919D0F2C013D01420E84
:10383000531E611C711C20919A0F30919B0FAC019B
:10384000BD01420F531F611D711D2091960F3091D4
:10385000970F5C016D01A20EB31EC11CD11CA98281
:10386000BA82CB82DC822091940F3091950F5C015B
:103870006D01A20EB31EC11CD11CAD82BE82CF82CF
:10388000D8862091920F3091930F5C016D01A20EAA
:10389000B31EC11CD11CA986BA86CB86DC862091BA
:1038A0008E0F30918F0F4C015D01820E931EA11C73
:1038B000B11C09811A812B813C810115110581E020
:1038C0002807310524F00FEF1FEF20E030E041150D
:1038D0005105E1E06E07710524F04FEF5FEF60E006
:1038E00070E041145104F1E06F0671042CF044249F
:1038F0004A94542C612C712C9701B20182EB9DE00B
:1039000077DC950184018114910441E0A406B1049F
:1039100024F00FEF1FEF20E030E049845A846B84DD
:103920007C844114510481E0680671042CF0442425
:103930004A94542C612C712C6D817E818F819885E5
:1039400061157105E1E08E07910524F06FEF7FEFBF
:1039500080E090E09101A20186EB9CE049DC80913F
:103960006F0F8093020E80916D0F8093060D8091F2
:10397000790F882309F409C463E08CED9DE066DCCF
:1039800080916E0F882309F4FEC363E080EE9CE013
:103990005DDC8091F210882309F4F1C380E09FEF91
:1039A000AFEFBFEF20919C0F30919D0F2C013D0197
:1039B000420E531E611C711C77FCF1C320919A0FBB
:1039C00030919B0FAC01BD01420F531F611D711D52
:1039D00077FD2FC42091960F3091970F5C016D01F8
:1039E000A20EB31EC11CD11C96018501D7FC1DC4BB
:1039F0008090940F9090950F5C016D01A80CB91CFC
:103A0000C11CD11CA982BA82CB82DC82D7FC08C43B
:103A10008090920F9090930F5C016D01A80CB91CDF
:103A2000C11CD11CAD82BE82CF82D886D7FCF3C325
:103A3000E0918E0FF0918F0F4C015D018E0E9F1E55
:103A4000A11CB11CB7FCE3C30115110581E02807D7
:103A5000310524F00FEF1FEF20E030E04115510554
:103A6000E1E06E07710524F04FEF5FEF60E070E07A
:103A700041145104F1E06F0671042CF044244A947F
:103A8000542C612C712C9701B2018CED9DE0B0DBC0
:103A9000950184018114910441E0A406B10424F04D
:103AA0000FEF1FEF20E030E04D805E806F80788464
:103AB0004114510481E0680671042CF044244A94B6
:103AC000542C612C712C69817A818B819C816115C8
:103AD0007105E1E08E07910524F06FEF7FEF80E044
:103AE00090E09101A20180EE9CE082DB80916F0F5B
:103AF00080932C0E80916D0F8093300D8091790F03
:103B0000882309F43AC363E086E09EE09FDB80915E
:103B10006E0F882309F42FC363E08AE09DE096DBF3
:103B20008091F210882309F422C380E092E0A0E0A3
:103B3000B0E020919C0F30919D0F2C013D01420E71
:103B4000531E611C711C20919A0F30919B0FAC0188
:103B5000BD01420F531F611D711D2091960F3091C1
:103B6000970F5C016D01A20EB31EC11CD11CA9826E
:103B7000BA82CB82DC822091940F3091950F5C0148
:103B80006D01A20EB31EC11CD11CAD82BE82CF82BC
:103B9000D8862091920F3091930F5C016D01A20E97
:103BA000B31EC11CD11CA986BA86CB86DC862091A7
:103BB0008E0F30918F0F4C015D01820E931EA11C60
:103BC000B11C09811A812B813C810115110581E00D
:103BD0002807310524F00FEF1FEF20E030E04115FA
:103BE0005105E1E06E07710524F04FEF5FEF60E0F3
:103BF00070E041145104F1E06F0671042CF044248C
:103C00004A94542C612C712C9701B20186E09EE0FD
:103C1000EFDA950184018114910441E0A406B10416
:103C200024F00FEF1FEF20E030E049845A846B84CA
:103C30007C844114510481E0680671042CF0442412
:103C40004A94542C612C712C6D817E818F819885D2
:103C500061157105E1E08E07910524F06FEF7FEFAC
:103C600080E090E09101A2018AE09DE0C1DA8091BC
:103C70006F0F8093560E80916D0F80935A0D809137
:103C8000790F882309F471C263E080E39EE0DEDAF5
:103C900080916E0F882309F466C263E084E39DE09F
:103CA000D5DA8091F210882309F459C280E09EEFA2
:103CB000AFEFBFEF20919C0F30919D0F2C013D0184
:103CC000420E531E611C711C77FC9DC220919A0FFD
:103CD00030919B0FAC01BD01420F531F611D711D3F
:103CE00077FD8DC22091960F3091970F5C016D0189
:103CF000A20EB31EC11CD11C96018501D7FC7BC24C
:103D00008090940F9090950F5C016D01A80CB91CE8
:103D1000C11CD11CA982BA82CB82DC82D7FC66C2CC
:103D20008090920F9090930F5C016D01A80CB91CCC
:103D3000C11CD11CAD82BE82CF82D886D7FC51C2B5
:103D4000E0918E0FF0918F0F4C015D018E0E9F1E42
:103D5000A11CB11CB7FC41C20115110581E0280767
:103D6000310524F00FEF1FEF20E030E04115510541
:103D7000E1E06E07710524F04FEF5FEF60E070E067
:103D800041145104F1E06F0671042CF044244A946C
:103D9000542C612C712C9701B20180E39EE028DA4B
:103DA000950184018114910441E0A406B10424F03A
:103DB0000FEF1FEF20E030E04D805E806F80788451
:103DC0004114510481E0680671042CF044244A94A3
:103DD000542C612C712C69817A818B819C816115B5
:103DE0007105E1E08E07910524F06FEF7FEF80E031
:103DF00090E09101A20184E39DE0FAD980916F0FD8
:103E00008093800E80916D0F8093840D8091790F47
:103E1000882309F4A2C163E08AE59EE017DA809165
:103E20006E0F882309F497C163E08EE59DE00EDAFA
:103E30008091F210882309F48AC180E093E0A0E029
:103E4000B0E020919C0F30919D0F2C013D01420E5E
:103E5000531E611C711C20919A0F30919B0FAC0175
:103E6000BD01420F531F611D711D2091960F3091AE
:103E7000970F5C016D01A20EB31EC11CD11CA9825B
:103E8000BA82CB82DC822091940F3091950F5C0135
:103E90006D01A20EB31EC11CD11CAD82BE82CF82A9
:103EA000D8862091920F3091930F5C016D01A20E84
:103EB000B31EC11CD11CA986BA86CB86DC86209194
:103EC0008E0F30918F0F4C015D01820E931EA11C4D
:103ED000B11C09811A812B813C810115110581E0FA
:103EE0002807310524F00FEF1FEF20E030E04115E7
:103EF0005105E1E06E07710524F04FEF5FEF60E0E0
:103F000070E041145104F1E06F0671042CF0442478
:103F10004A94542C612C712C9701B2018AE59EE0E1
:103F200067D9950184018114910441E0A406B1048C
:103F300024F00FEF1FEF20E030E049845A846B84B7
:103F40007C844114510481E0680671042CF04424FF
:103F50004A94542C612C712C6D817E818F819885BF
:103F600061157105E1E08E07910524F06FEF7FEF99
:103F700080E090E09101A2018EE59DE039D9809129
:103F80006F0F8093AA0E80916D0F8093AE0D80917C
:103F9000790F882309F4D9C063E084E89EE056D9FC
:103FA00080916E0F882309F4CEC063E088E89DE01D
:103FB0004DD98091F210882309F4C1C080E09DEFB3
:103FC000AFEFBFEF20919C0F30919D0F2C013D0171
:103FD000420E531E611C711C77FCFBC020919A0F8E
:103FE00030919B0FAC01BD01420F531F611D711D2C
:103FF00077FDEBC02091960F3091970F5C016D011A
:10400000A20EB31EC11CD11C96018501D7FCD9C0DC
:104010008090940F9090950F5C016D01A80CB91CD5
:10402000C11CD11CA982BA82CB82DC82D7FCC4C05D
:104030008090920F9090930F5C016D01A80CB91CB9
:10404000C11CD11CAD82BE82CF82D886D7FCAFC046
:10405000E0918E0FF0918F0F4C015D018E0E9F1E2F
:10406000A11CB11CB7FC9FC00115110581E02807F8
:10407000310524F00FEF1FEF20E030E0411551052E
:10408000E1E06E07710524F04FEF5FEF60E070E054
:1040900041145104F1E06F0671042CF044244A9459
:1040A000542C612C712C9701B20184E89EE0A0D8B9
:1040B000950184018114910441E0A406B10424F027
:1040C0000FEF1FEF20E030E04D805E806F8078843E
:1040D0004114510481E0680671042CF044244A9490
:1040E000542C612C712C69817A818B819C816115A2
:1040F0007105E1E08E07910524F06FEF7FEF80E01E
:1041000090E09101A20188E89DE072D82C960FB64C
:10411000F894DEBF0FBECDBFDF91CF911F910F91FD
:10412000FF90EF90DF90CF90BF90AF909F908F90D7
:104130007F906F905F904F903F902F90089580E018
:1041400090E0DC013FCF61E031CF61E026CF80E03D
:1041500090E0DC0176CE61E068CE61E05DCE80E08B
:1041600090E0DC01A7CD61E099CD61E08ECD80E0EB
:1041700090E0DC01DECC61E0D0CC61E0C5CC80E039
:1041800090E0DC010FCC61E001CC61E0F6CB80E097
:1041900090E0DC0146CB61E038CB61E02DCB412CD7
:1041A000512C32010BCC812C912C54015DCF1D82FE
:1041B0001E821F8218864CCF19821A821B821C8293
:1041C00037CF00E010E0980123CF40E050E0BA0183
:1041D00011CF412C512C320101CF812C912C540153
:1041E000BBCD1D821E821F821886AACD19821A821B
:1041F0001B821C8295CD00E010E0980181CD40E04B
:1042000050E0BA016FCD412C512C32015FCD812C91
:10421000912C540119CC1D821E821F82188608CC55
:1042200019821A821B821C82F3CB00E010E09801F5
:10423000DFCB40E050E0BA01CDCBCF92DF92EF92DE
:10424000FF92CF93DF93EC01CC80DD80EE80FF8086
:104250008F2D9927AA27BB27892B8A2B8B2B09F017
:1042600042C089A5823009F433C070F5813009F469
:1042700044C040E050E02AA13BA1AA27429FB12DB3
:10428000539FC001349FB00D811D9A1F529FB00DE6
:10429000811D9A1F112428A139A1820F931F9DA36C
:1042A0008CA3488159816A817B814C0D5D1D6E1DF7
:1042B0007F1D4C835D836E837F83DF91CF91FF9061
:1042C000EF90DF90CF9008958330A1F0843089F68D
:1042D0008EA1811122C0BB27AF2D9E2D8D2DAC014B
:1042E00040955095C8CFCE019FD3CC80DD80EE8025
:1042F000FF80B7CF4C895D89BECF8EA1811105C0EB
:1043000077276F2D5E2D4D2DB6CF44E853E0C701C2
:10431000B6010E94E43EAC01AECF44E851E0C701D3
:10432000B6010E94E43EDBCFE82FE86F86958695C4
:10433000869528E030E001C0220F8A95EAF72095A3
:104340002E23AFB7F894CB01892F992786958695B0
:10435000F82F56EC51BB469A482F440F342F367035
:104360003068807199278260942F990F9072982BF2
:10437000407C942B8F2F86958270806215B838B957
:104380009BB98EB947E841BB769567957695679559
:10439000362F51BB469AF62FFF0F962F9695331F57
:1043A0003327331F8F2F8670382B30686071772743
:1043B00062608F2F880F8072862BF07C8F2B92701B
:1043C00015B838B98BB99EB941BB51BB469A3E2F3F
:1043D000330F367031649E2F96959270906AE1E0AB
:1043E000E5B938B9B0EFBBB99EB941BB85E08A9554
:1043F000F1F7000051BB469AF22FFF0F622F66952E
:10440000722F771F7727771F8F2F8670782B706416
:1044100020718F2F880F8072822BF07C8F2B62701F
:10442000606AE5B978B98BB96EB941BB8AE08A9503
:10443000F1F700C051BB469AE5B938B9BBB99EB98E
:1044400041BB8AE08A95F1F700C0AFBF0895211102
:1044500007C0BB27A92F982F872FBC01CB01089538
:10446000A72FE82F8F3FE9F08F5F90E0880F991F0B
:10447000F0E0EE0FFF1FE40FF51F20813181FA01FC
:10448000E80FF91F80819181821B930B892F992757
:10449000A89FB001A99F700D1124620F731FCB015B
:1044A00008958EEF91E0E4CFCF92DF92EF92FF92EA
:1044B0000F931F93CF93DF93EC01CC80DD80EE80D0
:1044C000FF808F2D9927AA27BB27892B8A2B8B2B1F
:1044D00009F04AC02A8D6C857D858E859F852330A5
:1044E00009F467C040F5213009F4ABC0EC89FD89BF
:1044F000C60ED71EE81EF91ECC82DD82EE82FF8238
:104500009F0140E050E0305841095109A889B9891C
:104510000E94BD6E2FEF3FEF40E050E00E94CD6E55
:104520003F8B2E8BDF91CF911F910F91FF90EF90DA
:10453000DF90CF900895243009F45FC02530B1F6A4
:1045400097018601E9E03695279517950795EA9535
:10455000D1F7F8011D8B0C8B298D222349F2E095B0
:10456000F095FD8BEC8BC4CFE1E0898DE81BE98FE2
:10457000E1116FC0C12CD12C7601CC82DD82EE829C
:10458000FF82FF27E1950CF4F095DF01AA0FBB1F16
:104590001196288539854A855B850E94C76E6C8790
:1045A0007D878E879F872A8D211159C0FD8BEC8BCB
:1045B0009DCFAD2DEE2DEF3F09F462C02E2D2F5F64
:1045C00030E0220F331FF0E0EE0FFF1FE650FF4EEA
:1045D00040815181F901E650FF4E20813181241B39
:1045E000350B232F3327A29FF001A39FF00D112439
:1045F000E40FF51FFD8BEC8B7BCFAB89A295AF70E1
:10460000088119812A813B81F32F000F111F221F7E
:10461000331FEF2FEE1FEE27EE1FBF2FB295B6957B
:10462000B770EB27EF27F695EF27E1700E2BA1501F
:1046300058F7088319832A833B83F8011D8B0C8B61
:1046400057CF33272F2D1E2D0D2DF8011D8B0C8BD1
:104650004FCFCC24CA94DC2CEC2CF12C8ECF223002
:1046600009F03DCF0E94B16E7D8B6C8B2A8D6C85DD
:104670007D858E859F85CC80DD80EE80FF802FCF6D
:104680002EEF31E0A0CFCF92DF92EF92FF920F9307
:104690001F93CF93DF9380916A0FC82FCC0FC80F61
:1046A000CF5F6091690F8EEA9EE00E94F7416C2F08
:1046B0008EEA9EE00E94AE3E8091590F90915A0F73
:1046C000A0915B0FB0915C0F8F3F2FEF9207A20775
:1046D000B20709F49CC02091AC0F3091AD0F2115A9
:1046E000324008F05DC0CFEFDFEFE0902C0FF0908C
:1046F0002D0F0090750F02C0F694E7940A94E2F72C
:104700004091A40F5091A50F411582E0580708F47D
:10471000ACC09A0132508091B00F9091B10F969534
:10472000879596958795811542E0940708F472C0A5
:104730008C0112508091770F882309F471C0AE016B
:10474000AA27249FB12D359FC001529FB00D811D16
:104750009A1F349FB00D811D9A1F11246091A20FE2
:104760007091A30FAC018EEA9EE00E94BE3EC8018C
:10477000809590958E159F0508F07AC04FEF5FEFFA
:104780006091AE0F7091AF0F89EC9EE0DF91CF91F9
:104790001F910F91FF90EF90DF90CF900C94BE3E51
:1047A00020915D0F30915E0F40E050E0820F931F2B
:1047B000A41FB51FC0905E09D0905F09E09060090A
:1047C000F0906109C816D906EA06FB0600F1C09010
:1047D0005E09D0905F09E0906009F0906109C81A05
:1047E000D90AEA0AFB0AC216D306E406F50608F05F
:1047F0007ACF9E2D8D2D7C2D66270E94F46EF901B7
:10480000EE0FFF1FEC57FC4FC081D1816ECFC0E08F
:10481000D0E06BCF00E010E08091770F81118FCF57
:10482000C901809590958E159F0530F54FEF5FEF8C
:104830006091A20F7091A30F8EEA9EE00E94BE3E8F
:104840009E01AA27029FB12D139FC001309FB00D7A
:10485000811D9A1F129FB00D811D9A1F1124609116
:10486000AE0F7091AF0FAC018FCF20E030E053CF8F
:10487000A8014E0D5F1D84CFA9014E0D5F1DD8CF3D
:104880008091EE1087FD09C06F7070E0992787FD59
:1048900090956817790709F0089580E8289F90019E
:1048A0001124242B3052220F331F220F331F309339
:1048B0002F0F20932E0F0E946A166FEF81E00C9449
:1048C0009B4D0F931F93CF93DF931F92CDB7DEB70E
:1048D0008B0140FD08C041FD14C00F90DF91CF91C6
:1048E0001F910F91089590932F0F80932E0F49835E
:1048F0000E946A166FEF81E00E949B4D498141FF43
:10490000ECCF10932D0F00932C0F0F90DF91CF91D0
:104910001F910F91B8CEE82FF0E0EE0FFF1FE4518A
:10492000F44F718360830895E82FF0E0EE0FFF1FCE
:10493000E451F44F118210820895E82FF0E0EE0F59
:10494000FF1FE451F44F8FEF9FEF91838083089511
:1049500060FD05C09093290C8093280C0895BC013C
:104960008EE1E2CC60FD05C09093210C8093200C79
:104970000895BC018AE1D8CC60FD05C090931F0C5E
:1049800080931E0C0895BC0189E1CECC60FD05C06A
:104990009093270C8093260C0895BC018DE1C4CC24
:1049A00060FD05C090931D0C80931C0C0895BC0104
:1049B00088E1BACC60FD05C09093230C8093220C53
:1049C0000895BC018BE1B0CCFC0126893789468D66
:1049D000578DAA27429FB12D539FC001349FB00D20
:1049E000811D9A1F529FB00D811D9A1F112480A313
:1049F00091A340955095AA27429FB12D539FC00186
:104A0000349FB00D811D9A1F529FB00D811D9A1FBA
:104A1000112482A393A340855185628573854083C9
:104A20005183628373830895FC0114821582168278
:104A30001782108211821282138281A58F5F81A753
:104A4000833009F43BC0853009F434C0823009F06A
:104A500008952689378935A324A344895589AA272F
:104A6000429FB12D539FC001349FB00D811D9A1FED
:104A7000529FB00D811D9A1F112480A391A34095D0
:104A80005095AA27429FB12D539FC001349FB00D6E
:104A9000811D9A1F529FB00D811D9A1F112482A360
:104AA00093A34485558566857785408351836283CA
:104AB0007383089511A615A214A2089511A210A23D
:104AC0008689978993A382A30895FC0111A210A25D
:104AD000268D378D46895789AA27249FB12D359F6A
:104AE000C001529FB00D811D9A1F349FB00D811DD2
:104AF0009A1F112482A393A34089518962897389E3
:104B00004083518362837383089590913B0B80911E
:104B10003A0B20913C0B211131C02091DB0D21116A
:104B2000EBC12091470B21116CC02091050E211182
:104B300051C12091520B211156C020912F0E2111ED
:104B4000B7C020915D0B211140C02091590E211159
:104B50008AC12091680B21112AC02091830E211156
:104B6000F0C02091730B211114C02091AD0E2111C2
:104B700056C090933B0B80933A0B08952091DB0D28
:104B80002111CFCF10923C0B10923E0B8FEF9FEF75
:104B9000C8CF2091AD0E2111ECCF1092730B109263
:104BA000750B2FEF2093720B2093710BE2CF2091A6
:104BB000830E2111D6CF1092680B10926A0B2FEF43
:104BC0002093670B2093660BCCCF2091590E2111B7
:104BD000C0CF10925D0B10925F0B2FEF20935C0BF8
:104BE00020935B0BB6CF20912F0E2111AACF1092EC
:104BF000520B1092540B2FEF2093510B2093500B1C
:104C0000A0CF2091050E211194CF1092470B109246
:104C1000490B2FEF2093460B2093450B8ACF109220
:104C2000AB0E1092A90E1092A80E1092880E109240
:104C3000890E10928A0E10928B0E1092A30E109273
:104C4000A20E1092AD0E1092A50E1092A40E10920C
:104C5000A70E1092A60E1092840E1092850E10923E
:104C6000860E1092870E1092AF0D1092AD0D10921D
:104C7000AC0D10928C0D10928D0D10928E0D109225
:104C80008F0D1092A70D1092A60D1092B10D1092DB
:104C9000A90D1092A80D1092AB0D1092AA0D1092B2
:104CA000880D1092890D10928A0D10928B0D61CF94
:104CB00010922D0E10922B0E10922A0E10920A0EA8
:104CC00010920B0E10920C0E10920D0E1092250EDB
:104CD0001092240E10922F0E1092270E1092260E74
:104CE0001092290E1092280E1092060E1092070EA6
:104CF0001092080E1092090E1092310D10922F0D85
:104D000010922E0D10920E0D10920F0D1092100D8C
:104D10001092110D1092290D1092280D1092330D42
:104D200010922B0D10922A0D10922D0D10922C0D19
:104D300010920A0D10920B0D10920C0D10920D0D89
:104D400000CF1092810E10927F0E10927E0E109264
:104D50005E0E10925F0E1092600E1092610E109215
:104D6000790E1092780E1092830E10927B0E109294
:104D70007A0E10927D0E10927C0E10925A0E1092A6
:104D80005B0E10925C0E10925D0E1092850D1092CB
:104D9000830D1092820D1092620D1092630D10928D
:104DA000640D1092650D10927D0D10927C0D109285
:104DB000870D10927F0D10927E0D1092810D109232
:104DC000800D10925E0D10925F0D1092600D10928A
:104DD000610DC7CE1092030E1092010E1092000EBC
:104DE0001092E00D1092E10D1092E20D1092E30D81
:104DF0001092FB0D1092FA0D1092050E1092FD0DFF
:104E00001092FC0D1092FF0D1092FE0D1092DC0D11
:104E10001092DD0D1092DE0D1092DF0D1092070D35
:104E20001092050D1092040D1092E40C1092E50CF6
:104E30001092E60C1092E70C1092FF0C1092FE0CF0
:104E40001092090D1092010D1092000D1092030D99
:104E50001092020D1092E00C1092E10C1092E20CF4
:104E60001092E30C66CE1092570E1092550E1092CF
:104E7000540E1092340E1092350E1092360E10927F
:104E8000370E10924F0E10924E0E1092590E109235
:104E9000510E1092500E1092530E1092520E10920C
:104EA000300E1092310E1092320E1092330E10927C
:104EB0005B0D1092590D1092580D1092380D1092F2
:104EC000390D10923A0D10923B0D1092530D109225
:104ED000520D10925D0D1092550D1092540D1092BE
:104EE000570D1092560D1092340D1092350D1092F0
:104EF000360D1092370D2DCE1092D90D1092D70D80
:104F00001092D60D1092B60D1092B70D1092B80DEA
:104F10001092B90D1092D10D1092D00D1092DB0DA0
:104F20001092D30D1092D20D1092D50D1092D40D77
:104F30001092B20D1092B30D1092B40D1092B50DE7
:104F40001092DD0C1092DB0C1092DA0C1092BA0C5D
:104F50001092BB0C1092BC0C1092BD0C1092D50C90
:104F60001092D40C1092DF0C1092D70C1092D60C29
:104F70001092D90C1092D80C1092B60C1092B70C5B
:104F80001092B80C1092B90CCCCD0F931F93072F31
:104F9000069510E00F771127282F2F774091EF10FB
:104FA0004F704069E0911218F091131863E070E0BF
:104FB00082E198E109951F910F910895CF92DF92B8
:104FC000EF92FF92CF93DF938091BC0F882309F477
:104FD00071C0813009F4BBC08091BD0F87FD44C012
:104FE00060E2805D0E94FB3A6091ED1084E00E94D7
:104FF000CE178091BC0F811135C061E08091ED101A
:10500000882381F186E00E94CE1760917209617059
:1050100087E00E94CE178091B50C81112AC061E013
:105020008091BC0F823009F060E0462F85E00E943D
:1050300092428091E5099091E6092091E30930912F
:10504000E409237F3093E4092093E309837F90935D
:10505000E6098093E509DF91CF91FF90EF90DF9013
:10506000CF90089560E0CECF60E280E20E94FB3AEC
:10507000BBCF6091B40C85E00E94CE1761E08091B7
:10508000B50C813009F060E082E00E94CE1780917B
:10509000B50C41E0823009F040E061E0813009F474
:1050A00054C083E0DF91CF91FF90EF90DF90CF90DD
:1050B0000C9492428091E3099091E4099D7F909332
:1050C000E4098093E3098091E5099091E6099D7FC9
:1050D0009093E6098093E509C090C00FD090C10F6E
:1050E000E090C20FF090C30FF7FCBECFC701B6012E
:1050F00020E932E040E050E00E94CD6EE90180916D
:10510000BF0F833081F0893171F08F3161F08F30C2
:1051100051F0803141F0BE01882777FD8095982FAE
:105120000E940F3B61CF9E012253310937FD1DC004
:10513000E90161E0C11480E8D806E104F1040CF053
:1051400060E089E00E94CE17E6CF60E0AACF6091D0
:10515000EB107091EC1080E090E00E940F3B6091AA
:10516000BE0F89E00E94CE173FCF319521953109BE
:10517000DFCFCF93C8E18C2F0E947845CF5FC83234
:10518000D1F7CF9108958F929F92AF92BF92CF9215
:10519000DF92EF92FF920F931F93CF93DF931F92B3
:1051A000CDB7DEB7B82E7B0149830E94203E6B2D20
:1051B00081E00E949B4D4981442329F08091B50CE8
:1051C000882309F497C08B2D9AE28902600111248B
:1051D00086EB882E8CE0982E8C0C9D1CF40114829A
:1051E0001582168217820689178964A175A1CB01E1
:1051F000A0E0B0E077276627980140E050E00E94E9
:10520000F46EB901F401378F268FAA24A394A1A6C6
:10521000AA27209FB12D319FC001129FB00D811D83
:105220009A1F309FB00D811D9A1F112480A391A356
:1052300060957095AA27609FB12D719FC001169F40
:10524000B00D811D9A1F709FB00D811D9A1F1124F2
:1052500082A393A380859185A285B3858083918362
:10526000A283B383A7A282EB9DE0C80ED91EF601EC
:1052700014821582168217820689178964A175A186
:10528000CB01A0E0B0E077276627980140E050E02E
:105290000E94F46EB901F601378F268FA1A6AA27C6
:1052A000209FB12D319FC001129FB00D811D9A1F0B
:1052B000309FB00D811D9A1F112480A391A360958A
:1052C0007095AA27609FB12D719FC001169FB00DE8
:1052D000811D9A1F709FB00D811D9A1F112482A3FA
:1052E00093A380859185A285B38580839183A283D2
:1052F000B383A7A2B7018B2D0F90DF91CF911F91A0
:105300000F91FF90EF90DF90CF90BF90AF909F9064
:105310008F900C948B1BFF920F931F93CF93DF936F
:10532000EC01F62E1C821D821E821F820E891F89AF
:105330006CA17DA1CB01A0E0B0E0772766279801A2
:1053400040E050E00E94F46EB9013F8F2E8FF110C3
:1053500023C084E089A719A218A2AA27209FB12DF3
:10536000319FC001129FB00D811D9A1F309FB00D5B
:10537000811D9A1F11248AA39BA388899989AA89D0
:10538000BB8988839983AA83BB83FFA2DF91CF91D6
:105390001F910F91FF90089581E089A7AA27209F70
:1053A000B12D319FC001129FB00D811D9A1F309FFA
:1053B000B00D811D9A1F112488A399A36095709543
:1053C000AA27609FB12D719FC001169FB00D811D4E
:1053D0009A1F709FB00D811D9A1F11248AA39BA351
:1053E00088859985AA85BB8588839983AA83BB8391
:1053F000FFA2DF91CF911F910F91FF9008952F92FF
:105400003F924F925F926F927F928F929F92AF9254
:10541000BF92CF92DF92EF92FF920F931F93CF93A1
:10542000DF93882E742E652E86958695869590E05E
:10543000E82DE770F0E0E95DF84F2081FC01EC5DBC
:10544000F54F662309F4B6C08081822B8083E82D56
:10545000F0E0EE0FFF1FEC5CF54F40835183312CE1
:10546000C0905E09D0905F09E0906009F0906109FA
:1054700080917E0B882309F405C180917C0B8823E1
:1054800031F1282D30E0823009F4DCC7813011F48D
:105490000C94503280E090E028173907A1F0E82FF3
:1054A000E695E695E695F0E0EC5DF54F4081442306
:1054B00051F0FC01E770FF27E95DF84F508154235C
:1054C00011F03324339401968038910529F790E048
:1054D000D6E7AD2EDBE0BD2E1BE0212E9924939460
:1054E000482C512C06E010E0E50189915E018F3FC8
:1054F00009F44DC0C92FDD27C7FDD0952C9E900122
:105500002D9E300D11242C5D354FF901E85EFE4FC4
:105510009082F901E75EFE4F9082F901E65EFE4F50
:105520009082F901EC5EFE4F70826182F901EA5EC1
:10553000FE4F8082F901E95EFE4FA201480F511D26
:105540004083F901E05FFE4FC082D182E282F382A4
:10555000432D672D762D892F16DE40917D0B04C0DB
:10556000C92FDD27C7FDD095CE010196B8010E9455
:105570003B6A9C01982FF901E95DF84F80818423F3
:1055800079F3DCE7AD16DBE0BD0609F0ADCFDF91C6
:10559000CF911F910F91FF90EF90DF90CF90BF9030
:1055A000AF909F908F907F906F905F904F903F90C3
:1055B0002F900895209580812823208390903C0B84
:1055C00070903A0B072D10E0A090470BA091450B6F
:1055D000B0E0E090520B2091500B30E0F0905D0B6A
:1055E00060915B0B70E0C090680B4091660B50E0DF
:1055F000B090730BC091710B2C2E312C80917C0BD1
:10560000823009F49CC280E090E0992009F420C225
:10561000A110E0C3B110F2C1D82EE82FE695E695AF
:10562000E695F0E0EC5DF54FA081AA2309F46FC385
:10563000FC01E770FF27E95DF84FE081EA2309F4F8
:1056400066C30817190709F462C3EE2021F0281772
:10565000390709F45CC3FF2021F06817790709F4C2
:1056600056C3CC2021F04817590709F450C3FC0158
:10567000EE0FFF1FEC5CF54F708061808D2C3324A2
:105680003394EECEE0917D0BCE2FC170E0FF17C0BA
:1056900080913C0B882309F4E1C28091340B9091F6
:1056A000350BA091360BB091370B8C159D05AE05CF
:1056B000BF0528F480913B0B881609F408CF4FEF03
:1056C0005FEFBA019FEF8E2F8270E1FF17C020912C
:1056D000470B222309F4D3C200913F0B1091400BDA
:1056E0002091410B3091420B0C151D052E053F05F5
:1056F00028F42091460B821609F405C724E0A22E57
:10570000AE22E2FF17C03091520B332309F4D3C20B
:1057100000914A0B10914B0B20914C0B30914D0B8B
:105720000C151D052E053F0528F43091510B8316ED
:1057300009F4E6C608E0B02EBE22E3FF17C0F091E0
:105740005D0B0091550B1091560B2091570B30912A
:10575000580BFF2309F4A5C20C151D052E053F05A6
:1057600028F4F0915C0B8F1609F4C7C6AE2FA07118
:10577000E4FF17C0F091680B0091600B1091610B72
:105780002091620B3091630BFF2309F4A6C20C1524
:105790001D052E053F0528F4F091670B8F1609F4BF
:1057A000A9C6BE2FB072E5FF17C0E091730BEE23C0
:1057B00009F49DC240916B0B50916C0B60916D0B85
:1057C00070916E0B4C155D056E057F0528F44091B8
:1057D000720B841609F499C29F3F09F079CEC1116A
:1057E00091C14FEF5FEFBA018823E1F01091450BB3
:1057F000E12FE695E695E695F0E0EC5DF54FD0817A
:10580000D11184C300913F0B1091400B2091410BAB
:105810003091420B041715072607370718F4B90112
:10582000A80191E0AA20E1F01091500BE12FE6953C
:10583000E695E695F0E0EC5DF54FD081D1113EC3E1
:1058400000914A0B10914B0B20914C0B30914D0B5A
:10585000041715072607370718F4B901A80192E0C5
:10586000BB20E1F010915B0BE12FE695E695E69504
:10587000F0E0EC5DF54FD081D11134C30091550BB0
:105880001091560B2091570B3091580B04171507A8
:105890002607370718F4B901A80193E0AA23E1F01D
:1058A0001091660BE12FE695E695E695F0E0EC5D4C
:1058B000F54FD081D11120C30091600B1091610B85
:1058C0002091620B3091630B0417150726073707E9
:1058D00018F4B901A80194E0BB23B1F01091710B49
:1058E000E12FE695E695E695F0E0EC5DF54FD08189
:1058F000DD2309F4D3C2E12FE770F0E0E95DF84F52
:10590000E081ED2309F4CAC29F3F09F0E1CDE091A7
:105910007C0BCC2309F471C4E13009F4B7C508F05D
:105920001DC54091340B5091350B6091360B709131
:10593000370B4F3FFFEF5F076F077F0709F090E0DE
:10594000811166C4F82DAA2009F477C4E13009F466
:105950006FC508F035C500914A0B10914B0B209193
:105960004C0B30914D0B041715072607370708F429
:105970005DC58A019B01B901A801BB2009F467C478
:105980000091550B1091560B2091570B3091580BED
:10599000041715072607370718F4B901A80193E083
:1059A000AA2309F45EC40091600B1091610B209151
:1059B000620B3091630B041715072607370708F4AD
:1059C0003FC58A019B01BB2381F0B901A801009169
:1059D0006B0B10916C0B20916D0B30916E0B0417BB
:1059E00015072607370708F490C19F3F09F4CFCD6C
:1059F0006FCD01968038910509F4DAC0D82EE82FD2
:105A0000E695E695E695F0E0EC5DF54FA081AA23DA
:105A100081F3FC01E770FF27E95DF84FE081EA239D
:105A200041F30817190729F3EE2019F02817390751
:105A300001F3FF2019F068177907D9F2CC2019F08B
:105A400048175907B1F22816390609F010CED1CF00
:105A5000B11063C1A1102EC0D82EE82FE695E695AF
:105A6000E695F0E0EC5DF54FA081AA23C9F0FC01BA
:105A7000E770FF27E95DF84FE081EA2389F0EE2027
:105A800019F02817390761F0FF2019F06817790716
:105A900039F0CC2009F4EBCD4817590709F0E7CDD0
:105AA000019680389105C1F68DC001968038910528
:105AB00009F481C0D82EE82FE695E695E695F0E04A
:105AC000EC5DF54FC081CC2381F3FC01E770FF272B
:105AD000E95DF84FE081EC2341F3A817B90729F3FA
:105AE000EE2019F02817390701F3FF2019F0681785
:105AF0007907D9F2CC2009F4BACD4817590709F033
:105B0000B6CDD3CF50913A0BE52FE695E695E695C5
:105B1000F0E0EC5DF54F40814111DAC14091340B6A
:105B20005091350B6091360B7091370B4F3FEFEF73
:105B30005E076E077E0709F457CE90E055CEFF2032
:105B400009F4EEC1EE2009F41EC2EFE7F0E0A11067
:105B500079C2CF01DE2EAE2FA695A695A695B0E010
:105B6000AC5DB54FFC90FF20F9F0DF01A770BB27BB
:105B7000A95DB84FAC91AF21B9F0992019F00E177B
:105B80001F0791F02E173F0779F06E177F0761F01E
:105B9000CC2019F04E175F0739F0BB2009F467CD10
:105BA0002E163F0609F063CD319798F6992019F02B
:105BB000781409F409C3AA2029F08091450B8815AF
:105BC00009F4ACC38091520B882329F08091500BCB
:105BD000881509F48BC380915D0B882329F080918F
:105BE0005B0B881509F46BC38091680B882329F03F
:105BF0008091660B881509F44BC38091730B882341
:105C000009F4C5CC8091710B8811C1CC1092750B31
:105C100080917F0B8111BBCC1092740B0E94203EAF
:105C200065E081E00E949B4D60E088E89DE073DBC9
:105C300060E084E89EE0DF91CF911F910F91FF908B
:105C4000EF90DF90CF90BF90AF909F908F907F901C
:105C50006F905F904F903F902F905DCB4091340BB1
:105C60005091350B6091360B7091370B4F3FDFEF42
:105C70005D076D077D0709F425CD90E024CD0091E7
:105C80003F0B1091400B2091410B3091420B0417B8
:105C900015072607370708F031CDB901A80191E0B3
:105CA0002DCD041715072607370708F05FCDB9017A
:105CB000A80193E05BCD00914A0B10914B0B209112
:105CC0004C0B30914D0B041715072607370708F0CA
:105CD00031CDB901A80192E02DCD04171507260793
:105CE000370708F05ECDB901A80194E05ACD0091C4
:105CF0006B0B10916C0B20916D0B30916E0B041798
:105D000015072607370708F067CD95E0E1CB019628
:105D10008038910509F080CC4BCFC1102DC0D82E12
:105D2000E82FE695E695E695F0E0EC5DF54F4081CD
:105D30004423C1F0FC01E770FF27E95DF84F508173
:105D4000542381F0AA2019F0A817B90759F0EE20C2
:105D500019F02817390731F0F11038C02816390624
:105D600009F085CC019680389105C9F624CF0196BB
:105D70008038910509F41FCFD82EE82FE695E695D7
:105D8000E695F0E0EC5DF54F1081112381F3FC0105
:105D9000E770FF27E95DF84FE081E12341F3AA2096
:105DA00019F0A817B90719F3EE2019F028173907C9
:105DB000F1F2FF2019F068177907C9F2481759075F
:105DC000B1F22816390609F052CCD1CF68177907FD
:105DD00029F6C8CFE11034C0D82EE82FE695E69515
:105DE000E695F0E0EC5DF54F20812223F9F0FC010F
:105DF000E770FF27E95DF84F30813223B9F00817CB
:105E00001907A1F0A817B90789F0FF2019F0681742
:105E1000790761F0CC2019F04817590739F0BB20F9
:105E200009F425CC2816390609F021CC01968038D2
:105E3000910591F6BDCE01968038910509F4B8CE52
:105E4000D82EE82FE695E695E695F0E0EC5DF54F67
:105E5000E080EE2081F3FC01E770FF27E95DF84F59
:105E6000E081EE2141F38017910729F38A179B0700
:105E700011F382179307F9F2FF2019F0861797079D
:105E8000D1F2CC2019F084179507A9F2BB2009F4B0
:105E9000EECB8215930509F0EACBCDCF00916B0BC9
:105EA00010916C0B20916D0B30916E0B0417150740
:105EB0002607370708F028CD95E00ACBE12FE770D9
:105EC000F0E0E95DF84FE081ED2309F0C9CCB8CCF2
:105ED0005770E52FF0E0E95DF84F5081542309F049
:105EE00080CC1CCEE12FE770F0E0E95DF84FE08157
:105EF000ED2309F0D3CCC2CCE12FE770F0E0E95DEF
:105F0000F84FE081ED2309F0E7CCD6CCE12FE77024
:105F1000F0E0E95DF84FE081ED2309F083CC72CC2D
:105F20006FE770E0992009F4F9C0A110C8C0CB0157
:105F3000D62EE62FE695E695E695F0E0EC5DF54F7A
:105F4000A081AA23E1F0FB01E770FF27E95DF84F8C
:105F5000E081EA23A1F00617170789F0EE2019F077
:105F60002617370761F0CC2019F04617570739F08C
:105F7000BB2009F47CCB2616370609F078CB61509C
:105F80007109A8F615CE2FE730E091102CC0C90199
:105F9000D22EE22FE695E695E695F0E0EC5DF54F22
:105FA00010811123E1F0F901E770FF27E95DF84F57
:105FB000E081E123A1F0AA2019F0A217B30779F03C
:105FC0006217730761F0CC2019F04217530739F0BC
:105FD000BB2009F44CCB2216330609F048CB2150E4
:105FE0003109A8F6E8CDC901D22EE22FE695E69553
:105FF000E695F0E0EC5DF54FF080FF20F9F0F90157
:10600000E770FF27E95DF84FE081EF21B9F0021753
:106010001307A1F0AA2019F0A217B30779F06217AD
:10602000730761F0CC2019F04217530739F0BB20F9
:1060300009F41DCB2216330609F019CB2150310982
:1060400090F6B6CDCF01DE2EEE2EE694E694E694E1
:10605000F12CC4E24C2ECAE05C2EE40CF51CE701E6
:106060006880662049F1C7E0EC2EF12CEE22FF2279
:10607000D7E24D2ED7E05D2EE40CF51CE701F88049
:10608000F620D1F0992019F0E017F107A9F0EA17EE
:10609000FB0791F0E217F30779F0E617F70761F0D5
:1060A000CC2019F0E417F50739F0BB2009F4DFCA5A
:1060B000E215F30509F0DBCA319720F677CDCB0165
:1060C000D62EE62FE695E695E695F0E0EC5DF54FE9
:1060D000F080FF20F9F0FB01E770FF27E95DF84F42
:1060E000E081EF21B9F006171707A1F0A617B7074F
:1060F00089F0EE2019F02617370761F0CC2019F04F
:106100004617570739F0BB2009F4B1CA26163706DF
:1061100009F0ADCA6150710990F64ACDB11029C09D
:10612000CB01D62EE62FE695E695E695F0E0EC5D00
:10613000F54FC081CC23C9F0FB01E770FF27E95D73
:10614000F84FE081EC2389F0AA2019F0A617B707D1
:1061500061F0EE2019F02617370739F0CC2009F44A
:1061600086CA4617570709F082CA61507109C0F6FE
:1061700022CDCB01D62EE62FE695E695E695F0E00A
:10618000EC5DF54F10811123D9F0FB01E770FF277B
:10619000E95DF84FE081E12399F0AA2019F0A617F4
:1061A000B70771F0EE2019F02617370749F0CC2019
:1061B00019F04617570721F02616370609F057CA77
:1061C00061507109B0F6F7CC10923E0B80917F0BB5
:1061D0008111F1CC10923D0B0E94203E60E081E0E5
:1061E0000E949B4D60E086EB9CE095D860E082EBDE
:1061F0009DE091D8A090470BDECC882309F443C0E2
:10620000E13009F4E5C008F0A2C04FEF5FEFBA013A
:1062100000913F0B1091400B2091410B3091420BAC
:10622000041715072607370708F4D0C08A019B0119
:10623000B901A801F82DA1108ECBBB2041F0E130AF
:1062400009F4DBC008F49CCBE23009F4A6C0AA2311
:1062500041F0E13009F4DAC008F4A5CBE23009F4EA
:10626000A5C0BB2309F4C1CBE13009F4D8C008F4C0
:10627000AECBE23009F0B9CB8091720B8F1708F0EA
:10628000B4CB95E025C9F82D4FEF5FEFBA015BCB9A
:1062900010926A0B80917F0B8111AFCC1092690B29
:1062A0000E94203E64E081E00E949B4D60E08EE50C
:1062B0009DE031D860E08AE59EE02DD89ECC10921A
:1062C0005F0B80917F0B81118FCC10925E0B0E942F
:1062D000203E63E081E00E949B4D60E084E39DE00E
:1062E0001AD860E080E39EE016D87ECC1092540B62
:1062F00080917F0B81116FCC1092530B0E94203E36
:1063000062E081E00E949B4D60E08AE09DE003D85E
:1063100060E086E09EE00E948B295DCC1092490BE4
:1063200080917F0B81114ECC1092480B0E94203E31
:1063300061E081E00E949B4D60E080EE9CE00E9465
:106340008B2960E08CED9DE00E948B293BCCF82DE1
:10635000E23071F04FEF5FEFBA01F5CAE23009F0B9
:106360004CCFF0913B0BF81578F1F82D882391F381
:106370008091460B8F1710F4F82F91E0AA2009F4B2
:10638000B5C04FEF5FEFBA018091510B8F1710F43A
:10639000F82F92E0BB2009F45ACF80915C0B8F1745
:1063A00010F4F82F93E0AA2309F45BCF8091670BD8
:1063B0008F1710F4F82F94E0BB2309F416CB5CCFB1
:1063C000E23009F03ACFE0CF90E0D0CF91E030CF8B
:1063D000882DF091460B8F1788F1F82FAA2009F429
:1063E00085C08F2F4FEF5FEFBA01F091510B8F17E0
:1063F00018F1F82FBB2009F42ACF80915C0BF81715
:10640000C8F08F2FF82FAA2309F42BCF8091670BA8
:10641000F81710F4F82F94E0BB2309F4E6CA809132
:10642000720BF81708F0E1CA95E052C892E0A3CACF
:106430008F2FDBCF93E0E6CF92E0DCCF91E0CECFA1
:1064400094E0C1CA80E090E007C033243394019601
:106450008038910509F43BC828173907C1F3E82FA4
:10646000E695E695E695F0E0EC5DF54F4081442336
:1064700071F3FC01E770FF27E95DF84F5081542369
:1064800031F3281739070CF482C8DFCFF0913B0BAA
:106490008F1650F1F82D882309F45CCF8F2F99CFF8
:1064A00080E090E007C03324339401968038910552
:1064B00009F40DC828173907C1F3E82FE695E695CA
:1064C000E695F0E0EC5DF54F4081442371F3FC016B
:1064D000E770FF27E95DF84F5081542331F38217AD
:1064E00093070CF454C8DFCF90E0D5CF4FEF5FEFA8
:1064F000BA01A3CE94E00C94682A93E00C94682A25
:1065000092E00C94682A91E00C94682A10927F0B18
:1065100080917D0B80FF04C090913D0B911188C04C
:1065200081FF04C09091480B911169C082FF04C0A3
:106530009091530B91114AC083FF04C090915E0B60
:1065400091112BC084FF04C09091690B91110CC074
:1065500085FF09C08091740B882329F08091750B09
:10656000882309F47EC0089590916A0B9111F0CFB1
:106570000E94203E64E081E00E949B4D60E08EE539
:106580009DE00E948B2960E08AE59EE00E948B29B5
:106590001092690B80917D0BDBCF90915F0B911175
:1065A000D1CF0E94203E63E081E00E949B4D60E0DD
:1065B00084E39DE00E948B2960E080E39EE00E94DE
:1065C0008B2910925E0B80917D0BBCCF9091540B68
:1065D0009111B2CF0E94203E62E081E00E949B4D6B
:1065E00060E08AE09DE00E948B2960E086E09EE00A
:1065F0000E948B291092530B80917D0B9DCF90911F
:10660000490B911193CF0E94203E61E081E00E94EE
:106610009B4D60E080EE9CE00E948B2960E08CED59
:106620009DE00E948B291092480B80917D0B7ECFBC
:1066300090913E0B911174CF0E94203E60E081E06A
:106640000E949B4D60E086EB9CE00E948B2960E0FD
:1066500082EB9DE00E948B2910923D0B80917D0B77
:106660005FCF0E94203E65E081E00E949B4D60E08C
:1066700088E89DE00E948B2960E084E89EE00E940B
:106680008B291092740B08951092250C1092240CF3
:10669000089510922B0C10922A0C08958091ED1001
:1066A0008823C9F08091EB109091EC100E94873FF5
:1066B0008823B9F08091ED108823D1F00E949C3C92
:1066C0001092BE0F81E09091ED10911101C080E019
:1066D0008093BC0F08958BED90E00E94873F81115D
:1066E000E9CF81E00E94EB3F8091ED108111E6CF70
:1066F0000E94B9288091BE0F20E0E22FF0E0DF0178
:10670000AC58B94FAC91AF3F69F0EE0FFF1FE658A0
:10671000F04FAA0FBB0BAA55B44F8D919C9191835A
:10672000808381E02F5F2E3141F78093BE0FC6CF6B
:10673000FF920F931F93CF93DF93FFB60E94493FC1
:10674000882309F43FC00E94263FC9ECDFE011C056
:10675000FE01E00FF11F808191810E943F3F0E5F9B
:106760001F4F04321105A1F7A49680E1C93ED80756
:1067700019F000E010E0ECCF8091EB109091EC105C
:106780000E943F3F8091E9109091EA100E943F3FA4
:106790008091ED100E941B3F8091EE100E94103FEF
:1067A0008091F0100E941B3F8091EF100E94103FDB
:1067B0008091F1100E941B3F8091F2100E94103FC7
:1067C0000E94A0578F2DDF91CF911F910F91FF90C5
:1067D0000C940E3F0F931F93CF93DF93CDB7DEB78B
:1067E000E6970FB6F894DEBF0FBECDBF92E2E6EBA0
:1067F000F6E0DE01119601900D929A95E1F7813055
:1068000011F58091EE10992787FD9095029661E130
:1068100070E00E943B6A81508093EE1089DF809186
:10682000EE10E1E0F0E0EC0FFD1F92E08902E00DD8
:10683000F11D112462817381CE0183960E945F6EE7
:106840006BE978E022C0823041F58091EF10992702
:1068500087FD9095019660E170E00E943B6A80930D
:10686000EF1066DF8091EF10E1E0F0E0EC0FFD1F2C
:1068700092E08902E00DF11D112462817381CE0145
:1068800083960E945F6E61EA78E0CE0183960E9453
:10689000546ECE018396D3D6C0C08330A1F48091CC
:1068A000C60B9091C70B9093EA108093E91040DFDC
:1068B0000E94864A41E060E070E00E94612487EA1D
:1068C00098E0BDD6AAC08430C9F48091FA12992705
:1068D00087FD9095019666E070E00E943B6A182F54
:1068E0008093FA1269EB78E0CE0183960E945F6E86
:1068F0001F5C1DA3CE018396A2D68FC08530D9F52B
:106900001091F0100091FA12212F30E0002E02C0F9
:10691000359527950A94E2F720FF12C06DEB78E0D9
:10692000CE0183960E945F6E21E030E0002E01C010
:10693000220F0A94EAF7209521232093F01010C02B
:1069400065EC78E0CE0183960E945F6E81E090E076
:10695000002E01C0880F0A94EAF7812B8093F01073
:10696000E7DE8091FA128F5C8DA3CE01839667D605
:106970000E94E04452C0863049F40E94CC568CEC10
:1069800098E05DD68BDE0E94E04447C0873031F44A
:1069900081E00E94EB3F0E94E0443FC0883009F54F
:1069A0008091F110992787FD9095019663E070E042
:1069B0000E943B6A8093F110BBDE8091F110813020
:1069C00041F0823051F0811126C08BED98E037D62E
:1069D00022C084EE98E033D61EC08EEE98E02FD60B
:1069E0001AC08930D1F48091F210992787FD9095D3
:1069F000019662E070E00E943B6A8093F21098DE9C
:106A00008091F210882321F088EF98E018D603C017
:106A100082E099E014D60E94E044E6960FB6F8941E
:106A2000DEBF0FBECDBFDF91CF911F910F910895B3
:106A3000CF93DF932091EE1027FD0BC06F7070E0B5
:106A4000332727FD30956217730719F0DF91CF9137
:106A500008958091ED108823C9F34436B8F7C42F08
:106A6000D0E08091EB109091EC10C817D90771F32A
:106A7000CE010E94873F882349F3D093EC10C09346
:106A8000EB101092BE0F54DEDF91CF910C94E044D6
:106A9000CF93DF9300D0CDB7DEB78091EE1087FDA6
:106AA0000DC06F7070E0992787FD90956817790782
:106AB00029F00F900F90DF91CF91089541111DC0E3
:106AC0003091ED10223008F452C0332391F3842F1B
:106AD00080518E31B8F1842F80558E31B8F0842FDB
:106AE00080538A3108F469C08091BE0F811124C09F
:106AF0000F900F90DF91CF910895413009F44EC06F
:106B0000403409F472C03091ED10DFCFE42FF0E093
:106B1000EE0FFF1FE652F14F8081918188279E7F03
:106B200030E0220F331F220F331F822B932B9183D0
:106B3000808381E08093BE0F0F900F90DF91CF9103
:106B40000C94E044E42FF0E0EE0FFF1FE65AF04F04
:106B5000808191818C7F9170522F550F40E0842B62
:106B6000952B9183808381E08093BE0FE5CF632FC7
:106B7000772767FD7095822F90E06817790709F4F1
:106B8000A4CF2093ED102A834983D2DD87DD0E94B4
:106B9000E0443091ED102A81498197CF822F880FF0
:106BA00010922C0F80932D0F2A8349830E94432338
:106BB0003091ED102A81498188CFE42FF0E0F097E1
:106BC000DF01A05AB04F30E0E852F94F408187E032
:106BD00090E0841B910902C0359527958A95E2F7CC
:106BE0002C9381E08093BE0FA7CF211105C00F9099
:106BF0000F90DF91CF918ACC81E080937F0B59CFAA
:106C000020910F16309110162F5034412130324010
:106C100038F4BC0180E090E04FE054E10C948F57D1
:106C20000895FF920F931F93CF93DF938C01FFB6CC
:106C30000E94493F8823D9F10E94263FC0E0EC2FF3
:106C4000F0E0EE0FFF1FE658F04F808191810E9427
:106C50003F3FCF5FC93199F7D0E0ED2FF0E0E05A28
:106C6000F04F80810E941B3FDF5FD731B1F7EC2FDF
:106C7000F0E0EE0FFF1FE658F04F808191810E94F7
:106C80003F3FCF5FCE3199F78091770F0E941B3F36
:106C90008091780F0E941B3FC6EBDFE089910E9434
:106CA0001B3F8FE0CC3BD807C9F7C801A9DF8F2D68
:106CB000DF91CF911F910F91FF900C940E3F609147
:106CC000C80F8A3030F5681305C0862F865F809321
:106CD000C80F14C0462F552747FD5095282F33273E
:106CE00027FD3095265F3F4F4217530729F4862F23
:106CF0008A508093C80F02C08093C80F8FEF9FEF18
:106D0000DC018093C40F9093C50FA093C60FB0937E
:106D1000C70F8091C80F861741F0B0D68091ED1053
:106D2000811103C08BED90E07CCF0895CF93DF936A
:106D3000DFB70E94F441882309F4A6C00E94B24044
:106D40000E9483420E94F51760E080E090E00E947C
:106D5000DA2480E00E94A24680E00E94754680E02E
:106D60000E945E1B80E00E94484680E00E941B4615
:106D700080E00E94EE4580E00E94311B60E080E0F0
:106D800090E00E94A82480DC84DC60E080E090E059
:106D90000E94D02460E080E090E00E94C62480E35E
:106DA0006BD580E769D582EB67D560E080E090E045
:106DB0000E94A824C2E18C2F0E9494248C2F86501C
:106DC0000E949D24CF5FC831B1F781E00E94A246A6
:106DD00060E08FEF9FEF0E94BC2460E080E090E0D5
:106DE0000E94B224C0E06C2F6E5E8C2F0E94CF46B2
:106DF000CF5FC630C1F780E00E94A24681E00E94CA
:106E00005E1B60E080E090E00E94BC2460E08FEFB9
:106E10009FEF0E94B2246C2F645F8C2F0E94CF469C
:106E2000CF5FCC30C1F780E00E945E1B60E080E065
:106E300090E00E94BC2460E080E090E00E94B224D8
:106E400060E08FEF9FEF0E94A8248C2F0E94942473
:106E5000CF5FC231D1F7CCE06C2F6A5F8C2F0E94DC
:106E6000CF46CF5FC231C1F760E080E090E00E9482
:106E7000A8248C2F0E949424CF5FC831D1F70E94A0
:106E800029190E94834254DC8D2FDF91CF910C94FD
:106E9000EC41EF92FF920F931F93CF93DF931F92DA
:106EA000CDB7DEB7182F7B010E947845E114F104BD
:106EB00009F0E6C0123171F539DF2CC00E9416428C
:106EC00089830E94194291E06981813009F490E040
:106ED000892F0E94325D1EC01B30E1F40E941942CE
:106EE000823091F018F08330A9F407C00E94164256
:106EF000682F83E00E94325D0DC00E941642682F09
:106F000082E00E94325D06C00E941642682F80E037
:106F10000E94325D0E941942082F8823B1F0E114CB
:106F2000F10409F4BAC01D3009F0B3C00E94164242
:106F300061E0811160E0802F0F90DF91CF911F9170
:106F40000F91FF90EF900C94325D173279F4E114B9
:106F5000F10411F045D401C026D484D48091ED1001
:106F600081119EC08BED90E05CDE9AC0EF2809F4A1
:106F70007EC01E3009F088C08091ED10882309F48E
:106F800083C08091BC0F882319F01092BC0F7CC085
:106F900081E08093BC0F78C0812F1CDC68C01C305E
:106FA00099F48091ED10811103C08BED90E039DEF2
:106FB00081E09091ED10911180E08093ED10B8DBAD
:106FC0006DDB0E94E04453C09091BC0F1D3069F40A
:106FD000923039F481E09091ED10911120C080E061
:106FE0001EC082E08093BC0F42C0911103C0812F6C
:106FF00066DE3DC01A3008F03AC0923069F018F4ED
:107000009130A9F503C0953090F50CC01093BD0FD9
:1070100083E08093BC0F2BC01093BD0F84E080935E
:10702000BC0F25C08091BD0F2AE0829F100D112456
:10703000812F1093BD0F943021F4992787FD9095EF
:10704000F0DD8091BD0F992787FD909560D788234B
:1070500051F08091BD0F992787FD90959093EC108A
:107060008093EB1065DB8FEF8093BD0F17DB0F90E4
:10707000DF91CF911F910F91FF90EF900C94E0441E
:107080001A3009F029CF1ACF8091720980FF87CF7B
:1070900083CF173209F06DCF5DCF173241F75CCF48
:1070A000EF2891F7E4CFF5CE3F924F925F926F9227
:1070B0007F928F929F92AF92BF92CF92DF92EF9288
:1070C000FF920F931F93CF93DF931F92CDB7DEB73D
:1070D0007FB6F894882309F425C1A12C9A2C990C29
:1070E000990C990CB6EC8B2E44244A941FE7E12EA0
:1070F000F12CCC24CA940FE7D02E81BA469A9A2D4F
:10710000990F292F26702064892F880F8072907C18
:10711000892B9A2D9695927031E035B928B98BB9A3
:107120009EB987E881BB4DE04A95F1F7000081BA2E
:10713000469A80EE87B997E09AB98DB935B980E45F
:1071400088B91BB88EB987E481BB82E08A95F1F7D4
:1071500000C026B199B18CB181BA479A122F169509
:107160001370A0E82A9F90011124122B292F20715F
:10717000122B292F269526952870122B96959076FE
:10718000192B90E0880F991F84709927182B87EE90
:1071900087B987EF8AB982EE8DB9B92C30E0F0EC6F
:1071A0006F2E690CA8ED5A2E590C07C082508083AF
:1071B00016953F5FB394383001F1EB2DF0E0ED59B7
:1071C000F64F8081982F9E7F89F7012F0170817083
:1071D000081771F3802F8A608083BFE3BB1540F1ED
:1071E000602F772767FD70958B2D39835CDF3981A0
:1071F00016953F5FB394383001F7A394A8E09A0E38
:10720000BFE0BA1508F079CF7FBE0F90DF91CF9124
:107210001F910F91FF90EF90DF90CF90BF90AF90B4
:107220009F908F907F906F905F904F903F900895C8
:107230009091B50C9923D9F1262D230F002309F441
:107240004BC0EDE2FCE0DF0105C04CE0AD3AB40715
:1072500009F48EC08D918F3FC1F3913009F476C04F
:10726000ADE2BCE080E090E004C00196803891057A
:1072700039F04D914F3FC9F7DC01A35DB34F2C931B
:107280008091B40C813009F093CF80818068819324
:107290008DEA9CE08E179F0709F48ACF8081806871
:1072A00081938DEA9CE08E179F0779F781CF352C6B
:1072B000330E40E050E8602F832D39830E94FF2970
:1072C0003981011132C040E4632D8091EF10398380
:1072D0000E94931439816CCF8091B40C811168CFD6
:1072E000913009F44EC0EDE2FCE080E090E004C093
:1072F00001968038910539F041914213F9CFFC0194
:10730000E35DF34F4082EDE2FCE081918F3F09F0B5
:107310004FCF9CE0ED3AF907C1F739830E94B85787
:10732000398146CF88E0A82ED9CE4091EF104F701A
:107330004069E0911218F091131800E4232D63E0E6
:1073400070E082E198E10995398132CF822F90E097
:10735000DC01A35DB34F2C93D701A81BB90BA35D30
:10736000B34F2C938091B40C813009F021CF8DCF95
:107370008091F110811171CFD092B10CC092B00CFC
:107380006CCF822F90E0FC01E35DF34F4082F70168
:10739000E81BF90BE35DF34F4082B5CF80389105D0
:1073A00038F4FC01E050FF4F208130E0C90108951E
:1073B0002FEF3FEFFBCFCF93DF93CFE0D6E1E88114
:1073C000F98185EA96E1A1E6B0E081939193A193DA
:1073D000B193F983E883DF91CF9108958091F11003
:1073E000813009F00895683F59F06A3FD9F78FEF6F
:1073F0009FE79093B10C8093B00C10925F0F0895AB
:1074000080915F0F8F5F80935F0F0895AFE0B6E1CB
:10741000ED91FC9111978191ED93FC930895AFE06C
:10742000B6E1ED91FC9111978191ED93FC93089554
:10743000AFE0B6E1ED91FC91119780819181329698
:10744000ED93FC930895AFE0B6E1ED91FC911197B7
:1074500060817181828193813496ED93FC930895CC
:10746000E82FE695E695E695F0E0EC5DF54F908126
:10747000992351F08770E82FF0E0E95DF84F208103
:10748000292381E009F0089580E00895FC01A18D91
:10749000BB27A1950CF4B095AA0FBB1F11962085B0
:1074A0003185428553850E94C76E648775878687BC
:1074B00097870895CF92DF92EF92FF92CF93603E2D
:1074C000710581059105F8F4DC01CB019F5FAF4F99
:1074D000BF4FCC24D82EE92EFA2EA0E0B0E020E059
:1074E00030E0EBBEF601C791A40FB51FCC932F5F20
:1074F0003F4FD9018FEFC81AD80AE80AF80A2115B8
:1075000081E0380771F7CF91FF90EF90DF90CF9037
:107510000895CF93DF93BC0180E090E04FE054E109
:10752000C9DFCFE0D4E1D0931016C0930F161092AC
:10753000111689DF653A76418146910551F080E068
:1075400092E0FE019C01119221503040E1F780E071
:1075500004C065DF8093111681E0DF91CF9108951B
:10756000AF92BF92CF92DF92EF92FF920F931F9351
:10757000CF93DF935C01C12CD12C7601C0E0D0E029
:10758000062F10E00EC0A601415F5B4EBE016A0DE2
:107590007B1D80E090E08EDF21962FEFD21AE20A69
:1075A000F20AC017D10778F3CFE0D4E1D0931016D8
:1075B000C0930F161092111646DF653A7641814648
:1075C000910551F080E092E0FE019C011192215062
:1075D0003040E1F780E004C022DF8093111681E0A3
:1075E000DF91CF911F910F91FF90EF90DF90CF909F
:1075F000BF90AF900895CF93DF931F92CDB7DEB7C2
:1076000090E06983CBDE8093E7096981862F90E063
:10761000C5DE8093E8090F90DF91CF91089524E6AD
:1076200030E040E050E00E94CD6E2AE030E040E0E3
:1076300050E00E94CD6E605D822F805DDCCF21E046
:107640002093ED09009721F48FEF8093EC090895C2
:107650001092EC09BC0183EF99E00E945F6E6BE52C
:1076600079E082EF99E00C94546E10923C0B1092EA
:107670003E0B8FEF80933B0B80933A0B1092340BB1
:107680001092350B1092360B1092370B1092470B5D
:107690001092490B8093460B8093450B10923F0B41
:1076A0001092400B1092410B1092420B1092520B11
:1076B0001092540B8093510B8093500B10924A0BF5
:1076C00010924B0B10924C0B10924D0B10925D0BC5
:1076D00010925F0B80935C0B80935B0B1092550BA9
:1076E0001092560B1092570B1092580B1092680B79
:1076F00010926A0B8093670B8093660B1092600B5D
:107700001092610B1092620B1092630B1092730B2C
:107710001092750B8093720B8093710B10926B0B10
:1077200010926C0B10926D0B10926E0B08951F93BC
:10773000CF93DF93D82FC92F162F80917E0B68131C
:107740000AC046E050E066E77BE08D2F0E94266E7F
:10775000009711F424C089DF10937E0B46E050E0BF
:107760006FEF70E086E79BE00E944D6EED2FFC2FDF
:10777000A6E7BBE080E091919F3F19F4882341F098
:1077800004C09D938F5F8630B1F71092760B07C0CF
:1077900086E0E6E7FBE0DF011D928A95E9F7DF91DD
:1077A000CF911F910895CF93DF9300D000D000D0E8
:1077B000CDB7DEB786E0E2EFF6E0DE01119601908C
:1077C0000D928A95E1F760E0CE010196B0DF269632
:1077D0000FB6F894DEBF0FBECDBFDF91CF910895F5
:1077E000EF92FF920F931F93CF93DF9300D000D0BF
:1077F00000D0CDB7DEB746E050E06FEF70E08E010D
:107800000F5F1F4FC8010E944D6EF12CE12C8F2D90
:1078100027DE8823A9F0F801EE0DF11DE7FCFA95AB
:10782000F082EE2021F089819F2D981B9083E394B4
:1078300085E08E152CF461E0CE01019678DF05C05D
:10784000F39490E8F912E3CFF6CF26960FB6F894AA
:10785000DEBF0FBECDBFDF91CF911F910F91FF9083
:10786000EF90089586E0E6E7FBE0A6EBBFE001902D
:107870000D928A95E1F7089596EC91BB469A482FB0
:10788000440F282F2695342F36703064982F991F77
:107890009927991F392B8071942F990F9072982BEB
:1078A000407C942B2270206615B838B99BB92EB94C
:1078B00087E881BB85E08A95F1F70000089555E0DF
:1078C0005A95F1F7000036EC31BB469A80EE87B945
:1078D00097E09AB98DB915B880E488B91BB880E2F1
:1078E0008EB987E481BB82E08A95F1F700C026B1AA
:1078F00099B18CB131BB479A37EE37B937EF3AB906
:1079000032EE3DB9422F4695437050E8259F9001D5
:107910001124422B292F2071422B292F26952695A1
:107920002870422B96959076492B90E0880F991FEE
:1079300084709927842B08951092820B1092830BE8
:107940001092840B1092850B8FEF8093E70B80933E
:10795000BF0F8FEF9FEFDC018093C00F9093C10F9B
:10796000A093C20FB093C30F0895CF93DF93CDB709
:10797000DEB728970FB6F894DEBF0FBECDBF92E0FA
:107980009D8393E09E8325E02F833CE03887298305
:107990009A8391E09B831C82823081F134F48823A6
:1079A00061F0813009F061C013C0843009F450C027
:1079B000D4F1853009F059C052C0440F551F661FDD
:1079C000771F8091690F8170842B8093690F4DC060
:1079D00080916B0F8F7C413051056105710521F459
:1079E000806180936B0F41C0423051056105710584
:1079F00009F001C0806280936B0F37C0DB01CA01C0
:107A000081709927AA27BB2721E0822780936F0FD7
:107A1000427055276627772775956795579547953F
:107A20004093790F22C0DB01CA0181709927AA27F0
:107A3000BB2721E0822780936D0F42705527662770
:107A40007727759567955795479540936E0F0DC0AD
:107A5000FE01E40FF51F85818093730F06C0FE01C0
:107A6000E40FF51F81818093750F28960FB6F89467
:107A7000DEBF0FBECDBFDF91CF910895BF92CF92F1
:107A8000DF92EF92FF920F931F93CF93DF93CDB7C7
:107A9000DEB764970FB6F894DEBF0FBECDBF00917E
:107AA000C80F8CE00802800111240C571A4F44DFE4
:107AB000D80112966D917C911397CE0101960E9488
:107AC0005F6E69E579E0CE0101960E94546EF8017F
:107AD00080818130B9F020F0823009F05AC025C091
:107AE000E181EE0FFF0BE658F04F80819181A0E01D
:107AF000B0E08093C00F9093C10FA093C20FB093DA
:107B0000C30F47C0E181FF27E7FDF095E05AF04F32
:107B10008081F801E80FF11DE80FF11D6481758186
:107B2000CE0101960E94546E34C08AE1E0E6FFE087
:107B3000A2E1B6E101900D928A95E1F7C12CD12C1A
:107B40007601B701A601F80181810FDF4AE150E01B
:107B500060E67FE082E196E10E94266E009771F474
:107B6000F8018C2D92E08902E00DF11D1124648151
:107B70007581CE0101960E94546E0BC0AFEFCA1AF8
:107B8000DA0AEA0AFA0AB4E0CB16D104E104F104F5
:107B9000C1F6CE01019653DD64960FB6F894DEBFB0
:107BA0000FBECDBFDF91CF911F910F91FF90EF904E
:107BB000DF90CF90BF9008958F929F92AF92BF9227
:107BC000CF92DF92EF92FF920F931F934A015B01D6
:107BD00068017901BC0180E090E00E948F6B9058B1
:107BE000A50194010E94CA6A0E94376BA701960101
:107BF0000E94EF6C0E94636BCB011F910F91FF906D
:107C0000EF90DF90CF90BF90AF909F908F900895AE
:107C10000F931F938091AC0F9091AD0F00E010E493
:107C20002CE135E440E050E86BE376E480959095F4
:107C3000C3DF90935E0F80935D0F1F910F910895A6
:107C40008091240A9091250A892B9091260A892BEC
:107C50009091270A892B9091280A892B9091290AC3
:107C6000892B90912A0A892B90912B0A892B90912C
:107C70002C0A892B90912D0A892B90912E0A892B01
:107C800090912F0A892B9091300A892B9091310A7B
:107C9000892B9091320A892B9091330A982B21E0FD
:107CA00009F420E08091520B9091470B892B909121
:107CB0005D0B892B9091680B892B90913C0B892B44
:107CC0009091730B892B59F48FEF9FEFDC01809318
:107CD000590F90935A0FA0935B0FB0935C0F222320
:107CE000A1F08091FF12811110C080915E099091E6
:107CF0005F09A0916009B09161098093590F909339
:107D00005A0FA0935B0FB0935C0F2093FF1208955E
:107D10000F931F93CF93DF93EC018A899B8900E037
:107D20001FEF2FE737E440E050E26BE476E4809504
:107D3000909542DFAC0160E070E0088C04C0440F15
:107D4000551F661F771F0A94D2F7488759876A879D
:107D50007B87DF91CF911F910F910895CF93DF9390
:107D6000EC01888D681739F0688FCE01D1DFCE0124
:107D7000DF91CF918BCBDF91CF910895CF93DF939C
:107D8000EC01598B488B8A899B896817790741F0E8
:107D90007B8B6A8BCE01BCDFCE01DF91CF9176CB9E
:107DA000DF91CF910895AC01AA27469FB12D579F2F
:107DB0009001749FB00D211D3A1F569FB00D211DDB
:107DC0003A1F1124C9010895A72F8F3FF9F0282FDA
:107DD0002F5F30E0220F331FE82FF0E0EE0FFF1F80
:107DE000E40FF51F60817181FA01E20FF31F8081BA
:107DF0009181861B970B892F9927A89F9001A99F96
:107E0000300D1124260F371FC90108952EEF31E0E0
:107E1000E3CF8FBF0895F89481E008958FBF089550
:107E2000EFE0F6E1A081B1818C9380819181019690
:107E3000918380830895EFE0F6E1A081B1818C9376
:107E4000808191810196918380830895CF93DF9300
:107E5000EFE0F4E180E092E0DF019C011D9221500F
:107E60003040E1F7F0931016E0930F16C1E1D6E130
:107E700084E08883A0DA8881DF91CF91DCCFAFE006
:107E8000B6E1ED91FC91119781939193ED93FC9361
:107E90000895F89481E00895CF92DF92EF92FF92D7
:107EA0000F931F93CF93DF931F92CDB7DEB7F82EBA
:107EB0008B01EFB69983EDDF99818823E9F08F2D4F
:107EC00028DBEFE0F5E16F018FE094E1C81AD90AF1
:107ED00082918823C1F3F092121623E136E1EFE09C
:107EE000F4E1A601BF01C9010E94336E9FEFC91AD8
:107EF000D90AF801D182C0828E2D0F90DF91CF91E7
:107F00001F910F91FF90EF90DF90CF9087CF1F933D
:107F1000CF93DF93EC011FB7BCDF811104C0812F29
:107F20007DDFC1E053C0CE01F4DA882309F44BC0F1
:107F30001092720F1092B60F9FEF9093B70F90931D
:107F4000B80F9093B90F9093BA0F9093BB0F809195
:107F50001116811102C0C1E037C0C0E069DAEC2F10
:107F6000F0E0EE0FFF1FE658F04F91838083CF5F64
:107F7000C931A1F7D0E053DAED2FF0E0E05AF04F2D
:107F80008083DF5FD731B9F780911116823018F303
:107F90004FDAEC2FF0E0EE0FFF1FE658F04F918321
:107FA0008083CF5FCE31A1F73ADA8093770F37DA4B
:107FB0008093780FC6EBDFE032DA89938FE0CC3B19
:107FC000D807D1F7ACCFC0E0812F28DF8C2FDF910D
:107FD000CF911F9108951F93CF93DF93182FDFB791
:107FE00058DF882309F448C08CE5E0E6FFE0DF01B4
:107FF0001D928A95E9F72FEF3FE730937F0F20938B
:108000007E0F3093850F2093840F4FEF5FEF5093D7
:10801000890F4093880F30938D0F20938C0F5093CE
:10802000990F4093980F50937D0F40937C0F30939E
:10803000A90F2093A80F3093B50F2093B40F30935E
:10804000AF0F2093AE0F85E08093730FC1E0C09314
:10805000740FC0936D0FC0936F0FC093750F82E0C4
:108060008093760F46E050E06FEF70E086EB9FE084
:108070000E944D6E111105C08D2FDF91CF911F9180
:10808000CDCEC093600FF8CFFF920F931F93CF9385
:10809000DF93FFB6FEDE811104C08F2DBFDEC1E08D
:1080A0005AC062E08CED90E05BDA882309F450C09E
:1080B0008FE38093F0101092F210809111168823B4
:1080C00019F0C9ECDFE012C0C1E043C0B1D9FE0134
:1080D000E00FF11F918380830E5F1F4F0432110563
:1080E000A9F7A49680E1C93ED80719F000E010E096
:1080F000EDCF9ED99093EC108093EB1099D990938B
:10810000EA108093E9108BD98093ED107FD980938A
:10811000EE10809111168230B8F281D98093F01060
:1081200075D98093EF1080911116833068F277D95A
:108130008093F11080911116843008F4C5CF66D970
:108140008093F21080911116853008F0A6CFBCCF35
:10815000C0E08F2D63DE8C2FDF91CF911F910F91A7
:10816000FF900895BF92CF92DF92EF92FF920F930C
:108170001F93CF93DF931092FE12C0E0D0E0B4E2E1
:10818000BB2E0CC00193119313870287778B668BEC
:108190008150C1F72196C830D10591F16C2F772716
:1081A00067FD7095872F972F0E94916B6B017C0163
:1081B0002CE83EE24AEB55E40E94EF6C20E030E40C
:1081C0004CE955E40E94636A0E94636B8B012CE8C2
:1081D0003EE24AE355E4C701B6010E94EF6C20E09D
:1081E00030E44CE156E40E94636A0E94636BBC9EDB
:1081F000F001BD9EF00D1124E753F04F86E0C2CF91
:10820000DF91CF911F910F91FF90EF90DF90CF9072
:10821000BF900895CF93CFB73CDE8823B1F02AE218
:1082200031E0E9ECFFE0DF01C9011D920197E9F7B8
:108230002FEF3FE73093EA102093E9108FEF809300
:10824000EE108FE38093F0108DDF8C2FCF91E6CD71
:10825000EF92FF920F931F93CF93DF93F82EE62EAA
:10826000ABEA8A9FA12D1124A695A695A6951A2F53
:108270001F5F50E0A83008F06AC08A2F90E0880F96
:10828000991FFC01EE0FFF1FEE0FFF1FEE0FFF1FE8
:10829000E80FF91FE40FF51FEE0FFF1FE753F04F34
:1082A000C081D181183008F476C0FA01EE0FFF1FAB
:1082B000EB53FF4E0190F081E02DDA01AA0FBB1FB6
:1082C000AF55BF4E8D919C919F01281B390BA12F5B
:1082D000B0E017970E94356A6E0F7F1F811D911DB8
:1082E0006115710521E08207910508F06AC08B01D4
:1082F0000C1B1D0B3E2D20E09BEAF99E912D1124B5
:10830000969596959695892F880F890F880F880FD7
:108310006F2D681B862F90E0A0E0B0E077276627DE
:10832000620F731F811D911D2CE030E040E050E092
:108330000E94F46ED8010E94BD6EC80FD91FCE01F5
:10834000DF91CF911F910F91FF90EF900895FA0167
:10835000EE0FFF1FEB53FF4E0190F081E02DEA017D
:10836000CC0FDD1FCF55DF4E888199819F01281BDF
:10837000390BB0E017970E94356A6E0F7F1F811D81
:10838000911D6115710521E082079105F8F4EB015B
:10839000183008F08ACF812F90E0880F991FFC01D8
:1083A000EE0FFF1FEE0FFF1FEE0FFF1FE80FF91F6D
:1083B000E40FF51FEE0FFF1FE753F04F608171814F
:1083C00096CF6FEF7FEF80E090E091CF6FEF7FEF80
:1083D00080E090E0EB01DCCF8FBF0895EDEFF2E19C
:1083E00080818F5F80830895F89481E00895CF9312
:1083F000DF93EC016A8F88819981AA81BB81892BE7
:108400008A2B8B2B51F460915E0970915F098091EA
:108410006009909161090E94B46E0E94B16E6883F8
:1084200079838A839B83DF91CF9108958091B40CE7
:1084300008958091B50C08950F931F93CF93DF9308
:10844000FC018BE1DF011D928A95E9F70AEF10E14B
:1084500060E070E080E89FEBC0E0D0E01BC0BE01B0
:10846000882777FD8095982F0E94916B21E830E84E
:1084700040E85BE30E94EF6C20E030E040E85FE31F
:108480000E94636A2BED3FE049E450E40E94EF6CE8
:108490000E94C76A20E030E040E85FE30E94636A20
:1084A00020E03FEF4FEF56E40E94EF6C0E94636BB9
:1084B000F801619371938F012196C115F1E0DF07F7
:1084C00071F6DF91CF911F910F9108950F931F9334
:1084D000082F10E0F801E45BFE4F8491F801E45BA3
:1084E000FD4F9491F801E45BFC4F049110E020E013
:1084F00030E0980111270027192B082BB801C9017A
:108500001F910F9108951092E7091092E8091092B7
:10851000E4091092E3091092E6091092E50910921D
:10852000ED09089521E030E002C0220F331F8A9543
:10853000E2F7D901A095B095E091E309F091E40943
:10854000EA23FB23F093E409E093E3098091E50932
:108550009091E6098A239B239093E6098093E5098D
:10856000662331F0E22BF32BF093E409E093E30967
:10857000442331F0282B392B3093E6092093E50969
:1085800008952F923F924F925F926F927F928F92B7
:108590009F92AF92BF92CF92DF92EF92FF920F9392
:1085A0001F93CF93DF93CDB7DEB729970FB6F8941B
:1085B000DEBF0FBECDBF782E662E4A831092FD120D
:1085C00070E080E090E00E948F6B9B01AC0160E066
:1085D00070E080E090E40E94526D24EA30ED42E8C1
:1085E00051E40E94EF6C9B01AC0160E074E284EF07
:1085F00099E40E94CA6A6B837C838D839E83262DB7
:10860000235081E090E0022E01C0880F0A94EAF71F
:1086100089833EE0532E00E010E88FEF9FEF9987AB
:108620008887E22FFF27E1950CF4F0954F01AA24EB
:1086300097FCA094BA2C672D8A810E94AE152885DC
:1086400039858217930768F5B901872D0E948B241D
:1086500089810E94181A6B017C016F3F3FEF7307FD
:108660008307930709F44FC0C501B4010E94916BC1
:108670009B01AC0160E070E080E090E40E94526DEC
:108680001B01482E9F83C701B6010E948F6B9B017F
:10869000AC01FF80622D732D842D9F2D0E94EF6C05
:1086A00004C06FEF7FEF8FE79FE7BB81AC81ED8167
:1086B000FE802B2F3A2F4E2F5F2D0E947B6C1816B9
:1086C0003CF488859985800F911F9987888706C01B
:1086D000E885F985E01BF10BF987E8871695079582
:1086E0005A9409F0A8CF22E1629EF0011124E70D0F
:1086F000F11DEE0FFF1FE753F04F88859985918399
:10870000808380E001C08FEF29960FB6F894DEBF1A
:108710000FBECDBFDF91CF911F910F91FF90EF90D2
:10872000DF90CF90BF90AF909F908F907F906F9091
:108730005F904F903F902F90089580912C0C8E7FEA
:108740009091600F9111816080932C0C4FB7F89439
:1087500080912C0C96EC91BB469A382F330F982FB2
:108760009695232F26702064582F551F5527551F87
:10877000252B582F5071832F880F8072852B307CCA
:10878000832B9270906631E035B928B98BB99EB9C8
:1087900087E881BB4FBF80912C0C877F9091630F3E
:1087A0009111886080932C0C4FB7F89480912C0C19
:1087B00096EC91BB469A382F330F982F9695232F1E
:1087C00026702064582F551F5527551F252B582FCD
:1087D0005071832F880F8072852B307C832B927091
:1087E000906631E035B928B98BB99EB987E881BB6D
:1087F0004FBF80912C0C8D7F9091610F9111826001
:1088000080932C0C4FB7F89480912C0C96EC91BB74
:10881000469A382F330F982F9695232F2670206471
:10882000582F551F5527551F252B582F5071832F13
:10883000880F8072852B307C832B9270906631E09C
:1088400035B928B98BB99EB987E881BB4FBF8091F4
:108850002C0C8F7E9091640F9111806180932C0C71
:108860004FB7F89480912C0C96EC91BB469A382F18
:10887000330F982F9695232F26702064582F551F5D
:108880005527551F252B582F5071832F880F807225
:10889000852B307C832B9270906631E035B928B9F6
:1088A0008BB99EB987E881BB4FBF80912C0C8B7F21
:1088B0009091660F9111846080932C0C4FB7F894BF
:1088C00080912C0C96EC91BB469A382F330F982F41
:1088D0009695232F26702064582F551F5527551F16
:1088E000252B582F5071832F880F8072852B307C59
:1088F000832B9270906631E035B928B98BB99EB957
:1089000087E881BB4FBF80912C0C8F7D9091670FC2
:108910009111806280932C0C4FB7F89480912C0CAD
:1089200096EC91BB469A382F330F982F9695232FAC
:1089300026702064582F551F5527551F252B582F5B
:108940005071832F880F8072852B307C832B92701F
:10895000906631E035B928B98BB99EB987E881BBFB
:108960004FBF80912C0C8F7B9091680F9111806488
:1089700080932C0C4FB7F89480912C0C96EC91BB03
:10898000469A382F330F982F9695232F2670206400
:10899000582F551F5527551F252B582F5071832FA2
:1089A000880F8072852B307C832B9270906631E02B
:1089B00035B928B98BB99EB987E881BB4FBF0895F7
:1089C000CF938091240A9091250A892B9091260AB1
:1089D000892B9091270A892B9091280A892B9091B5
:1089E000290A892B90912A0A892B90912B0A892B8D
:1089F00090912C0A892B90912D0A892B90912E0A07
:108A0000892B90912F0A892B9091300A892B909174
:108A1000310A892B9091320A892B9091330A982B35
:108A200021E009F420E08091520B9091470B892BB3
:108A300090915D0B892B9091680B892B90913C0B49
:108A4000892B9091730B892B59F48FEF9FEFDC01E9
:108A50008093590F90935A0FA0935B0FB0935C0FC4
:108A6000222321F08091FF12882359F12093FF12D5
:108A7000CFD863DE8091710F811134C00E94D33B47
:108A8000C091F01080917D0BC81721F00E94353BFA
:108A9000C0937D0BC091720F80917C0BC81731F091
:108AA0000E94353BC33058F4C0937C0B0E94432393
:108AB0000E94CC1B0E946A16CF910C94DE27C0E066
:108AC000F3CF80915E0990915F09A0916009B09108
:108AD00061098093590F90935A0FA0935B0FB09345
:108AE0005C0FC4CF61E086EB9FE00E94973BC8CF4C
:108AF000E82FF0E0ED59F64F90819170803209F443
:108B000056C078F0843209F44CC0A0F1863209F4E2
:108B100045C008F058C09093670F81E08093BE0F66
:108B20004FCF8C31C8F08C3109F444C0809180095A
:108B3000817090916B0F9073892B9091810990FDBA
:108B400047C090E0892B9091820990FF45C092E048
:108B5000892B80936B0FE1CF8A31A8F080917E0939
:108B6000817090917D0990FD35C090E0892B8093B4
:108B70006C0FD3CF8232C1F018F09093630FCDCF3A
:108B80009093610FCACF883131F0893109F008958F
:108B90009093650FC2CF9093620FBFCF9093680FF1
:108BA000BCCF9093640FB9CF9093660FB6CF9093DC
:108BB000600FB3CF90917F098091690F90FB80F98E
:108BC0008093690FAACF873211F79093710FA5CFC9
:108BD00098E0B8CF92E0CACF90E0BACF90912C0C39
:108BE0009F7B8111906490932C0C4FB7F8948091E7
:108BF0002C0C96EC91BB469A382F330F982F9695F4
:108C0000232F26702064582F551F5527551F252BBD
:108C1000582F5071832F880F8072852B307C832BC7
:108C20009270906631E035B928B98BB99EB987E862
:108C300081BB4FBF089590912C0C9F7D8111906254
:108C400090932C0C4FB7F89480912C0C96EC91BB20
:108C5000469A382F330F982F9695232F267020642D
:108C6000582F551F5527551F252B582F5071832FCF
:108C7000880F8072852B307C832B9270906631E058
:108C800035B928B98BB99EB987E881BB4FBF089524
:108C900090912C0C9F7E8111906190932C0C4FB77A
:108CA000F89480912C0C96EC91BB469A382F330F98
:108CB000982F9695232F26702064582F551F5527DF
:108CC000551F252B582F5071832F880F8072852BAD
:108CD000307C832B9270906631E035B928B98BB91E
:108CE0009EB987E881BB4FBF089590912C0C9D7F62
:108CF0008111926090932C0C4FB7F89480912C0CBA
:108D000096EC91BB469A382F330F982F9695232FC8
:108D100026702064582F551F5527551F252B582F77
:108D20005071832F880F8072852B307C832B92703B
:108D3000906631E035B928B98BB99EB987E881BB17
:108D40004FBF089590912C0C9E7F8111916090935C
:108D50002C0C4FB7F89480912C0C96EC91BB469A52
:108D6000382F330F982F9695232F26702064582F75
:108D7000551F5527551F252B582F5071832F880FAE
:108D80008072852B307C832B9270906631E035B9F0
:108D900028B98BB99EB987E881BB4FBF08950F935F
:108DA0001F93CF93DF93D82F062F8093FE12862F29
:108DB0000E949D24DC3008F057C013E04CE0612F86
:108DC0008D2FDFDB811103C01F5F1730B9F7ED2F47
:108DD000F0E0DF01AA0FBB1FAB5CBF4E8D919C91F1
:108DE0009C01220F331FDF01AA0FBB1FA75ABF4EE2
:108DF0004D915C91241B350BDF01AA0FBB1FAF5EA9
:108E0000BF4E2D933C93A901440F551F481B590B8E
:108E1000DF01AA0FBB1FA351B04F4D935C93440FCA
:108E2000551FDF01AA0FBB1FA753B04F421B530BA7
:108E30004D935C93DF01AA0FBB1FAB53BF4ECF0115
:108E4000880F991F8F559F4EEC0128813981220F81
:108E5000331FEE0FFF1FE358FF4E80819181281BC7
:108E6000390B2D933C9323C014E044E2612F8D2FE6
:108E700088DB882341F0ED2FF0E0EE0FFF1FE75A6B
:108E8000FF4E44E004C01F5F183079F7F4CFDF01D4
:108E9000949720813181220F331F84A195A1281B33
:108EA000390B11963C932E934150FD0181F7802F91
:108EB0000E949424DF91CF911F910F910C94291956
:108EC00036EC20EE97E0A0E8F7E4E7EE77EF62EE0D
:108ED0005FB7F89431BB469A27B99AB92DB915B83E
:108EE000A8B99BB91EB8F1BB42E04A95F1F700C0A2
:108EF00046B1B9B1BCB131BB479AE7B97AB96DB9DE
:108F00005FBF55E05A95F1F7000042FFE1CF5FB730
:108F1000F89496EC91BB469A382F330F982F96957C
:108F2000232F26702068482F441F4427441F242BDA
:108F300080718360432F440F4072842B307C832BDD
:108F40009270906215B828B98BB99EB987E881BB39
:108F500085E08A95F1F700005FBF0895EF92FF92D8
:108F60000F93CF93DF931F92CDB7DEB77B016115CF
:108F7000710539F40F90DF91CF910F91FF90EF9031
:108F80000895842F29839CDF298182E0E816F1046B
:108F900088F3822F95DFE2E0EE16F10459F3802F7B
:108FA0000F90DF91CF910F91FF90EF9089CF26EC3A
:108FB00090EE87E0F0E8E7E477EE67EF52EE4FB728
:108FC000F89421BB469A97B98AB99DB915B8F8B9F2
:108FD0008BB91EB8E1BB32E03A95F1F700C036B16B
:108FE000A9B1ACB121BB479A77B96AB95DB94FBF96
:108FF00045E04A95F1F7000032FFE1CF8FB7F894D2
:1090000096EC91BB469A15B890E898B993E09BB955
:1090100090E29EB997E891BB95E09A95F1F7000030
:109020008FBF089526EC90EE87E0F0E8E7E477EE56
:1090300067EF52EE4FB7F89421BB469A97B98AB9B9
:109040009DB915B8F8B98BB91EB8E1BB32E03A95B5
:10905000F1F700C036B1A9B1ACB121BB479A77B9DD
:109060006AB95DB94FBF45E04A95F1F7000032FF9C
:10907000E1CF8FB7F89496EC91BB469A15B892E879
:1090800098B993EC9BB990E29EB997E891BB95E0B3
:109090009A95F1F700008FBF089526EC90EE87E0D7
:1090A000F0E8E7E477EE67EF52EE4FB7F89421BBB4
:1090B000469A97B98AB99DB915B8F8B98BB91EB84F
:1090C000E1BB32E03A95F1F700C036B1A9B1ACB1DD
:1090D00021BB479A77B96AB95DB94FBF45E04A9558
:1090E000F1F7000032FFE1CF8FB7F89496EC91BB17
:1090F000469A15B894E898B993E19BB992E29EB963
:1091000097E891BB95E09A95F1F700008FBF08951D
:1091100026EC90EE87E0F0E8E7E477EE67EF52EEBA
:109120004FB7F89421BB469A97B98AB99DB915B83B
:10913000F8B98BB91EB8E1BB32E03A95F1F700C03F
:1091400036B1A9B1ACB121BB479A77B96AB95DB95B
:109150004FBF45E04A95F1F7000032FFE1CF8FB7EE
:10916000F89496EC91BB469A15B892E898B993E0BA
:109170009BB990E29EB997E891BB95E09A95F1F77B
:1091800000008FBF089526EC90EE87E0F0E8E7E45A
:1091900077EE67EF52EE4FB7F89421BB469A97B936
:1091A0008AB99DB915B8F8B98BB91EB8E1BB32E0E0
:1091B0003A95F1F700C036B1A9B1ACB121BB479ADD
:1091C00077B96AB95DB94FBF45E04A95F1F700003C
:1091D00032FFE1CF9FB7F89486EC81BB469A15B871
:1091E00087E888B923ED2BB922E22EB981BB85E04F
:1091F0008A95F1F700009FBF0895CF93882339F136
:109200008091E9098F5F8093E909853148F081E019
:109210009091EA099111CDC08093EA091092E90971
:10922000C091ED09C11179C05091E7099091E80909
:10923000E091EE09E13009F4DEC008F4AFC0E2309D
:1092400009F4C4C020E0F0E0ED51F64F2487AFB739
:10925000F89456EC51BB469A41E045B980E488B990
:109260001BB880E28EB937E831BB00C000C080E196
:1092700090E00090EE0902C0880F991F0A94E2F76F
:10928000282F51BB469A782F770F682F6695221F9B
:109290002227221F972F9670292B20648071972FE9
:1092A000990F9072982B707C972B627045B928B9F2
:1092B0009BB96EB931BB00C000C0E091EE09F0E08F
:1092C000ED51F64F848551BB469A582F550F982F74
:1092D0009695252F26702064682F661F6627661FC7
:1092E000262B682F6071852F880F8072862B507C0B
:1092F000852B9270906245B928B98BB99EB931BB64
:10930000AFBF8091EE0990E0019663E070E00E94AB
:109310003B6A8093EE09CF9108954091EB094F5F2E
:109320004093EB09E2EFF9E001900020E9F7E35FF9
:10933000F9402091EC09332727FD3095C9010196AA
:109340006E2F772767FD70950E943B6AF901ED51FA
:10935000F64F278530E02038310588F15FEFE82FA0
:10936000FF27E7FDF095ED51F64F278530E02038D7
:10937000310550F5F901E050FF4F9081403108F47C
:1093800057CF8093EC091092EB09811151CF1C1635
:109390000CF04ECFC150C093ED094ACF2091E309A4
:1093A0008091EA09882309F44ECF8091E5092827A6
:1093B0004ACF80E08093EA091092E90931CFF901A0
:1093C000E050FF4F5081CBCF9FEFD8CF292F2F7781
:1093D0008091E3099091E40990FD20688091E5096E
:1093E0009091E60990FF2FCF8091EA09882309F434
:1093F0002ACF205828CF252F2F778091E3099091ED
:10940000E40991FD20688091E5099091E60991FFBA
:109410001ACFEACF86EC81BB469A15B896E898B980
:1094200093E09BB91EB897E891BBEFE9FFE0319755
:10943000F1F700C0000081BB469A15B823E828B9AF
:1094400023E12BB922E02EB991BBFAE0FA95F1F7AE
:1094500000C081BB469A20EE27B997E09AB92DB992
:1094600015B820E828B99BB91EB897E491BB92E0E3
:109470009A95F1F700C096B199B19CB181BB479A1A
:1094800087EE87B987EF8AB982EE8DB9EAE0EA956F
:10949000F1F700C0089526EC90EE87E0F0E8E7E4ED
:1094A00077EE67EF52EE4FB7F89421BB469A97B923
:1094B0008AB99DB915B8F8B98BB91EB8E1BB32E0CD
:1094C0003A95F1F700C036B1A9B1ACB121BB479ACA
:1094D00077B96AB95DB94FBF45E04A95F1F7000029
:1094E00032FFE1CF8FB7F89496EC91BB469A15B84E
:1094F00091E898B993ED9BB990E29EB997E891BB3A
:1095000095E09A95F1F700008FBF0895CF92DF9212
:10951000EF92FF928091C60B9091C70BA0E0B0E054
:10952000E091E910F091EA106F01E12CF12C8C151B
:109530009D05AE05BF05E4F4A7019601281B390B74
:109540004A0B5B0BA0E0B0E80E94C96EA701960130
:109550000E94CD6E2F3F8FE7380741055105FCF083
:109560002FEF3FE7C901FF90EF90DF90CF90089574
:109570009C01AD012C193D094E095F09AFEFBFE712
:109580000E94BD6E9F012095309540E050E00E9402
:10959000CD6E2F3F8FE73807410551050CF7DA01F3
:1095A000C901811520E892072FEFA207B2073CF00E
:1095B0009C01C901FF90EF90DF90CF90089580E06B
:1095C00090E8AFEFBFEF9C01F4CF2F923F924F9204
:1095D0005F926F927F928F929F92AF92BF92CF9243
:1095E000DF92EF92FF920F931F93CF93DF9300D000
:1095F000CDB7DEB7382E4FB6F894282F2595259590
:109600002595259580E290E002C0959587952A954D
:10961000E2F7932D9F70982B86EC81BB469A492FD9
:10962000440F292F2695392F331F3327331F842FBB
:109630008670382B30649071842F880F8072892B4C
:10964000407C842B2270206491E095B938B98BB9A5
:109650002EB987E881BB25E02A95F1F70000832D1C
:10966000992787FD90959A838983FC01E850F94FEB
:10967000E081F0E080E190E08E1B9F0B66246A940D
:10968000762C082E02C0769467940A94E2F702C002
:10969000660C771C8A95E2F740E050E020E030E865
:1096A0008FEF9FEF66EC262E17E877E0972EAA241F
:1096B000A394A0E4BA2EB0E2CB2E07E4D02E67EE3E
:1096C000E62E77EFF72EA2EE5A2E0AC0820F931FD6
:1096D000369527954F5F5F4FE417F5070CF46BC085
:1096E000BC01672F772766956695062F21BA469AA3
:1096F000B62FBB0FAB2FA670A06860717727626092
:109700007B2F770F7072762BB07C7B2B602F66954A
:109710006270606215B8A8B97BB96EB911BBBC01A3
:109720007695679576956795A62F21BA469A062F66
:10973000000FB62FB695AA1FAA27AA1F0F2EF6E074
:109740008F2EF02D8022A829A06860717727626093
:10975000702F770F7072762B007C702BB27015B85B
:10976000A8B97BB9BEB911BBA2E0AA95F1F700C0B8
:1097700021BA469AB0EEB7B99AB8BDB9A5B8B8B88B
:109780001BB8CEB8D1BA62E06A95F1F700C066B1F5
:1097900069B17CB121BA479AE7B8FAB85DB865FDFE
:1097A00095CF821B930B369527954F5F5F4FE4173C
:1097B000F5070CF095CF26EC21BB469A21E025B9A0
:1097C00027E428B920EF2BB922E42EB927E821BBE2
:1097D000A5E0AA95F1F7000086219721E981FA8199
:1097E000EE0FFF1FEA55F44F91838083892F99274D
:1097F000A981BA81AE57B44F14962C91149730E0DA
:10980000281B390B37FD19C025303105E4F44FBE54
:109810000F900F90DF91CF911F910F91FF90EF90DC
:10982000DF90CF90BF90AF909F908F907F906F9080
:109830005F904F903F902F90089531952195310979
:109840002530310524F314968C9381E090E0A0E05C
:10985000B0E0032C04C0880F991FAA1FBB1F0A94F5
:10986000D2F74091820B5091830B6091840B7091E1
:10987000850B842B952BA62BB72B8093820B909373
:10988000830BA093840BB093850B3092E70BBFCF73
:109890006F928F929F92AF92BF92CF92DF92EF9290
:1098A000FF920F931F93CF93DF93E0913218F091C3
:1098B0003318309719F082E198E109952FB7F894A1
:1098C0008091FB189091FA18891708F009C100914E
:1098D000FC18080F091B2FBF10E00115110509F432
:1098E00076C0C0E0D0E02091FC18EE24E394F12C87
:1098F000E3E09E2EF4E08F2EA2E0AA2EBB24B394C8
:10990000892F622F90E070E00E943B6AE091FD1881
:10991000F091FE18E80FF91FF081F83F08F065C0DC
:10992000F7FF71C080913718843031F0F09334180C
:10993000F0923918E09238188F2F807F803B79F1B0
:1099400098F4803961F1803A51F1803841F1F03F6B
:1099500009F4B1C0F73F09F4C6C01092371810924D
:109960003918109238181DC0803D09F4A1C008F4C0
:109970009CC0803EA1F0803F51F7EF2FE15FEF30B8
:1099800030F7AE2FB0E0A85EB84F8C91813009F46B
:109990009BC0E8F2823009F48BC08330F1F69092DC
:1099A00037183FB7F8949091FA18892F90E00196F4
:1099B0002091FC18622F70E00E943B6A982F8093E0
:1099C000FA183FBF2196C017D10708F499CFDF914D
:1099D000CF911F910F91FF90EF90DF90CF90BF90AC
:1099E000AF909F908F906F900895D0903718B0925D
:1099F000371820E040E06F2F81E090E00E94A6142D
:109A0000D0923718CECF60903718662051F240912F
:109A10003818509139189A01ABEABAEA0E94E86EF8
:109A20006C01D694C794C601880F991F8C0D9D1D9B
:109A30006A01C81AD90AD601AE5EB74E9296FC9357
:109A4000CA010196909339188093381821E0C21604
:109A5000D104B9F022E0C216D10409F0A2CF2091BE
:109A6000361840913518609134180E94A6148091E0
:109A70003718843009F495CFF0923918E0923818ED
:109A800090CF22E062128DCF20E040913518609196
:109A900034180E94A61480913718843009F481CFBD
:109AA000D0923918C09238187CCF803C09F04FCF43
:109AB000A092371876CF80923718F0933418F0922E
:109AC0003918E09238186DCF8093371820E040E0C5
:109AD0006F2F81E090E00E94A6141092371861CF9A
:109AE000082F091BF8CE40913818509139189A0167
:109AF000ABEABAEA0E94E86E969587959C01220F20
:109B0000331F280F391FDA01A21BB30BAE5EB74E0D
:109B10009296FC93CA010196909339188093381855
:109B20002091361840913518609134180E94A6147F
:109B30001092371836CF2F923F924F925F926F92CA
:109B40007F928F929F92AF92BF92CF92DF92EF92CD
:109B5000FF920F931F93CF93DF93CDB7DEB76B9731
:109B60000FB6F894DEBF0FBECDBF762E882309F462
:109B700094C0E091860FF091870F8090880F9090AD
:109B8000890F40917A0F50917B0F8091800F9091B7
:109B9000810F2091B20F3091B30F4090C40B5090C1
:109BA000C50B60906C0F6091760F5092011340923C
:109BB0000013F0930313E093021390920513809225
:109BC0000413509307134093061390930913809343
:109BD000081330930B1320930A1360920C136093B5
:109BE0000D13440C452C441C5508519482011A95C0
:109BF00018870F83EE0FEF2FEE1FFF0BF1958F01EC
:109C00001A951A8B098BA12CB12C75016401CC0C0F
:109C1000DD1CEE1CFF1CCC0CDD1CEE1CFF1CC80C5C
:109C2000D91CEA1CFB1C13E0F694E794D794C79464
:109C30001A95D1F7569547955695479596958795D8
:109C4000969587950D2D11271C870B87052F1127BA
:109C50001A830983092F1127DD24EE24FF246623AC
:109C600009F440C0623008F436C6ECE0F0E08981C7
:109C70009A81BF010E943B6A49815A81481B590B56
:109C80005A834983C801BF010E943B6A081B190B14
:109C9000188A1F861E861D862DC04090C40B5090CA
:109CA000C50B8091001390910113E091860FF09104
:109CB000870F8415950509F4E9C58090880F909069
:109CC000890F40917A0F50917B0F8091800F909176
:109CD000810F2091B20F3091B30F60906C0F6091A3
:109CE000760F63CFBA0177277E876D87DC01BB27AC
:109CF000B88BAF875091710F5D8B7091F2107F8B95
:109D0000832F99279C8B8B8B2091580F2E8B77FC60
:109D100029C1772009F426C177FCCEC431E073163F
:109D200009F4CAC477FCDFC332E0731609F4DBC35D
:109D300077FCEDC233E0731609F4E9C277FCFAC18F
:109D400034E0731609F4F6C177FC1CC045E07416C4
:109D5000C9F06B960FB6F894DEBF0FBECDBFDF9192
:109D6000CF911F910F91FF90EF90DF90CF90BF9018
:109D7000AF909F908F907F906F905F904F903F90AB
:109D80002F9008958091730B882319F38091720BA3
:109D9000282F30E0285131093C832B83020F131FF9
:109DA0002F813885442737FD4095542F2F833887DE
:109DB00049875A8780903A0F90903B0FAA2497FCCE
:109DC000A094BA2C820E931EA41EB51E89819A817E
:109DD0002B813C81820F931F97FDF6C645E06D8570
:109DE0000E94284114012501280E391E411C511CD6
:109DF00057FCA3C62114310431E0430651040CF092
:109E00009AC58090460F9090470FAA2497FCA09483
:109E1000BA2C2F81388549855A85820E931EA41E3F
:109E2000B51E29893A89C901AA2797FDA095BA2F9D
:109E3000880E991EAA1EBB1EC80117FD86C64BE0E0
:109E40006F850E942841880E991EA11CB11CB7FC89
:109E50007FC68114910431E0A306B1040CF060C503
:109E60008B859C856110BBC50091520F1091530FDB
:109E700041E16C2D0E942841A801662757FD60959D
:109E8000762F480F591F611D711D77FDAAC6411518
:109E9000510531E06307710524F04FEF5FEF60E09B
:109EA00070E00D89011104C01F89112309F48FC6C8
:109EB0008B899C89880F991F2B893C89820F931F5E
:109EC000919581959109AA2797FDA095BA2F9201A6
:109ED0008101080F191F2A1F3B1F37FD96C6011568
:109EE0001105E1E02E07310524F00FEF1FEF20E010
:109EF00030E09801880E991EAA1EBB1EB7FCA5C6AD
:109F000081149104F1E0AF06B1042CF088248A9406
:109F1000982CA12CB12C480F591F6A1F7B1F77FD6D
:109F200090C64115510501E06007710524F04FEF1F
:109F30005FEF60E070E01E89112309F4D8C530930B
:109F4000130F2093120F90921F0F80921E0F5093A9
:109F50002B0F40932A0F6110FCCE5093070F4093B4
:109F6000060FF7CE80913C0B882309F4D5CE809163
:109F70003B0B282F30E0285131093B8F2A8F200FCF
:109F8000311F4F815885662757FD6095762F4B838B
:109F90005C836D837E832090300F3090310F4101C0
:109FA000AA2497FCA094BA2C840E951EA61EB71E58
:109FB00089819A816A8D7B8D860F971F97FDB3C526
:109FC00040E06D85288F398F0E94284114012501BA
:109FD000280E391E411C511C288D398D57FCEAC5AD
:109FE0002114310471E0470651040CF0B4C4809090
:109FF0003C0F90903D0FAA2497FCA094BA2C8B8123
:10A000009C81AD81BE81880E991EAA1EBB1EE98966
:10A01000FA89CF01AA2797FDA095BA2F880E991E1D
:10A02000AA1EBB1EC90137FD81C546E06F850E948F
:10A030002841880E991EA11CB11CB7FC7AC5811459
:10A040009104F1E0AF06B1040CF07BC48B859C85D4
:10A050006110A7C42091480F3091490F4CE06C2D3E
:10A06000288F398F0E942841288D398DA9016627B4
:10A0700057FD6095762F480F591F611D711D77FDA3
:10A08000A8C54115510521E06207710524F04FEF85
:10A090005FEF60E070E03D89311103C03F893323F9
:10A0A000C9F12B893C89C901AA2797FDA095BA2F30
:10A0B000280E391E4A1E5B1E57FCBFC521143104F1
:10A0C00031E0430651042CF022242A94322C412CF6
:10A0D000512C880E991EAA1EBB1EB7FCAAC581145E
:10A0E0009104E1E0AE06B1042CF088248A94982C07
:10A0F000A12CB12C480F591F6A1F7B1F77FD95C5F6
:10A1000041155105F1E06F07710524F04FEF5FEF46
:10A1100060E070E02E892111C4C43092E50E2092D7
:10A12000E40E9092F10E8092F00E5093FD0E40934B
:10A13000FC0EF2CD8091680B882309F405CE809146
:10A14000670B282F30E0285131093B8F2A8F200FD1
:10A15000311F4F815885662757FD6095762F4B83B9
:10A160005C836D837E832090380F3090390F4101DE
:10A17000AA2497FCA094BA2C840E951EA61EB71E86
:10A1800089819A816A8D7B8D860F971F97FD16C5F1
:10A1900044E06D85288F398F0E94284114012501E4
:10A1A000280E391E411C511C288D398D57FCC9C4FD
:10A1B0002114310471E0470651040CF0ECC3809087
:10A1C000440F9090450FAA2497FCA094BA2C8B8141
:10A1D0009C81AD81BE81880E991EAA1EBB1EE98995
:10A1E000FA89CF01AA2797FDA095BA2F880E991E4C
:10A1F000AA1EBB1EC90137FDBEC44AE06F850E947E
:10A200002841880E991EA11CB11CB7FCB7C481144B
:10A210009104F1E0AF06B1040CF0B3C38B859C85CB
:10A220006110CEC32091500F3091510F40E16C2D41
:10A23000288F398F0E942841288D398DA9016627E2
:10A2400057FD6095762F480F591F611D711D77FDD1
:10A25000CCC44115510521E06207710524F04FEF90
:10A260005FEF60E070E03D89311103C03F89332327
:10A27000F1F18B899C89880F991F2B893C89820F6A
:10A28000931FAA2797FDA095BA2F280E391E4A1EA4
:10A290005B1E57FCE2C42114310431E04306510433
:10A2A0002CF022242A94322C412C512C880E991EF9
:10A2B000AA1EBB1EB7FCCDC481149104E1E0AE061A
:10A2C000B1042CF088248A94982CA12CB12C480F2E
:10A2D000591F6A1F7B1F77FD94C441155105F1E09A
:10A2E0006F07710524F04FEF5FEF60E070E02E899B
:10A2F000211106C43092ED0E2092EC0E9092F90ED0
:10A300008092F80E5093050F4093040F1DCD80915D
:10A310005D0B882309F412CD80915C0B282F30E06F
:10A32000285131093B8F2A8F200F311F4F815885CB
:10A33000662757FD6095762F4B835C836D837E8304
:10A340002090360F3090370F4101AA2497FCA0943B
:10A35000BA2C840E951EA61EB71E89819A816A8D1D
:10A360007B8D860F971F97FD2CC443E06D85288F4A
:10A37000398F0E94284114012501280E391E411CE5
:10A38000511C288D398D57FCEBC32114310471E029
:10A39000470651040CF0EFC28090420F9090430F9B
:10A3A000AA2497FCA094BA2C8B819C81AD81BE819C
:10A3B000880E991EAA1EBB1EE989FA89CF01AA2719
:10A3C00097FDA095BA2F880E991EAA1EBB1EC90123
:10A3D00037FDCAC349E06F850E942841880E991E47
:10A3E000A11CB11CB7FCC3C381149104F1E0AF06FA
:10A3F000B1040CF0B6C28B859C856110FFC2209120
:10A400004E0F30914F0F4FE06C2D288F398F0E94E7
:10A410002841288D398DA901662757FD6095762F33
:10A42000480F591F611D711D77FDE7C34115510587
:10A4300021E06207710524F04FEF5FEF60E070E00C
:10A440003D89311103C02F892223E9F18B899C8931
:10A45000919581959109880F991FAA2797FDA0953D
:10A46000BA2F280E391E4A1E5B1E57FC02C4211447
:10A470003104E1E04E0651042CF022242A94322CBF
:10A48000412C512C880E991EAA1EBB1EB7FCEDC391
:10A4900081149104F1E0AF06B1042CF088248A9471
:10A4A000982CA12CB12C480F591F6A1F7B1F77FDD8
:10A4B000D8C34115510521E06207710524F04FEF23
:10A4C0005FEF60E070E03E893111FEC23092EB0E2A
:10A4D0002092EA0E9092F70E8092F60E5093030FA0
:10A4E0004093020F2BCC8091520B882309F420CC8F
:10A4F0008091510B282F30E0285131093B8F2A8F52
:10A50000200F311F4F815885662757FD6095762FA4
:10A510004B835C836D837E832090340F3090350FA6
:10A520004101AA2497FCA094BA2C840E951EA61E65
:10A53000B71E89819A816A8D7B8D860F971F97FD43
:10A5400028C342E06D85288F398F0E94284114016D
:10A550002501280E391E411C511C288D398D57FCB0
:10A5600025C32114310471E0470651040CF0CCC11D
:10A570008090400F9090410FAA2497FCA094BA2C91
:10A580008B819C81AD81BE81880E991EAA1EBB1E47
:10A59000E989FA89CF01AA2797FDA095BA2F880EDD
:10A5A000991EAA1EBB1EC90137FDF9C248E06F857E
:10A5B0000E942841880E991EA11CB11CB7FCF2C252
:10A5C00081149104F1E0AF06B1040CF093C18B85C6
:10A5D0009C85611022C220914C0F30914D0F4EE0AE
:10A5E0006C2D288F398F0E942841288D398DA90123
:10A5F000662757FD6095762F480F591F611D711D05
:10A6000077FDEBC24115510521E06207710524F089
:10A610004FEF5FEF60E070E03D89311103C02F899B
:10A620002223D1F18B899C89880F991FAA2797FD36
:10A63000A095BA2F280E391E4A1E5B1E57FC25C353
:10A6400021143104E1E04E0651042CF022242A9416
:10A65000322C412C512C880E991EAA1EBB1EB7FC11
:10A6600010C381149104F1E0AF06B1042CF08824EA
:10A670008A94982CA12CB12C480F591F6A1F7B1F5C
:10A6800077FDFBC24115510521E06207710524F0F9
:10A690004FEF5FEF60E070E03E893111EFC1309223
:10A6A000E90E2092E80E9092F50E8092F40E5093EF
:10A6B000010F4093000F3CCB8091470B882309F496
:10A6C00031CB8091460B282F30E0285131093B8F48
:10A6D0002A8F200F311F4F815885662757FD6095BF
:10A6E000762F4B835C836D837E832090320F309076
:10A6F000330F4101AA2497FCA094BA2C840E951E16
:10A70000A61EB71E89819A816A8D7B8D860F971F41
:10A7100097FD42C241E06D85288F398F0E94284104
:10A7200014012501280E391E411C511C288D398D1C
:10A7300057FC12C22114310471E0470651040CF099
:10A74000E9C080903E0F90903F0FAA2497FCA09400
:10A75000BA2C8B819C81AD81BE81880E991EAA1E68
:10A76000BB1EE989FA89CF01AA2797FDA095BA2FC8
:10A77000880E991EAA1EBB1EC90137FD03C247E001
:10A780006F850E942841880E991EA11CB11CB7FC40
:10A79000FCC181149104F1E0AF06B1040CF0A0C03B
:10A7A0008B859C85611048C120914A0F30914B0FD9
:10A7B0004DE06C2D288F398F0E942841288D398DCE
:10A7C000A901662757FD6095762F480F591F611D17
:10A7D000711D77FD0EC24115510521E0620771051B
:10A7E00024F04FEF5FEF60E070E03D89311103C06E
:10A7F0002F892223D9F18B899C8991958195910983
:10A80000AA2797FDA095BA2F280E391E4A1E5B1E57
:10A8100057FC07C221143104E1E04E0651042CF02C
:10A8200022242A94322C412C512C880E991EAA1EC7
:10A83000BB1EB7FCF2C181149104F1E0AF06B10474
:10A840002CF088248A94982CA12CB12C480F591FE5
:10A850006A1F7B1F77FDDDC14115510521E06207AD
:10A86000710524F04FEF5FEF60E070E03E89311139
:10A87000F2C03092E70E2092E60E9092F30E809294
:10A88000F20E5093FF0E4093FE0E4CCA80910213BD
:10A89000909103138090880F9090890FE817F90723
:10A8A00009F00FCA809104139091051340917A0F1B
:10A8B00050917B0F8816990609F427C28091800F6A
:10A8C0009091810F2091B20F3091B30F60906C0F77
:10A8D0006091760F6AC9188A1F861E861D860ACA6D
:10A8E00088248A94982CA12CB12C8B859C8561108E
:10A8F000A3C05ACF88248A94982CA12CB12C8B8584
:10A900009C8561108AC067CE22242A94322C412C67
:10A91000512C2ECE22242A94322C412C512C11CF92
:10A9200088248A94982CA12CB12C8B859C85662038
:10A9300009F49ACA54C022242A94322C412C512C56
:10A9400060CA88248A94982CA12CB12C8B859C8574
:10A95000611027C07FCB22242A94322C412C512C09
:10A9600046CB88248A94982CA12CB12C8B859C856D
:10A97000611044C044CD22242A94322C412C512C05
:10A980000BCD88248A94982CA12CB12C8B859C8586
:10A99000611016C047CC22242A94322C412C512C11
:10A9A0000ECC41E0641609F47EC18B859C852A8D0E
:10A9B0003B8D820F931F97FF4DCB80E090E04ACBF9
:10A9C00041E0641609F465C18B859C852A8D3B8D19
:10A9D000820F931F97FF26CC80E090E023CC41E0CC
:10A9E000641609F488C18B859C852B813C81820F7C
:10A9F000931F97FF39CA80E090E036CA31E06316B2
:10AA000009F465C18B859C852A8D3B8D820F931F30
:10AA100097FFF5CC80E090E0F2CC31E0631609F4CA
:10AA20004CC18B859C852A8D3B8D820F931F97FF90
:10AA3000D2CD80E090E0CFCD31E0631609F451C172
:10AA40008B859C852A8D3B8D820F931F97FFACCE03
:10AA500080E090E0A9CE30920B0F20920A0F9092E6
:10AA6000170F8092160F5093230F4093220F6110FF
:10AA700059C95093FF0E4093FE0E54C930920D0FEA
:10AA800020920C0F9092190F8092180F5093250F5F
:10AA90004093240F61104CC95093010F4093000F55
:10AAA00047C93092090F2092080F9092150F80929B
:10AAB000140F5093210F4093200F61102DC9509314
:10AAC000FD0E4093FC0E28C930920F0F20920E0FFE
:10AAD00090921B0F80921A0F5093270F4093260FCE
:10AAE00061102CC95093030F4093020F27C9309374
:10AAF000EF0E2093EE0E9092FB0E8092FA0E2DCA6E
:10AB00003092110F2092100F90921D0F80921C0F07
:10AB10005093290F4093280F611016C95093050FC9
:10AB20004093040F11C980E090E04ACA80E090E0B1
:10AB30007CCA812C912C540182CA212C312C2101F8
:10AB400059C9212C312C210133CB80E090E077C909
:10AB5000812C912C54017DC9212C312C2101EACD6D
:10AB6000212C312C210111CC80E090E033CC812CC0
:10AB7000912C540139CC80E090E03FCB812C912C7A
:10AB8000540145CB80E090E0FACD812C912C54010A
:10AB900000CE80E090E0D5CC80E090E0BBCD80E0BE
:10ABA00090E004CD812C912C54010ACD212C312C24
:10ABB0002101D7CC212C312C210112CA80E090E058
:10ABC000E7CA80E090E0D1CB80E090E007C9910136
:10ABD000B2C940E050E0BA0154CA40E050E0BA01C6
:10ABE00011CD40E050E0BA0152C940E050E0BA0156
:10ABF00030CB40E050E0BA01EECD40E050E0BA0189
:10AC000015CC40E050E0BA0168CB00E010E09801BC
:10AC100066C940E050E0BA011FCE812C912C54014E
:10AC20000ACE212C312C2101F5CD40E050E0BA01B3
:10AC300067CA812C912C540152CA212C312C21013C
:10AC40003DCA40E050E0BA016CC9812C912C5401FE
:10AC500057C9812C912C54012FCB212C312C21014F
:10AC60001ACB40E050E0BA0124CC812C912C540145
:10AC70000FCC212C312C2101FACB40E050E0BA015D
:10AC800001CD812C912C5401ECCC212C312C2101B3
:10AC9000D7CC8A8D9B8D97FD55C09C013595279506
:10ACA0003B8F2A8F91CE8A8D9B8D97FD4DC09C0145
:10ACB000359527953B8F2A8F78CE8A8D9B8D97FD72
:10ACC00045C09C01359527953B8F2A8FAACE8A8D4A
:10ACD0009B8D97FD3FC09C01359527953B8F2A8F13
:10ACE00091CE8A8D9B8D97FD33C09C01359527951C
:10ACF0003B8F2A8FA5CE8B819C8197FD2DC08C0127
:10AD0000159507951C830B836ECE80910613909149
:10AD100007134817590709F0D1CD8091800F909102
:10AD2000810F209108133091091382179307B1F016
:10AD30002091B20F3091B30F60906C0F6091760F3D
:10AD40000C94D54D0196A9CF0196B1CF0196B9CFFC
:10AD50000196CBCF0196BFCF0196D1CF2091B20FF4
:10AD60003091B30F60910A1370910B1360906C0FC8
:10AD70002617370721F06091760F0C94D54D60911E
:10AD80000C136612F8CF6091760F70910D13671354
:10AD90000C94D54D0C94A94E7F928F929F92AF92B6
:10ADA000BF92CF92DF92EF92FF920F931F93CF93B8
:10ADB000DF9300D0CDB7DEB71A821982C12CD12C17
:10ADC00008C08FEFC81AD80A84E6C816D10409F45F
:10ADD00068C0C6010E94873F882399F3BE016F5F58
:10ADE0007F4FC6010E944C3FE980FA807FB6F894FD
:10ADF00081E0E81AF108F594E794F594E7948FEF71
:10AE0000E81AF80A0E944B4A0E94D7470E9412484B
:10AE10000E944D480E9488481E141F04BCF500E0A3
:10AE200010E0F801EE0FFF1FEE0FFF1FEE5EF94E70
:10AE30008080A1809280B380882D8F770E946047A8
:10AE40008A2D8F770E946047892D8F770E946047F7
:10AE50008B2D8F770E946047992D929596959470CF
:10AE60003A2D3295369536953270932B2B2D2295AF
:10AE70002870922B882D881F8827881F892B0E9475
:10AE800060470F5F1F4F0E151F055CF20E94C348FD
:10AE90007FBE8FEFC81AD80A84E6C816D10409F01D
:10AEA00098CF0F900F90DF91CF911F910F91FF904E
:10AEB000EF90DF90CF90BF90AF909F908F907F905A
:10AEC0000895842F2091EE1027FD09C06F7070E067
:10AED000332727FD30956217730709F0089540E086
:10AEE00050E060E00C94FF29842FE091EE10E7FD24
:10AEF00009C06F7070E0FF27E7FDF0956E177F07C0
:10AF000009F00895422F50E0542F4427550F415027
:10AF10005E4F61E0211101C060E00C94FF29603EAA
:10AF200071058105910508F00895DC01CB019F5F53
:10AF3000AF4FBF4F6627782F892F9A2F0C9400F8B8
:10AF400080910F16909110168F509441813092404D
:10AF500070F44FE054E16CED70E080E090E0DFDFF2
:10AF60004FE055E16DED70E080E090E0D8CF0895BE
:10AF7000CF93C091AF0CCF3F79F0CF77C85E40E060
:10AF800050E060E08C2F0E94FF2940E06C2F809100
:10AF9000EF10CF910C949314CF9108952F923F927C
:10AFA0004F925F926F927F928F929F92AF92BF92D9
:10AFB000CF92DF92EF92FF920F931F93CF93DF9385
:10AFC0008091B50C882339F18091B00C9091B10C2F
:10AFD00001969093B10C8093B00C2091B20C3091FB
:10AFE000B30C82179307B8F01092B10C1092B00C0A
:10AFF000EDE2FCE004C08CE0ED3AF80761F08191ED
:10B000008F3FC9F3B5DF8091B50C823069F1833091
:10B01000A1F1813091F1DF91CF911F910F91FF90BC
:10B02000EF90DF90CF90BF90AF909F908F907F90E8
:10B030006F905F904F903F902F90089561507109ED
:10B040008109910960687F6F8F6F9F6F6F5F7F4F7E
:10B050008F4F9F4FFB017093AE0C6093AD0CE35D7F
:10B06000F34F80818F3F21F50E94B16E6F77772774
:10B070008827907897FFEECFE1CF2091AD0C3091EB
:10B08000AE0C07C09C01FC01E35DF34F40814F3FD4
:10B0900059F4C90101968F77907897FFF3CF019704
:10B0A00080689F6F0196EECF8093AD0C9093AE0CAD
:10B0B0007080EFE77E22F8E17F0EE72DE695E695BA
:10B0C000E695F0E0EC5DF54FA72DA770B0E0A95D27
:10B0D000B84F80819C91892B8083A72CB12CF501DE
:10B0E000EE0FFF1FEC5CF54F80E090E891838083CA
:10B0F000C0905E09D0905F09E0906009F09061090E
:10B1000080917E0B8111BAC1E0917D0BCE2FC17071
:10B11000E0FF5EC280913C0B8111C5C24091340BAF
:10B120005091350B6091360B7091370B4F3F8FEF7D
:10B1300058076807780709F44EC290E02E2F227056
:10B14000E1FF14C08091470B20903F0B3090400BE3
:10B150004090410B5090420B8111B9C22416350624
:10B160004606570618F4B201A10191E08E2F8470B3
:10B17000E2FF14C03091520B20904A0B30904B0BE1
:10B1800040904C0B50904D0B311175C22416350672
:10B190004606570618F4B201A10192E03E2F38701E
:10B1A000E3FF14C0F0915D0B2090550B3090560BCF
:10B1B0004090570B5090580BF11169C22416350678
:10B1C0004606570618F4B201A10193E0AE2FA07114
:10B1D000E4FF14C0F091680B2090600B3090610B7D
:10B1E0004090620B5090630BF1117DC2241635061E
:10B1F0004606570618F4B201A10194E0BE2FB072C2
:10B20000E5FF17C0E091730BEE2309F424C24091CF
:10B210006B0B50916C0B60916D0B70916E0B4C151C
:10B220005D056E057F0528F44091720B741609F4D4
:10B2300010C29F3F09F0B1C0CC2309F4D7C150918F
:10B240003A0BE52FE695E695E695F0E0EC5DF54FD7
:10B2500040814111C2C14091340B5091350B609136
:10B26000360B7091370B4F3FEFEF5E076E077E078F
:10B2700009F090E02223E1F01091450BE12FE695D3
:10B28000E695E695F0E0EC5DF54FD081D11147C22F
:10B2900020903F0B3090400B4090410B5090420B60
:10B2A000241635064606570618F4B201A10191E0AE
:10B2B0008823E1F01091500BE12FE695E695E69595
:10B2C000F0E0EC5DF54FD081D11133C220904A0BF4
:10B2D00030904B0B40904C0B50904D0B2416350684
:10B2E0004606570618F4B201A10192E03323E1F0BB
:10B2F00010915B0BE12FE695E695E695F0E0EC5DAD
:10B30000F54FD081D1111FC22090550B3090560BB4
:10B310004090570B5090580B24163506460657069A
:10B3200018F4B201A10193E0AA23E1F01091660B99
:10B33000E12FE695E695E695F0E0EC5DF54FD081DE
:10B34000D1110BC22090600B3090610B4090620BCA
:10B350005090630B241635064606570618F4B201C2
:10B36000A10194E0BB23B1F01091710BE12FE695A0
:10B37000E695E695F0E0EC5DF54FD081DD2309F42C
:10B38000BEC1E12FE770F0E0E95DF84FE081ED2309
:10B3900009F4B5C19F3F09F49BC0512C36E7832EB9
:10B3A0003BE0932E4BE0442E66246394212C50E81E
:10B3B000352E06E010E0F40181914F018F3F09F432
:10B3C0004EC0C92FDD27C7FDD0954C9E90014D9EE4
:10B3D000300D11242C5D354FF901E85EFE4F60827F
:10B3E000F901E75EFE4F6082F901E65EFE4F608282
:10B3F000F901EC5EFE4F31822082F901EA5EFE4FD8
:10B400007082F901E95EFE4FA501480F511D40838E
:10B41000F901E05FFE4FC082D182E282F382452DC6
:10B4200060E070E8892F0E94C32840917D0B04C022
:10B43000C92FDD27C7FDD095CE010196B8010E9426
:10B440003B6A9C01982FF901E95DF84F80818423C4
:10B4500079F3FCE78F16FBE09F0609F0ACCF60E0C4
:10B4600070E8872D0E94C527E091AD0CF091AE0CDD
:10B47000E35DF34F80818093AF0CCDCD80917C0B49
:10B48000512C882319F1823009F422C2813009F449
:10B49000FCC180E090E0A816B906A1F0E82FE6957F
:10B4A000E695E695F0E0EC5DF54F2081222351F022
:10B4B000FC01E770FF27E95DF84F3081322311F07E
:10B4C0005524539401968038910529F790E066CF72
:10B4D000E0917C0BCC2309F498C1E13009F4BCC1A4
:10B4E00008F0AFC14091340B5091350B6091360B91
:10B4F0007091370B4F3FFFEF5F076F077F0709F032
:10B5000090E0222309F409C21A012B0140913F0B5C
:10B510005091400B6091410B7091420B42155305C5
:10B520006405750508F4ADC1B201A101F72D8823AA
:10B5300009F450C120904A0B30904B0B40904C0BBB
:10B5400050904D0B241635064606570618F4B201E6
:10B55000A10192E0332309F41FC10091550B109112
:10B56000560B2091570B3091580B041715072607DF
:10B57000370708F484C18A019B01B901A801AA23F5
:10B5800009F413C10091600B1091610B2091620BC3
:10B590003091630B041715072607370708F473C1AA
:10B5A0008A019B01BB2381F0B901A80100916B0BBB
:10B5B00010916C0B20916D0B30916E0B04171507D9
:10B5C0002607370708F445C09F3F09F448CFE5CE6A
:10B5D0004FEF5FEFBA019FEFB1CD5770E52FF0E06D
:10B5E000E95DF84F5081542309F435CE4FEF5FEFFA
:10B5F000BA0140CEF72D2091460BF21708F439C15D
:10B600002F2FF22F882309F4E2C04FEF5FEFBA012A
:10B610008091510BF81708F430C18F2FF82F332386
:10B6200009F4BAC080915C0BF81710F4F82F93E07E
:10B63000AA2309F4BAC08091670BF81710F4F82F09
:10B6400094E0BB2309F4C0CF8091720BF81708F087
:10B65000BBCF95E0A2CE20906B0B30906C0B40904E
:10B660006D0B50906E0B241635064606570608F0F3
:10B67000E0CD95E092CE2C143D044E045F0408F01A
:10B680008DCD3091510B731289CD92E086CE2C1462
:10B690003D044E045F0408F099CDF0915C0B7F12DD
:10B6A00095CD93E07ACE8091340B9091350BA0919B
:10B6B000360BB091370B8C159D05AE05BF0508F014
:10B6C00087CF80913B0B781283CF90E066CE2C140D
:10B6D0003D044E045F0408F049CD8091460B78127A
:10B6E00045CD91E05ACE2C143D044E045F0408F081
:10B6F00085CDF091670B7F1281CD94E04ECE2090E6
:10B700006B0B30906C0B40906D0B50906E0B2416B1
:10B7100035064606570608F03DCE95E03ECEE12FB1
:10B72000E770F0E0E95DF84FE081ED2309F0C0CD6E
:10B73000AFCDE12FE770F0E0E95DF84FE081ED2358
:10B7400009F0D4CDC3CDE12FE770F0E0E95DF84F0B
:10B75000E081ED2309F0E8CDD7CDE12FE770F0E0EF
:10B76000E95DF84FE081ED2309F0FCCDEBCDF72D3D
:10B770004FEF5FEFBA01882369F1E13009F448CF58
:10B7800008F4D8CEE23031F58091510B8F1710F4C8
:10B79000F82F92E0311127C0AA2339F0E13009F4E3
:10B7A0004ACF08F4EFCEE23031F1BB2309F40CCFDD
:10B7B000E13009F449CF08F4F9CEE23009F004CFC2
:10B7C0008091720B8F1708F0FFCE95E0E6CD4FEF1A
:10B7D0005FEFBA01332301F3E13009F423CF08F41A
:10B7E000BCCEE230C9F680915C0B8F1710F4F82FB5
:10B7F00093E0AA23D1F28091670B8F1710F4F82FF2
:10B8000094E0BB2309F4E0CEDBCF222309F4AFCFD1
:10B81000E13009F4EFCE28F422242A94322C2101BD
:10B8200075CEE23009F0A3CF272DF091460BF21729
:10B8300008F471C0F22F882351F24FEF5FEFBA0185
:10B84000A3CFE23011F7F0913B0BF715A0F0F72DE5
:10B85000222349F02F2FE9CFF0913B0B7F1638F0D0
:10B86000F72D2111C8CE4FEF5FEFBA0184CF90E0E2
:10B87000F8CF91E0C6CE90E0EBCF92E0CFCE93E050
:10B880007CCE91E053CE94E08DCE80E090E0A8167F
:10B89000B906C1F0E82FE695E695E695F0E0EC5D97
:10B8A000F54F2081222371F0FC01E770FF27E95D4D
:10B8B000F84F3081322331F08A159B050CF4CFCD3F
:10B8C0005524539401968038910509F790E066CD90
:10B8D00080E090E0A816B906C1F0E82FE695E6955D
:10B8E000E695F0E0EC5DF54F2081222371F0FC013C
:10B8F000E770FF27E95DF84F3081322331F0A81659
:10B90000B9060CF4ACCD55245394019680389105BA
:10B9100009F790E043CD91E08ECFF72D2CCFCF9358
:10B92000DF934FB7F89436EC31BB469A80EE87B977
:10B9300097E09AB98DB981E085B980E488B91BB8E0
:10B9400080E28EB987E481BB52E05A95F1F700C0DE
:10B9500026B199B18CB131BB479AC22FC695C3703D
:10B9600050E8259F90011124C22B292F2071C22B52
:10B97000292F269526952870C22B96959076C92B4F
:10B9800090E0880F991F84709927C82B87EE87B99C
:10B9900087EF8AB982EE8DB94FBF8091710FD09138
:10B9A0000E14882311F0C5FF0DC08D2F8C2785FD47
:10B9B00025C08091F110823099F0C0930E14DF9170
:10B9C000CF910895D5FFF1CF0E94F03B86E0E6E7E6
:10B9D000FBE0A6EBBFE001900D928A95E1F7E9CF7D
:10B9E000C0FFEBCFD0FDE9CF80915F0F8F5F8093D9
:10B9F0005F0FC0930E14DF91CF9108958091B50C25
:10BA00008823A1F0C5FF1FC08091B40C882399F052
:10BA1000EDE2FCE09FEF05C031965CE0ED3AF50702
:10BA200051F0808187FFF8CF9083F6CFC5FF07C024
:10BA30000E948632BECF80E08093B40CBACF81E002
:10BA400080937F0BB6CF8091B40C823049F0EDE249
:10BA5000FCE08081806881938CE0ED3AF807C9F7BB
:10BA600082E0EACFCF93DF93D82FC62F8091B50C19
:10BA70008D17C1F07DDA2FEF3FEF3093AE0C20939E
:10BA8000AD0C8FEF8093AF0C40E850E06FEF70E0AB
:10BA90008DE29CE00E944D6E0E94353B8091F1103A
:10BAA00081112EC08091B40C8C17A1F0EDE2FCE066
:10BAB000C11117C02FEF05C031968CE0ED3AF807A1
:10BAC00049F0908197FFF8CF208331968CE0ED3AD2
:10BAD000F807B9F7D093B50CC093B40CDF91CF91B0
:10BAE00008959081906891938CE0ED3AF80791F376
:10BAF0009081906891938CE0ED3AF80791F7EACF46
:10BB00002FEF3FE73093B10C2093B00CCBCFCF9207
:10BB1000DF92FF920F931F93CF93DF9300D0CDB7A7
:10BB2000DEB78C01FFB67A8369830E94493F5A8150
:10BB300069818823E1F0EFE0F4E120E032E0DF0109
:10BB4000C9011D920197E9F7C62ED52E27E136E1EE
:10BB5000462FB901CF010E94336EC601815F9B4E13
:10BB60009093101680930F16C8010E9400368F2DF7
:10BB70000F900F90DF91CF911F910F91FF90DF9069
:10BB8000CF900C940E3F2F923F924F925F926F9204
:10BB90007F928F929F92AF92BF92CF92DF92EF925D
:10BBA000FF920F931F93CF93DF93CDB7DEB7C958A2
:10BBB000D1090FB6F894DEBF0FBECDBF839709F051
:10BBC000F7C280911216813009F0F2C280911316EB
:10BBD000823009F0EDC220911416AE962FAFAE97C9
:10BBE000243608F0E5C2DE01A35ABF4F80E090E0A2
:10BBF0009C012E5E394EF9014481F0E14F9FA00176
:10BC00001124F90123812F70242B2D930296803269
:10BC1000910571F7A3962FADA397922F92959695C4
:10BC200096959370A4964FADA497842F8F70880F2C
:10BC3000880F892B982E990C990C812CB401609552
:10BC40007095E0967FAF6EAFE097A2968FADA2970A
:10BC5000A82EA694AA0CAA0CA1963FADA197932F4B
:10BC6000969596959695FF24F394F822F294FF0CFE
:10BC7000B0EEFB22F92AFF0CFF0C582F551F552759
:10BC8000551F2F73220F922F952B80E0BC0161501E
:10BC90007048E2967FAF6EAFE2976E968FAD6E976B
:10BCA000782F770FCF57DF4F7883C158D040AB96AE
:10BCB0002FADAB97922F9E7FCE57DF4F9883C25800
:10BCC000D04042954F70A5969FADA59717E0D12E15
:10BCD000D922D29400EFD022D42A492F46954695F6
:10BCE0004695A6969FADA697092F01700295000F65
:10BCF000007E042B000F000F692F660F660F562F72
:10BD0000587740E0BA017058E4967FAF6EAFE49781
:10BD1000492F429546954770A7969FADA797A92FA3
:10BD2000A170AA0FAA0FAA0FA42BB0E0A15DB84F73
:10BD30007C91EC967FAFEC97B92EB694B29440EF1D
:10BD4000B422492F429546954770A8969FADA89773
:10BD5000A92FA170AA0FAA0FAA0FA42BB0E0A15D72
:10BD6000B84F4C91ED964FAFED97A92FA695AF70B8
:10BD7000B0E0A15DB84F6C91EE966FAFEE97492F92
:10BD8000429546954770A9969FADA997A92FA17096
:10BD9000AA0FAA0FAA0FA42BB0E0A15DB84F7C9107
:10BDA000EF967FAFEF97C92EC694C29450EFC5228D
:10BDB000929596959770AA964FADAA97A42FA170C9
:10BDC000AA0FAA0FAA0FA92BB0E0A15DB84F9C91B2
:10BDD000C158DF4F9883CF57D040A42FA695AF709E
:10BDE000B0E0A15DB84F6C91C058DF4F6883C05878
:10BDF000D040881F8827881F6F965FAD6F97652F8B
:10BE00006770660F682B962F990F990F990F80E036
:10BE1000BC017058E6967FAF6EAFE697952F991FDD
:10BE20009927991FA0968FADA097182F1F73110FF8
:10BE3000192B110F952F96959C7382958695869553
:10BE400083703770330F330F382B80E1389FB00188
:10BE50001124E8967FAF6EAFE897429546954770FC
:10BE60002170220F220F220F242B40E050E029F0F6
:10BE7000522F550F550F40E05054AD964FACAD9733
:10BE8000742D717041FA662760F9AC968FADAC974E
:10BE9000282F2170E9962FAFE99743FA332730F91D
:10BEA000EA963FAFEA9744FA332730F981FB22271D
:10BEB00020F942FA222420F845FA332430F846FAD1
:10BEC000442440F884FB552450F886FBEE27E0F923
:10BED000F0E0EE0FFF1F87FBEE24E0F8EE0CEE0C17
:10BEE000EE2A85FBEE27E0F9EE2A83FB662460F854
:10BEF00082FF02C082E001C080E0680EAD967FAC98
:10BF0000AD9777FA772470F88FB7EB968FAFEB97F2
:10BF1000CA57DF4F2883C658D040CB57DF4F3883EE
:10BF2000C558D040C957DF4F4883C758D040C8577D
:10BF3000DF4F5883C858D040CC57DF4F6883C45870
:10BF4000D040CD57DF4F7883C358D040C757DF4F1D
:10BF50009883C958D0400E940B3FCA57DF4F2881B1
:10BF6000C658D040CB57DF4F3881C558D040C9574D
:10BF7000DF4F4881C758D040C857DF4F5881C85855
:10BF8000D040CC57DF4F6881C458D040CD57DF4FE9
:10BF90007881C358D040C757DF4F9881C958D040E7
:10BFA000882309F4E7C08CE5E0E6FFE0DE011196A6
:10BFB00001900D928A95E1F77093600F6093610F85
:10BFC000E9966FADE9976093620FEA967FADEA97C5
:10BFD0007093630F3093640F2093650F2092660F68
:10BFE0003092670F4092680F5092690F10926A0F5B
:10BFF000E0926B0F60926C0F10926D0F81E0809356
:10C000006E0F10926F0F7092710F1092720F23E0EB
:10C010002093730F8093740F22E02093750F809309
:10C02000760F8093790F10927A0FA0927B0FE09693
:10C030002EAD3FADE09730937D0F20937C0F109293
:10C040007E0FCF57DF4F3881C158D04030937F0FDC
:10C050001092800FF092810F9092830F8092820F46
:10C060001092840FCE57DF4F6881C258D040609342
:10C07000850FE2962EAD3FADE2973093870F209368
:10C08000860F1092880FD092890F10928A0F00931A
:10C090008B0FE4966EAD7FADE49770938D0F609338
:10C0A0008C0F10928E0FEC967FADEC9770938F0FE4
:10C0B0001092900FB092910F1092920FED962FADBB
:10C0C000ED972093930F1092940FEE963FADEE975D
:10C0D0003093950F1092960FEF966FADEF97609398
:10C0E000970F1092980FC092990F10929A0FC15803
:10C0F000DF4F7881CF57D04070939B0F10929C0FE9
:10C10000C058DF4F2881C058D04020939D0FE6963D
:10C110006EAD7FADE69770939F0F60939E0F109268
:10C12000A00F1093A10F1092A20F9093A30FE89667
:10C130002EAD3FADE8973093A50F2093A40F5093F9
:10C14000A70F4093A60F1092A90F1092A80F10925C
:10C15000AB0F1092AA0FAE968FADAE9790E00E94F3
:10C1600011368CE5FE013196A0E6BFE001900D92FC
:10C170008A95E1F7EB968FADEB97C757DF4F0FB678
:10C18000F894DEBF0FBECDBFDF91CF911F910F910D
:10C19000FF90EF90DF90CF90BF90AF909F908F90E7
:10C1A0007F906F905F904F903F902F900C94093F3D
:10C1B000C757DF4F0FB6F894DEBF0FBECDBFDF917C
:10C1C000CF911F910F91FF90EF90DF90CF90BF9094
:10C1D000AF909F908F907F906F905F904F903F9027
:10C1E0002F9008952F923F924F925F926F927F927D
:10C1F0008F929F92AF92BF92CF92DF92EF92FF9277
:10C200000F931F93CF93DF93803F09F440C0873F84
:10C21000B1F02091800B3091810B211592E039070C
:10C220000CF456C041E050E020E030E0F901EE5E51
:10C23000F94E80835093810B4093800B36C08091E0
:10C240001216813009F448C0811109C0809113167B
:10C25000813629F480911416863109F448C0109271
:10C26000810B1092800BDF91CF911F910F91FF9066
:10C27000EF90DF90CF90BF90AF909F908F907F9086
:10C280006F905F904F903F902F900C94E0441092ED
:10C29000810B1092800B80E092E0E2E1F6E1DF0199
:10C2A0009C011D9221503040E1F7DF91CF911F9109
:10C2B0000F91FF90EF90DF90CF90BF90AF909F9045
:10C2C0008F907F906F905F904F903F902F90089548
:10C2D000A9014F5F5F4FAACF80911316823009F0FA
:10C2E000BECF8091800B9091810B4DDCB8CF8091B7
:10C2F0001516813009F0B3CF8091800B9091810B9E
:10C30000049765E070E00E943B6A1B0177FD72C0F4
:10C31000E6E1AE2EE6E1BE2EF7E1CF2EF6E1DF2E0E
:10C32000A8E1EA2EA6E1FA2E09E116E12B01440C60
:10C33000551C440C551C460E571E39E0430E511C2B
:10C34000C4E0D0E084E0682E712C72E1872E76E1A3
:10C35000972E8C0E9D1E44E050E0B401C3018E5E0A
:10C36000994E0E943C6ED40114962C91B0E82B9FFC
:10C37000C0011124F5019081982B9083922F927027
:10C380009295990F990F907CD6018C91982B9C9344
:10C39000922F94709295990F907EF7018081982B3F
:10C3A0009083822F88708295807FD8019C91892B01
:10C3B0008C93B4E06B0E711C2596E4E0AE0EB11CBC
:10C3C000F4E0CF0ED11C24E0E20EF11C0C5F1F4FF5
:10C3D000C415D50509F0B9CFC1010296880F991F80
:10C3E000880F991FBC01655071098091161690E065
:10C3F0008EDB35CF84E090E0F5CFEF92FF920F9384
:10C40000CF93DF931F92CDB7DEB77B016091800B96
:10C410007091810B6115710529F0E61AF70A81E028
:10C42000E81AF108E114F10439F40F90DF91CF918B
:10C430000F91FF90EF900895842F2983D3DE2981F7
:10C44000E2E0EE16F10488F3822FCCDEF2E0EF1684
:10C45000F10459F3802F0F90DF91CF910F91FF904E
:10C46000EF90C0CE1F920F920FB60F9211240F9033
:10C470000FBE0F901F9018951F920F920FB60F923C
:10C4800011240F900FBE0F901F9018951F920F92BE
:10C490000FB60F9211240BB60F921F932F933F9359
:10C4A0004F935F936F937F938F939F93AF93BF93BC
:10C4B000CF93DF93EF93FF9334999BC0CFB7F8945A
:10C4C00056EC51BB469A70EE77B967E06AB97DB910
:10C4D00015B8D0E8D8B96BB91EB8B7E4B1BB82E0E3
:10C4E0008A95F1F700C026B199B18CB151BB479A3A
:10C4F000422F46954370E0E82E9F90011124422B75
:10C50000292F2071422B292F269526952870422B02
:10C5100096959076492B90E0880F991F8470992703
:10C52000482BA7EEA7B9F7EFFAB9E2EEEDB985E02F
:10C530008A95F1F7000047FF5BC040FF59C051BB2F
:10C54000469A77B96AB97DB915B8D8B96BB980E29E
:10C550008EB9B1BB82E08A95F1F700C026B199B1DE
:10C560008CB151BB479AD22FD695D37050E8259FF6
:10C5700090011124D22B292F2071D22B292F2695FF
:10C5800026952870D22B96959076D92B90E0880F1F
:10C59000991F84709927D82BA7B9FAB9EDB985E00E
:10C5A0008A95F1F7000044FD3AC01FB7F894209136
:10C5B000FB1830E0C90101966091FC1870E05BD770
:10C5C0004091FA1850E08417950789F0E091FD1822
:10C5D000F091FE18E20FF31FD0838091FB1890E0DA
:10C5E00001966091FC1870E046D78093FB181FBF3E
:10C5F000CFBFFF91EF91DF91CF91BF91AF919F910D
:10C600008F917F916F915F914F913F912F911F91EA
:10C610000F900BBE0F900FBE0F901F9018950E94A9
:10C620000A4AE6CF1F920F920FB60F9211240BB653
:10C630000F922F933F934F935F936F937F938F93BB
:10C640009F93AF93BF93CF93DF93EF93FF93CEE688
:10C65000D0E088818D7F888385B3876085BB78949F
:10C660000E944602F894888182608883FF91EF914E
:10C67000DF91CF91BF91AF919F918F917F916F91FA
:10C680005F914F913F912F910F900BBE0F900FBE76
:10C690000F901F901895CF93DF93CDB7DEB76497B7
:10C6A0000FB6F894DEBF0FBECDBF20E82093610027
:10C6B00010926100F89414B817B81AB81DB810BADF
:10C6C00015B880EE88B91BB81EB893EE91BB3FEF4A
:10C6D00034B987B947E04AB98DB990BB9CE797BD9B
:10C6E00094B5926094BD95B5936095BD90916E00A0
:10C6F000926090936E00EC9A96EC91BB469A87B943
:10C700004AB98DB915B828B91BB81EB887E481BBE2
:10C7100042E04A95F1F700C086B189B18CB191BB76
:10C72000479A87EE87B987EF8AB982EE8DB906EB13
:10C730001CE08AEA92E0D801FC011D923197E9F7EA
:10C74000E3E6F9E0DF011D922A95E9F781E4E3EEE3
:10C75000F9E0DF011D928A95E9F780E28093F20902
:10C7600085E4E8EEFBE0DF011D928A95E9F786E6B5
:10C77000E2E8FBE0DF011D928A95E9F73093E70BD1
:10C780000E94B2408CE591E0E4E2FAE0DF019C0116
:10C790001D9221503040E1F78FE380937D0B46E0FE
:10C7A00050E06FEF70E086E79BE00E944D6E1092C4
:10C7B000760B0E940A4A89E8EDE2FCE0DF011D9257
:10C7C0008A95E9F78FEF2FEF8193BCE0ED3AFB07F5
:10C7D000D1F78FEF9FEF9093AE0C8093AD0C209329
:10C7E000AF0C8DE0ECEBFFE0DF011D928A95E9F7DD
:10C7F0002093BD0F2093BF0F8FEF9FEFDC0180933D
:10C80000C00F9093C10FA093C20FB093C30F81E0EC
:10C810008093BE0F2093C80F1092371810923918CA
:10C820001092381880EC8093FC188AE398E190937A
:10C83000FE188093FD181092FB181092FA181092AF
:10C840001B1810921A1810921F1810921E1810928E
:10C850002318109222181092251810922418109262
:10C8600027181092261810922B1810922A1810923E
:10C870002F1810922E181092311810923018109212
:10C880003318109232188EEA97E49093131880931D
:10C89000121884E797E5909317188093161881E68D
:10C8A00097E5909319188093181888E495E390936E
:10C8B00015188093141888E195E3909321188093BC
:10C8C000201880E494E290931D1880931C188DEF3B
:10C8D00091E690932D1880932C188EEE99E3909307
:10C8E0002918809328181092810B1092800B8AE2ED
:10C8F000E2EBFDE0DF01282F1D922A95E9F7D80130
:10C90000E82F1D92EA95E9F7ECEDFDE0DF01282F15
:10C910001D922A95E9F7E0EEFCE0DF01282F1D9239
:10C920002A95E9F7E6E0FEE0DF01282F1D922A951F
:10C93000E9F7EAE0FDE0DF01282F1D922A95E9F7EB
:10C94000E0E3FEE0DF01282F1D922A95E9F7E4E3FA
:10C95000FDE0DF01282F1D922A95E9F7EAE5FEE0C8
:10C96000DF01282F1D922A95E9F7EEE5FDE0DF01B2
:10C97000282F1D922A95E9F7E4E8FEE0DF01282F31
:10C980001D922A95E9F7E8E8FDE0DF011D928A95FE
:10C99000E9F78EEA9EE00E941C4289EC9EE00E942C
:10C9A0001C4261E089EC9EE00E94F74164E089EC62
:10C9B0009EE00E94AE3E8BED90E00E94873F811189
:10C9C00006C00E94EB3F8BED90E00E9411360E9462
:10C9D0004440811104C00E940A410E94963681E0C1
:10C9E0000E9454388091E60B00E210E046E1D42E1C
:10C9F0000E94E54A2091E60B203109F407C1332754
:10CA000027FD30952F5F3F4F2F71307837FF06C0DD
:10CA100021503109206E3F6F2F5F3F4F822F2093AF
:10CA2000E60B0150110921F781E00E94E54A80E1FF
:10CA30000E94E54A8EE10E94E54A8DE10E94E54AA6
:10CA40000E944E330E94E0448FE397E00E941F3B18
:10CA5000789406ECC02EBB24B39487E8D82E93E4D8
:10CA6000892E20EF922E30EAA32E9FB7F894809162
:10CA7000F3108F5F8093F310C1BA469A80FBEE24C7
:10CA8000E0F8F12CEE0CFF1CEE0CFF1CB1E3EB2ADE
:10CA90008E2D86958270806CB5B8E2E4E8B9F0E539
:10CAA000FBB98EB9D1BA9FBF1092820B1092830B43
:10CAB0001092840B1092850B2FEF2093E70B80913F
:10CAC000E60B0E94E54A2091E60B203109F44BC1A8
:10CAD000332727FD30952F5F3F4F2F71307837FD7B
:10CAE000FEC3822F2093E60B0E94E54A2091E60BBD
:10CAF000203109F433C1332727FD30952F5F3F4F95
:10CB00002F71307837FDE4C3822F2093E60B0E940B
:10CB1000E54A2091E60B203109F41BC1332727FD9C
:10CB200030952F5F3F4F2F71307837FDCAC3822F6A
:10CB30002093E60B0E94E54A8091E60B803109F4D0
:10CB400006C1992787FD909501968F71907897FD82
:10CB5000CDC38093E60B81E00E94E54A80E10E940C
:10CB6000E54A8EE10E94E54A8DE10E94E54A109176
:10CB7000E70B1F3F11F41091BF0F1093BF0F173138
:10CB800009F4A2C08091820B9091830BA091840B39
:10CB9000B091850B0091BE0F2091ED10E4E7F6E017
:10CBA0002223C1F12AE73FE0212E332427FC3094D1
:10CBB000898B9A8BAB8BBC8B22C0462F552747FDA8
:10CBC000509549885A886B887C8804C0769467940D
:10CBD000579447946A95D2F740FE0BC0440F551FF7
:10CBE0004A55544FDA014D915C91D9014D935C93B4
:10CBF00001E02E5F3F4FB6E0E239FB0711F1619192
:10CC00006F3FB9F36113D9CFA101E8CFD092E60B02
:10CC100086E107CFAAE7BFE09D0181918F3F59F0E0
:10CC2000880F990B8A55944FDC018D919C91D90105
:10CC30008D939C9301E02E5F3F4FB6E0E239FB07F6
:10CC400061F70093BE0F1F3F61F1E12FEE0FFF0B65
:10CC5000EA55F44F80819181A0E0B0E04091C00F8F
:10CC60005091C10F6091C20F7091C30F8417950747
:10CC7000A607B707B1F08093C00F9093C10FA093A0
:10CC8000C20FB093C30F0E94DE278091BF0F863181
:10CC900009F4A2C3803109F4B6C38450883008F483
:10CCA00085C34091F3104370423009F4ABC0433068
:10CCB00009F45EC0413009F4F9C10E9443236FEFCB
:10CCC00080E00E949B4DD1CEE091C80FE7FD5ACF86
:10CCD0002091D40B3091D50BA90160E070E08091D8
:10CCE000C00F9091C10FA091C20FB091C30F481710
:10CCF00059076A077B0709F445CFFF27E7FDF09541
:10CD0000CF01880F991F8E0F9F1F880F991F880FC3
:10CD1000991F8C579A4FFC01DE0111961CE001907F
:10CD20000D921A95E1F7DC010C9111961C910111FD
:10CD3000E2C2E12FEE0FFF0BE658F04F3183208364
:10CD4000B092BE0F0E94E0441091BF0F1BCF86E14E
:10CD500000CF56E15093E60B86E1ECCE46E14093DE
:10CD6000E60B86E1D4CE36E13093E60B86E1BCCE0D
:10CD70000E949D4300E010E423E035E440E050EEE3
:10CD80006BE276E48091A60F9091A70F0E94DC3DA4
:10CD90009C019093570F8093560F81E0203D3740C0
:10CDA0000CF080E08093580F8091B40F9091B50FF4
:10CDB0002091F110222309F400C3AC0160E070E07F
:10CDC000DB01CA01880F991FAA1FBB1F880F991F7B
:10CDD000AA1FBB1F880F991FAA1FBB1F840F951F77
:10CDE000A61FB71F880F991FAA1FBB1FFD01EE0FBB
:10CDF000FF1FEE56F94F808191819093B30C809381
:10CE0000B20C5DCF80917C0F90917D0F6FB7F8943D
:10CE10009C01232F332726952695722FC1BA469A57
:10CE2000522F550F452F46704068207133272260DE
:10CE3000352F330F3072322B507C352B272F269510
:10CE40002270206215B848B93BB92EB9D1BA96956F
:10CE5000879596958795282FC1BA469A482F440FF3
:10CE6000382F3695221F2227221F542F5670252B2C
:10CE70002068807199278260942F990F9072982B67
:10CE8000407C942B327015B828B99BB93EB9D1BA01
:10CE9000C1BA469AB5B888B89BB8AEB8D1BA45E021
:10CEA0004A95F1F70000C1BA469AB5B888B850E77C
:10CEB0005BB9AEB8D1BA8AE08A95F1F700C0C1BAC1
:10CEC000469AB5B888B89BB8AEB8D1BA9AE09A95E8
:10CED000F1F700C06FBF8091820F9091830F6FB701
:10CEE000F8949C01232F332726952695E22FC1BA6B
:10CEF000469A722F770F472F46704068207133276C
:10CF00002260372F330F3072322B707C372B2E2F4D
:10CF100026952270206215B848B93BB92EB9D1BA0E
:10CF20009695879596958795282FC1BA469A482F4A
:10CF3000440F382F3695221F2227221F742F767018
:10CF4000272B2068807199278260942F990F907207
:10CF5000982B407C942B327015B828B99BB93EB9F8
:10CF6000D1BAC1BA469AB5B885E488B99BB8AEB80B
:10CF7000D1BAA5E0AA95F1F70000C1BA469AB5B8B2
:10CF800088B95BB9AEB8D1BABAE0BA95F1F700C0CA
:10CF9000C1BA469AB5B888B99BB8AEB8D1BAEAE07A
:10CFA000EA95F1F700C06FBF2091C20B3091C30B1F
:10CFB0008091540F9091550FAA2797FDA095BA2FF5
:10CFC000820F931FA11DB11DB7FDF3C10097F1E0C2
:10CFD000AF07B10524F08FEF9FEFA0E0B0E05FB79F
:10CFE000F8949C01232F332726952695722FC1BADA
:10CFF000469A622F660F462F46704068207133278D
:10D000002260362F330F3072322B607C362B272F65
:10D0100026952270206215B848B93BB92EB9D1BA0D
:10D020009695879596958795282FC1BA469A482F49
:10D03000440F382F3695221F2227221F642F667037
:10D04000262B2068807199278260942F990F907207
:10D05000982B407C942B327015B828B99BB93EB9F7
:10D06000D1BAC1BA469AB5B887E488B99BB8AEB808
:10D07000D1BA25E02A95F1F70000C1BA469AB5B8B1
:10D0800088B990E79BB9AEB8D1BA3AE03A95F1F7D2
:10D0900000C0C1BA469AB5B888B99BB8AEB8D1BA83
:10D0A0004AE04A95F1F700C05FBF09CE8091A00F1A
:10D0B0009091A10F6FB7F8949C01232F33272695E9
:10D0C0002695E22FC1BA469A722F770F572F5670C6
:10D0D0005068207133272260372F330F3072322B84
:10D0E000707C372B2E2F26952270206215B858B9E8
:10D0F0003BB92EB9D1BA9695879596958795282FE5
:10D10000C1BA469A582F550F382F3695221F22271D
:10D11000221F752F7670272B2068807199278260D7
:10D12000952F990F9072982B507C952B327015B8D3
:10D1300028B99BB93EB9D1BAC1BA469A45B981E47A
:10D1400088B99BB8AEB8D1BAE5E0EA95F1F700002E
:10D15000C1BA469A45B988B950E75BB9AEB8D1BAF9
:10D16000FAE0FA95F1F700C0C1BA469A45B988B914
:10D170009BB8AEB8D1BA2AE02A95F1F700C06FBFCC
:10D1800080918A0F90918B0F6FB7F8949C01232F99
:10D19000332726952695F22FC1BA469AE22FEE0F35
:10D1A0007E2F767070682071332722603E2F330FF8
:10D1B0003072322BE07C3E2B2F2F2695227020627E
:10D1C00015B878B93BB92EB9D1BA96958795969589
:10D1D0008795282FC1BA469A782F770F382F369522
:10D1E000221F2227221FE72FE6702E2B2068807136
:10D1F00099278260972F990F9072982B707C972BAC
:10D20000327015B828B99BB93EB9D1BAC1BA469A9D
:10D2100045B995E498B99BB882EA8EB9D1BA35E0A0
:10D220003A95F1F70000C1BA469A45B998B95BB989
:10D230008EB9D1BAAAE0AA95F1F700C0C1BA469A50
:10D2400045B998B99BB88EB9D1BABAE0BA95F1F799
:10D2500000C06FBF2FB7F894C1BA469A15B890E8CE
:10D2600098B932E33BB930E23EB9D1BAC1BA469A75
:10D2700015B898B992E09BB91EB8D1BAC1BA469A0E
:10D2800045B988B89BB88EB9D1BAE5E0EA95F1F70F
:10D290000000C1BA469A45B988B85BB98EB9D1BA0F
:10D2A000FAE0FA95F1F700C0C1BA469A45B988B8D4
:10D2B0009BB88EB9D1BA3AE03A95F1F700C02FBFCA
:10D2C000FECC21503109206E3F6F2F5F3F4F2FCC96
:10D2D00021503109206E3F6F2F5F3F4F15CC2150F9
:10D2E0003109206E3F6F2F5F3F4FFBCB0197806E60
:10D2F0009F6F01962ECC033008F022CD2D875E87DC
:10D300006F87788B0E949C3C8D819E814D855E85C8
:10D310006F857889892B09F4A4C08F819885892B22
:10D3200009F489C089859A85892B09F480C08B8589
:10D330009C85892B09F485C0440F551F661F771FF4
:10D34000440F551F661F771F2B01772457FC7094DD
:10D35000672C8091C40F9091C50FA091C60FB0911A
:10D36000C70F481659066A067B0671F0F20132961D
:10D37000EE0FFF1F21E030E02C0F3D1FE20FF31FE7
:10D38000808191810E941F3B0130B9F5E12FFF2779
:10D39000E7FDF095E05AF04F40824092C40F509262
:10D3A000C50F6092C60F7092C70FCACC0E94CC1BEB
:10D3B00078CC80E090E0DC0109CE00E010E02AEFBC
:10D3C00033E440E050EE6BEA76E40E94DC3D90935B
:10D3D000B30C8093B20C73CC0091D20B1091D30B91
:10D3E00010932D0F00932C0F0E94432342E0B801AD
:10D3F00080E090E00E94351454CCB301A201812F4B
:10D400000E94B53CCACF0E94864A8C0190932F0F90
:10D4100080932E0F0E946A166FEF81E00E949B4D51
:10D4200041E060E070E0C8010E9435143ACC440F3E
:10D43000551F661F771F2B01772457FC7094672CAC
:10D4400088CF2A013B01440C551C661C771C440EF6
:10D45000551E661E771E2301772457FC7094672C97
:10D4600078CF412C512C320174CFB2D4B7FF08953C
:10D47000821B930B089597FB072E16F4009406D099
:10D4800077FD08D00BD007FC05D03EF49095819530
:10D490009F4F0895709561957F4F0895AA1BBB1B00
:10D4A00051E107C0AA1FBB1FA617B70710F0A61BA4
:10D4B000B70B881F991F5A95A9F780959095BC01C5
:10D4C000CD0108955058BB27AA270ED0C9C192D1CB
:10D4D00030F097D120F031F49F3F11F41EF462C177
:10D4E0000EF4E095E7FB58C1E92FDCD180F3BA17C1
:10D4F000620773078407950718F071F49EF5F4C16D
:10D500000EF4E0950B2EBA2FA02D0B01B90190015E
:10D510000C01CA01A0011124FF27591B99F0593FA2
:10D5200050F4503E68F11A16F040A22F232F342FEA
:10D530004427585FF3CF469537952795A795F04038
:10D540005395C9F77EF41F16BA0B620B730B840B4D
:10D55000BAF09150A1F0FF0FBB1F661F771F881F05
:10D56000C2F70EC0BA0F621F731F841F48F487955D
:10D5700077956795B795F7959E3F08F0B3CF93954C
:10D58000880F08F09927EE0F97958795089541D158
:10D59000E39577C10CD064C134D140F02BD130F089
:10D5A00021F45F3F19F0F8C051119FC1FBC07AD13F
:10D5B00098F39923C9F35523B1F3951B550BBB275A
:10D5C000AA2762177307840738F09F5F5F4F220F07
:10D5D000331F441FAA1FA9F333D00E2E3AF0E0E800
:10D5E00030D091505040E695001CCAF729D0FE2F4C
:10D5F00027D0660F771F881FBB1F261737074807DE
:10D60000AB07B0E809F0BB0B802DBF01FF27935893
:10D610005F4F2AF09E3F510568F0BEC066C15F3F74
:10D62000ECF3983EDCF3869577956795B795F7957B
:10D630009F5FC9F7880F911D9695879597F9089573
:10D64000E1E0660F771F881FBB1F6217730784070F
:10D65000BA0720F0621B730B840BBA0BEE1F88F71E
:10D66000E095089519F40EF097C03EC19BC022D1F9
:10D67000C8F39638C0F707F80F92E8942BE33AEA1C
:10D6800048EB5FE7BAD10F920F920F924DB75EB79A
:10D690000F9272D1ECEAF0E088D04F915F91EF9158
:10D6A000FF91E595EE1FFF1F49F0FE57E068442704
:10D6B000EE0F441FFA95E1F74195550B29D10F90D4
:10D6C00007FE1DC10895F6D088F09F5790F0B92F3E
:10D6D0009927B751A0F0D1F0660F771F881F991FC7
:10D6E0001AF0BA95C9F712C0B13081F0FDD0B1E09F
:10D6F0000895FAC0672F782F8827B85F39F0B93FAF
:10D70000CCF3869577956795B395D9F73EF49095C8
:10D710008095709561957F4F8F4F9F4F0895E89446
:10D7200009C097FB3EF490958095709561957F4F69
:10D730008F4F9F4F9923A9F0F92F96E9BB27939517
:10D74000F695879577956795B795F111F8CFFAF427
:10D75000BB0F11F460FF1BC06F5F7F4F8F4F9F4F58
:10D7600016C0882311F096E911C0772321F09EE8B6
:10D77000872F762F05C0662371F096E8862F70E01C
:10D7800060E02AF09A95660F771F881FDAF7880FF6
:10D790009695879597F9089597F99F6780E870E0C7
:10D7A00060E008959FEF80EC0895DF93CF931F937F
:10D7B0000F93FF92EF92DF927B018C01689405C07A
:10D7C000DA2EEF0118D1FE01E894A591259135914B
:10D7D00045915591AEF3EF0187DEFE019701A80157
:10D7E000DA9479F7DF90EF90FF900F911F91CF912E
:10D7F000DF91089500240A941616170618060906E4
:10D80000089500240A9412161306140605060895B6
:10D81000C9CF50D0E8F3E894E0E0BB279F57F0F081
:10D820002AED3FE049EC06C0EE0FBB0F661F771FE5
:10D83000881F28F0B23A62077307840728F0B25AAB
:10D84000620B730B840BE3959A9572F7803830F472
:10D850009A95BB0F661F771F881FD2F7904894C117
:10D86000092E0394000C11F4882352F0BB0F40F4EE
:10D87000BF2B11F460FF04C06F5F7F4F8F4F9F4F2E
:10D880000895EF93E0FF06C0A2EA2AED3FE049ECDD
:10D890005FEB2ADEE5DF0F90039401FC9058E4ED86
:10D8A000F0E07EC157FD9058440F551F59F05F3F7F
:10D8B00071F04795880F97FB991F61F09F3F79F0B2
:10D8C00087950895121613061406551FF2CF469534
:10D8D000F1DF08C0161617061806991FF1CF8695B6
:10D8E0007105610508940895E894BB27662777279A
:10D8F000CB0197F9089522D108F48FEF08959B0189
:10D90000AC0160E070E080E89FE344CE45CF3AC1CF
:10D91000D1DFE8F39923D9F3940F511DBBF3915054
:10D92000504094F059F0882332F0660F771F881F1B
:10D9300091505040C1F79E3F510544F7880F911D0B
:10D940009695879597F908955F3FACF0983E9CF0C7
:10D95000BB27869577956795B79508F4B160939541
:10D96000C1F7BB0F58F711F460FFE8CF6F5F7F4F2F
:10D970008F4F9F4FE3CFB9CFFA01DC01AA0FBB1F36
:10D980009B01AC01BF5728F4222733274427507846
:10D990001FC0B75188F4AB2F0024469537952795C3
:10D9A000011CA395D2F3002069F0220F331F441FFE
:10D9B000B395DAF30DD086CD61307105A0E88A0702
:10D9C000B94630F49B01AC01662777278827907809
:10D9D000309621F0208331834283538308950BD006
:10D9E0003FCF08DF28F00DDF18F0952309F0D4CEE3
:10D9F000D9CE11247ACF56DFA0F3959FD1F3950F9E
:10DA000050E0551F629FF001729FBB27F00DB11DC2
:10DA1000639FAA27F00DB11DAA1F649F6627B00D52
:10DA2000A11D661F829F2227B00DA11D621F739F3B
:10DA3000B00DA11D621F839FA00D611D221F749F49
:10DA40003327A00D611D231F849F600D211D822F90
:10DA5000762F6A2F11249F5750408AF0E1F08823D7
:10DA60004AF0EE0FFF1FBB1F661F771F881F9150E4
:10DA70005040A9F79E3F510570F08ECE36CF5F3FE4
:10DA8000ECF3983EDCF3869577956795B795F79517
:10DA9000E7959F5FC1F7FE2B880F911D969587959F
:10DAA00097F90895FA01EE0FFF1F30962105310511
:10DAB00099F16115710561F48038BFE39B0749F165
:10DAC00068949038810561F08038BFEF9B0741F082
:10DAD000992342F5FF3FE1053105210511F1E89455
:10DAE0000894E795D901AA2329F4AB2FBE2FF85F3C
:10DAF000D0F310C0FF5F70F4A695E0F7F73950F04F
:10DB000019F0FF3A38F49F779F930CD00F9007FCE1
:10DB1000905808953EF046CE60E070E080E89FE3C4
:10DB200008954FE79F775F934F933F932F934ED086
:10DB30002F913F914F915F9152DF99CD990F00083E
:10DB4000550FAA0BE0E8FEEF16161706E807F907CF
:10DB5000C0F012161306E407F50798F0621B730B6A
:10DB6000840B950B39F40A2661F0232B242B252BEB
:10DB700021F408950A2609F4A140A6958FEF811D8E
:10DB8000811D08959F3F31F0915020F4879577953E
:10DB90006795B795880F911D9695879597F9089584
:10DBA0009F938F937F936F93FF93EF939B01AC01B0
:10DBB00016DFEF91FF91F9DD2F913F914F915F912A
:10DBC0000ECF0EF0DFCFEECD6894E6CD73DEC8F356
:10DBD0009923D1F3C6F3DF93CF931F930F93FF9253
:10DBE000C92FDD2788232AF02197660F771F881F0A
:10DBF000DAF720E030E040E85FEB9FE3883920F07F
:10DC0000803E30F021968F775EDCE2EFF0E003C0DB
:10DC10005ADCEFE1F1E0C9DD8B01BE01EC01FB2E26
:10DC20006F5771097595771F880B990B7ADD28E17D
:10DC300032E741E35FE3DFDEAF2D9801AE01FF90F5
:10DC40000F911F91CF91DF914FDC0ACEFB01DC01D8
:10DC500004C08D910190801921F441505040C8F7C3
:10DC6000881B990B0895FB01DC0102C001900D9205
:10DC700041505040D8F708956817790768F4FB01C0
:10DC8000DC01E40FF51FA40FB51F02C002900E9235
:10DC900041505040D8F70895E6CFDC0101C06D93A4
:10DCA00041505040E0F70895FB01DC010D90002049
:10DCB000E9F7119701900D920020E1F70895FB011B
:10DCC000DC0101900D920020E1F708958F929F9260
:10DCD000AF92BF92CF92DF92EF92FF92CF93DF93FA
:10DCE000EC01688179818A819B81611571058105CB
:10DCF000910521F464E279ED8BE597E02DE133EFB6
:10DD000041E050E04AD049015A019B01AC01A7EA29
:10DD1000B1E433D06B017C01ACEEB4EFA50194010A
:10DD200038D0C60ED71EE81EF91EF7FE06C081E0E9
:10DD3000C81AD108E10880E8F80AC882D982EA82C4
:10DD4000FB82E894F7F8B601C701DF91CF91FF900D
:10DD5000EF90DF90CF90BF90AF909F908F900895FD
:10DD6000B5CF80E891E0B2CF6093800170938101DC
:10DD7000809382019093830108952AD0A59F900DEE
:10DD8000B49F900DA49F800D911D11240895B7FF9D
:10DD9000F4CFF3DF821B930B0895052E97FB16F447
:10DDA000009406D057FD0CD01FD007FC09D07EF49C
:10DDB00090958095709561957F4F8F4F9F4F0895F7
:10DDC00050954095309521953F4F4F4F5F4F0895A7
:10DDD000A29FB001B39FC001A39F01D0B29F700D5D
:10DDE000811D1124911D0895A1E21A2EAA1BBB1BAF
:10DDF000FD010DC0AA1FBB1FEE1FFF1FA217B30717
:10DE0000E407F50720F0A21BB30BE40BF50B661F2C
:10DE1000771F881F991F1A9469F7609570958095F0
:10DE200090959B01AC01BD01CF010895F894FFCFFF
:10DE300000000000000000000000000000000000E2
:10DE400000000000000000000000000000000000D2
:10DE5000003022366D247D20390F76461040105256
:10DE60003F065B4F666D7D077F6F484861484327DB
:10DE70007B777F393F79713D76060E763837373FAD
:10DE8000733F776D783E3E7E76665B39640F23087C
:10DE900002777C585E79716F74040C743837545C67
:10DEA0007367506D781C1C7E766E5B39300F0100F5
:10DEB0000100000000006207640E3415D21B4122ED
:10DEC0008128942E7B34383ACB3F37457B4A994F93
:10DED000925467591A5EAB621A676A6B9B6FAD7397
:10DEE000A2777B7B387FD9826186CF89258D62902E
:10DEF000889398969199759C449FFFA1A6A43AA7F0
:10DF0000BBA92AAC88AED5B011B33DB559B766B937
:10DF100064BB54BD36BF0BC1D2C28CC43AC6DCC789
:10DF200072C9FDCA7CCCF1CD5BCFBBD011D25ED320
:10DF3000A1D4DBD50CD734D854D96DDA7DDB85DCA0
:10DF400086DD80DE73DF5FE044E123E2FCE2CEE3C6
:10DF50009BE461E522E6DEE695E746E8F2E89AE929
:10DF60003DEADBEA74EB0AEC9BEC28EDB1ED36EE12
:10DF7000B8EE36EFB0EF27F09AF00BF178F1E2F15E
:10DF800049F2ADF20EF36DF3C9F322F479F4CDF456
:10DF90001FF56FF5BCF507F651F698F6DDF620F79C
:10DFA00061F7A0F7DEF71AF854F88DF8C4F8F9F81D
:10DFB0002DF95FF990F9C0F9EEF91BFA47FA71FAF9
:10DFC0009BFAC3FAEAFA10FB35FB58FB7BFB9DFB7F
:10DFD000BEFBDEFBFDFB1BFC38FC55FC70FC8BFC28
:10DFE000A5FCBFFCD8FCF0FC07FD1EFD34FD49FD7F
:10DFF0005EFD72FD86FD99FDABFDBDFDCFFDE0FD33
:10E00000F0FD01FE10FE1FFE2EFE3CFE4AFE58FEF5
:10E0100065FE72FE7EFE8AFE96FEA2FEADFEB7FE95
:10E02000C2FECCFED6FEE0FEE9FEF2FEFBFE04FFE1
:10E030000CFF14FF1CFF23FF2BFF32FF39FF40FFB3
:10E0400047FF4DFF53FF59FF5FFF65FF6BFF70FFF9
:10E0500075FF7BFF80FF84FF89FF8EFF92FF96FF95
:10E060009BFF9FFFA3FFA7FFAAFFAEFFB1FFB5FF76
:10E07000B8FFBBFFBFFFC2FFC5FFC8FFCAFFCDFF90
:10E08000D0FFD2FFD5FFD7FFDAFFDCFFDEFFE0FFD6
:10E09000E3FFE5FFE7FFE9FFEAFFECFFEEFFF0FF3C
:10E0A000F1FFF3FFF5FFF6FFF8FFF9FFFBFFFCFFC1
:10E0B000FDFFFFFF0000EE01DA03C305A9078C098D
:10E0C0006C0B4A0D250FFD10D212A41474164118C2
:10E0D0000B1AD31B981D5A1F1A21D72291244926A7
:10E0E000FE27B129612B0E2DB92E62300832AB33D9
:10E0F0004D35EB368738213AB93B4E3DE03E714015
:10E10000FE418A4313459A461F48A149224B9F4C22
:10E110001B4E944F0C518152F4536455D3563F58C3
:10E12000A959115B775CDB5D3D5F9C60FA615663CA
:10E13000AF6407665C67B068016A516B9E6CEA6DFC
:10E14000346F7B70C171057347748775C57602782B
:10E150003C79757AAC7BE17C147E457F7580A38128
:10E16000CF82F983218548866D879188B289D28ACA
:10E17000F18B0D8D288E418F59906F9183929693DC
:10E18000A794B695C496D197DB98E599EC9AF29B43
:10E19000F79CFA9DFB9EFB9FFAA0F7A1F2A2ECA3CD
:10E1A000E5A4DCA5D2A6C6A7B9A8AAA99AAA88AB55
:10E1B00076AC61AD4CAE35AF1CB003B1E7B1CBB2BC
:10E1C000ADB38EB46EB54CB629B705B8DFB8B8B9E3
:10E1D00090BA67BB3CBC10BDE3BDB4BE85BF54C0A4
:10E1E00022C1EEC1BAC284C34DC415C5DCC5A2C6E6
:10E1F00066C729C8ECC8ADC96DCA2BCBE9CBA5CC85
:10E2000061CD1BCED4CE8DCF44D0FAD0AFD162D267
:10E2100015D3C7D378D427D5D6D584D630D7DCD775
:10E2200086D830D9D9D980DA27DBCCDB71DC15DD93
:10E23000B7DD59DEFADE9ADF39E0D7E074E110E2AB
:10E24000ACE246E3DFE378E410E5A6E53CE6D1E6A0
:10E2500065E7F9E78BE81CE9ADE93DEACCEA5AEB62
:10E26000E7EB74EC00ED8AED14EE9EEE26EFAEEFD8
:10E2700035F0BBF040F1C4F148F2CBF24DF3CEF3F0
:10E280004FF4CFF44EF5CCF54AF6C7F643F7BEF798
:10E2900039F8B3F82CF9A5F91DFA94FA0AFB80FBBA
:10E2A000F5FB6AFCDDFC50FDC3FD34FEA5FE16FF48
:10E2B00085FFF4FF001D670700000000000000005C
:10E2C00002006D07770781078A070000001A94078C
:10E2D0000000000000000000001B9C070000000080
:10E2E000000000000019A40700000000000000006A
:10E2F0000202AE07B807C107CA07D2070114DA073E
:10E30000C108E307E707EB070016EF07000000006E
:10E3100000000000001CF5070000000000000000E5
:10E320000017FC070000000000000000001D670748
:10E330000000000000000000020105080D081008A0
:10E340000E080000010A12081C0820080000000046
:10E35000020525082F081C08200833080117380873
:10E36000400844080000000002034808B807C1073D
:10E37000CA07D207020452085D08610865086908E7
:10E3800001126D0872081C082008000001167708A9
:10E390007D0882088B080000001892080000000029
:10E3A000000000001E00181D0C0D1F0102030405D3
:10E3B000060708090A0B191B1A1CFFFFFFFFFFFFC6
:10E3C000FFFF8001C000A8009000800060004800AE
:10E3D00030002400180012000C00090006000400A0
:10E3E0000300020001000D09120916091A091E098D
:10E3F000220926092A092E09320936093B09400952
:10E4000045094A094F0954090101010101010101AE
:10E4100001030206020101010101020402030201DB
:10E42000020000FFFFFFFFFF080C080A08080808A9
:10E4300008080808080A080C0C0000000000080C76
:10E440000A0A0A0A0A0C0C08020302000001000171
:10E4500001010101000101010204081020408000B7
:10E460003756656F7C878B8F949AA4B0B9BFD2471B
:10E470006C69476C6927732050363030207570679F
:10E480007261646520616C7068612053657020332F
:10E49000302032303134007370656564006C666F13
:10E4A0002073686170650070756C73652D74726996
:10E4B0000072616E642D73696E006E6F6973652DF5
:10E4C0007361770056696220737064005669622038
:10E4D000616D74006D6F642064656C617900616DBD
:10E4E0007020736861706500666173742D65787063
:10E4F00000666173742D6C696E00736C6F2D6578A6
:10E500007000736C6F2D6C696E0062656E642074B0
:10E5100067740056636F0056636600566F6C006741
:10E520006C69646500646574756E6500616D70206A
:10E5300056656C6F006C666F2074677400616200D2
:10E5400061006C666F2072616E6765006C6F7700AA
:10E5500068696768006D6F642072616E6765006D41
:10E56000696E0066756C6C006D6F64207467740072
:10E570006C666F005669620066696C207368617032
:10E58000650062656E642072616E676500326E645C
:10E590000033726400357468004F637400707269F0
:10E5A0006F006C61737400706974636800667265F3
:10E5B000650073656D69746F6E65006F6374615695
:10E5C000650066696C2056656C6F00207265637625
:10E5D000002073656E640062656E6465722063611D
:10E5E0006C696272617465640056632D0056632D18
:10E5F000206F66660056632D206F6E007072657323
:10E600006574732064756D70656400496E74207361
:10E61000796E63004D6964692073796E630074617B
:10E6200070652073796E6300737072656164206F2A
:10E630006E00737072656164206F6666006F6D6E48
:10E64000690063683100636832006368330063689F
:10E6500034006368350063683600636837006368B8
:10E660003800636839006368313000636831310015
:10E6700063683132006368313300636831340063AA
:0EE68000683135006368313600203D2000000F
:020000021000EC
:10E000002F923F924F925F926F927F928F929F9248
:10E01000AF92BF92CF92DF92EF92FF920F931F9336
:10E02000CF93DF93CDB7DEB72A970FB6F894DEBF54
:10E030000FBECDBF2FEF31EE44E0215030404040C5
:10E04000E1F700C00000F89414B817B81AB81DB86A
:10E0500010BA15B890EE98B91BB81EB883EE81BB04
:10E060002FEF24B997B947E04AB99DB980BB36EC88
:10E0700031BB469A97B94AB99DB915B880E888B9B5
:10E080001BB81EB8F7E4F1BB52E05A95F1F700C097
:10E0900086B189B18CB131BB479AE7EEE7B977EF2A
:10E0A0007AB962EE6DB931BB469AA1E0A5B982E4B6
:10E0B00088B91BB81EB887E881BB8DE08A95F1F757
:10E0C000000031BB469A97B94AB99DB9A5B920E479
:10E0D00028B91BB82EB9F1BBB2E0BA95F1F700C070
:10E0E00086B159B1BCB131BB479AE7B97AB96DB9BC
:10E0F000BDE0BA95F1F7000031BB469A97B94AB92D
:10E100009DB9A5B928B91BB82EB9F1BBF2E0FA95B3
:10E11000F1F700C026B199B14CB131BB479AE7B9CC
:10E120007AB96DB93DE03A95F1F70000422F469576
:10E13000437060E8269F90011124242B392F307101
:10E14000322B292F269526952870232B969590768D
:10E15000922B907C21E0903C09F020E0382F3695FE
:10E160003370A0E88A9FC0011124832B952F9071F2
:10E17000982B852F869586958870982B852F869568
:10E180008076982B907C81E0903C09F080E082239F
:10E1900009F4B4C286EC81BB469A21E025B990E42B
:10E1A00098B99BB91EB897E891BBBAE0BA95F1F758
:10E1B00000C081BB469A25B934E438B930E73BB991
:10E1C00032E23EB991BBEAE0EA95F1F700C081BBCB
:10E1D000469A25B922E428B920E52BB920EC2EB9BE
:10E1E00091BBFAE0FA95F1F700C081BB469A15B8E9
:10E1F00026E828B923E02BB91EB891BBAFE9BFE0F0
:10E200001197F1F700C0000081BB469A15B823E8CA
:10E2100028B923E12BB922E02EB991BBBAE0BA9517
:10E22000F1F700C081BB469A20EE27B997E09AB972
:10E230002DB915B870E878B99BB91EB867E461BB11
:10E24000E2E0EA95F1F700C036B139B13CB181BBEB
:10E25000479A57EE57B947EF4AB932EE3DB9F5E064
:10E26000FA95F1F7000081BB469A27B99AB92DB902
:10E2700015B878B99BB990E29EB961BB22E02A95A6
:10E28000F1F700C096B199B19CB181BB479A57B9DB
:10E290004AB93DB935E03A95F1F7000099249394D5
:10E2A000612C712C0F2EF1E14F2EF3E15F2EF02D3A
:10E2B0000F2EF1E12F2EF4E13F2EF02D88248394D0
:10E2C0009FD499230CF405C2803F9105C9F798D4D7
:10E2D000892B09F0FEC194D48136910509F0F9C16A
:10E2E0008FD4469709F0F5C18BD48B36910509F090
:10E2F000F0C186D499230CF4ECC1A3015827052E54
:10E300000294202D2F702527352F3025330F307E96
:10E310002327302D3527307F3695052E000C331FEF
:10E320005695569556955F7153275427422F7A017B
:10E330008F7799278C011695102F00271795079531
:10E340005FD499230CF4C5C1D701B8270B2E0294D2
:10E35000202D2F702B273B2F3025330F307E232786
:10E36000302D3B27307F36950B2E000C331FB69592
:10E37000B695B695BF71B327BA27A22F7D018F77C7
:10E380009927082B192B0115B1E01B0721F0012B50
:10E3900009F4A1C19EC134D46C0199230CF499C134
:10E3A00087011827012E0294802D8F708127912FCD
:10E3B0009025990F907E8927902D9127907F969593
:10E3C000012E000C991F1695169516951F71192789
:10E3D0001027082F15D45C0199230CF47AC1F80199
:10E3E000F8270F2E0294802D8F708F279F2F902556
:10E3F000990F907E8927902D9F27907F96950F2EBD
:10E40000000C991FF695F695F695FF71F927FE27F2
:10E41000E82FFA87E9878201F3D399230CF4F4C03B
:10E42000E984FA84A7015827052E0294202D2F7025
:10E430002527352F3025330F307E2327302D3527E4
:10E44000307F3695052E000C331F56955695569500
:10E450005F7153275427422F7A015A874987DC017D
:10E46000AF77BB27BA83A983CBD399230CF4CCC055
:10E47000F701F8270F2E0294202D2F702F273F2F02
:10E480003025330F307E2327302D3F27307F3695C0
:10E490000F2E000C331FF695F695F695FF71F327B6
:10E4A000FE27E22F7F01FA87E9879C012F77332728
:10E4B0003C832B83A5D399230CF4A6C0A70158272E
:10E4C000052E0294202D2F702527352F3025330F50
:10E4D000307E2327302D3527307F3695052E000CD2
:10E4E000331F5695569556955F7153275427422FE3
:10E4F0007A015A874987DC01AF77BB27BE83AD839A
:10E500007FD399230CF480C0F701F8270F2E0294D3
:10E51000202D2F702F273F2F3025330F307E2327BC
:10E52000302D3F27307F36950F2E000C331FF69588
:10E53000F695F695FF71F327FE27E22F7F01FA8704
:10E54000E9879C012F77332738872F8359D3992365
:10E550000CF45AC0A7015827052E0294202D2F70C5
:10E560002527352F3025330F307E2327302D3527B3
:10E57000307F3695052E000C331F569556955695CF
:10E580005F7153275427422F5A874987F8013397E1
:10E590009C013695322F2227379527955981252BB7
:10E5A0002083F80132979C0122703327002436958E
:10E5B00027950794369527950794322F202D6B8148
:10E5C000262B2083F80131979C0124703327220FDA
:10E5D000331F22953295307F3227207F3227AD813D
:10E5E0002A2B20838870992782959295907F98276F
:10E5F000807F9827BF818B2BF80180830C5F1F4F92
:10E600000215130509F008CFFBD299230CF461C061
:10E610008C01102F0027110FF3D299230CF459C04D
:10E620008F779927880F991F880F991F082B192B0F
:10E63000E7D299230CF44DC083709927082B192B2E
:10E6400029853A850217130709F043C0D9D2873FBD
:10E65000910509F03EC0990C3FE3391508F4982C58
:10E6600046EC41BB469A892D880F392D3695282FC7
:10E6700026702064992D991F9927991F292B992D70
:10E680009071482F440F4072942B807C982B832FDD
:10E690008270806285B828B99BB98EB957E851BBA2
:10E6A0006AE06A95F1F700C0B5016F777727C60178
:10E6B0008F7799279695982F882797958795682B18
:10E6C000792B762F662780E090E04EE053E198D4D6
:10E6D000F7CD89E701C08DE696EC91BB469A982F5D
:10E6E0009071906E86958270806221E025B922E457
:10E6F00028B99BB98EB987E881BBFFCF2A960FB6A0
:10E70000F894DEBF0FBECDBFDF91CF911F910F9167
:10E71000FF90EF90DF90CF90BF90AF909F908F9041
:0EE720007F906F905F904F903F902F900895E4
:10EC000045E04A95F1F70000349B04C000C000C005
:10EC10003499FCCF86EC81BB469A20EE27B997E069
:10EC20009AB92DB915B820E828B99BB91EB897E450
:10EC300091BB52E05A95F1F700C096B129B13CB1B1
:10EC400081BB479A87EE87B987EF8AB982EE8DB983
:10EC500085E08A95F1F70000392F3695337040E84A
:10EC6000949FC0011124832B922F9071892B922F96
:10EC7000969596959870892B26952076282B217B42
:10EC8000213809F040C026EC21BB469A90EE97B996
:10EC900087E08AB99DB915B890E898B98BB980E238
:10ECA0008EB987E481BB52E05A95F1F700C036B1C6
:10ECB00099B14CB121BB479A87EE87B987EF8AB9E2
:10ECC00082EE8DB985E08A95F1F70000832F869555
:10ECD000837050E8359F90011124282B892F807173
:10ECE000282B892F869586958870282B9695907667
:10ECF000292B50E0CA01880F991F84709927822B15
:10ED0000282F30E002C02FEF3FEF822F932F08957E
:10F000008F929F92AF92BF92CF92EF92FF92CF9347
:10F01000DF93EA01CFB6F894F999FECF23E0FB0124
:10F0200080935B002093570010D707B600FCFDCFFC
:10F03000DE01B3954B015C0121E04881F980E12CB0
:10F04000F701E40FF11DAF0122960A01F401A0922D
:10F050005B0020935700F9D61124F2E08F0E911C2B
:10F06000A11CB11CAC17BD0741F725E0FB01809343
:10F070005B0020935700E9D607B600FCFDCF81E185
:10F0800080935700E2D6CFBEDF91CF91FF90EF90F3
:0CF09000CF90BF90AF909F908F9008959C
:00000001FF
